:020000040106F3
:1000000000000000000000000000000000000000F0
:1000100000000000000000000000000000000000E0
:1000200000000000000000000000000000000000D0
:1000300000000000000000000000000000000000C0
:10040000C01F002181220601811906015522060123
:1004100055220601552206015522060155220601E4
:10042000000000000000000000000000851A060126
:1004300055220601000000000D1A0601413D06018B
:10044000E51B0601E51B0601E51B0601E51B060190
:10045000E51B0601E51B0601E51B0601E51B060180
:10046000E51B0601E51B0601E51B0601E51B060170
:10047000E51B0601E51B0601E51B0601E51B060160
:10048000E51B0601E51B0601E51B0601E51B060150
:10049000E51B0601E51B0601E51B0601E51B060140
:1004A000E51B0601E51B0601E51B0601E51B060130
:1004B000E51B0601E51B0601E51B0601E51B060120
:1004C000E51B0601E51B0601E51B0601E51B060110
:1004D000E51B0601E51B0601E51B0601E51B060100
:1004E000E51B0601E51B0601E51B0601E51B0601F0
:1004F000E51B0601E51B0601E51B0601E51B0601E0
:10050000E51B0601E51B0601E51B0601E51B0601CF
:10051000E51B0601E51B0601E51B0601E51B0601BF
:10052000E51B0601E51B0601E51B0601E51B0601AF
:10053000E51B0601E51B0601E51B0601E51B06019F
:10054000E51B0601E51B0601E51B0601E51B06018F
:10055000E51B0601E51B0601E51B0601E51B06017F
:10056000E51B0601E51B0601E51B0601E51B06016F
:10057000E51B0601E51B0601E51B0601E51B06015F
:10058000E51B0601E51B0601E51B0601E51B06014F
:10059000E51B0601E51B0601E51B0601E51B06013F
:1005A000E51B0601E51B0601E51B0601E51B06012F
:1005B000E51B0601E51B0601E51B0601E51B06011F
:1005C000E51B0601E51B0601E51B0601E51B06010F
:1005D000E51B0601E51B0601E51B0601E51B0601FF
:1005E000E51B0601E51B0601E51B0601E51B0601EF
:1005F000E51B0601E51B0601E51B0601E51B0601DF
:10060000E51B0601E51B0601E51B0601E51B0601CE
:10061000E51B0601E51B0601E51B0601E51B0601BE
:10062000E51B0601E51B0601E51B0601E51B0601AE
:10063000E51B0601E51B0601E51B0601E51B06019E
:100640000A49C0F307230246C0B2CB5C095C0B44E5
:10065000162B08DC0C2043430549C818CB589A4296
:1006600018BF002070470020704700BFD0D406019B
:10067000F8280021F8B506460F461725054C2368D3
:1006800013B139462046B047013D04F10C04F6D1C0
:10069000F8BD00BFF82800210000000000000000A5
:1006A000000000000000000000000000000000004A
:1006B000000000000000000000000000000000003A
:1006C000000000000000000000000000000000002A
:1006D000000000000000000000000000000000001A
:1006E000000000000000000000000000000000000A
:1006F00000000000000000000000000000000000FA
:1007000000000000000000000000000000000000E9
:1007100000000000000000000000000000000000D9
:1007200000000000000000000000000000000000C9
:1007300000000000000000000000000000000000B9
:10074000C3438B4210B50ED332F01F030BD10139D6
:1007500002F014030144102B81EA00043DD004DCB4
:1007600063B1042B32D0002041E0142BFBD11F2CAD
:1007700040E8C0F30CD941E8C0F105E01F2C40E887
:1007800000F305D941E800F11C460B468C42EAD142
:1007900022F01402013A0A2AE5D801A151F822F008
:1007A000FD070601F7070601E907060167070601CD
:1007B00067070601670706016707060103080601C8
:1007C000FD070601F1070601E90706011F2C40E8B5
:1007D00040F3DDD941E840F1D6E71F2C40E880F333
:1007E000D6D941E880F1CFE713F4001FBBD010BD8C
:1007F00013F4801FFAE75B02F9D5B4E713F4002F76
:10080000F4E713F4802FF1E753B94AB9002908BF80
:1008100000281CBF4FF0FF314FF0FF3000F00CB844
:10082000ADF1080C6DE904CE00F008F8DDF804E045
:10083000DDE9022304B07047704700BF2DE9F04F97
:1008400007468C460846099E15463C461946002B2D
:1008500040F0C5808242B2FA82F746D94FB1C7F163
:10086000200E00FA07F3BD4024FA0EFEBC404EEA0B
:10087000030C4FEA15481FFA85FE220CBCFBF8F961
:1008800008FB19C309FB0EFA42EA03439A4528D92B
:10089000EB1809F1FF3004D29A4502D9A9F1020000
:1008A0002B44A3EB0A03A4B2B3FBF8F208FB123308
:1008B00002FB0EFE44EA0344A64514D92C1902F1AA
:1008C000FF3303D2A64501D9931E2C44A4EB0E049A
:1008D00043EA00401EB1FC40002334607360BDE871
:1008E000F08F4846DDE71346F0E702B9FFDE87BB2D
:1008F000831A01214FEA154EAAB2200CB3FBFEFC6D
:100900000EFB1C330CFB02F840EA0343984562D906
:10091000EB180CF1FF3004D2984502D9ACF102007B
:100920002B44A3EB0803A4B2B3FBFEFC0EFB1C3369
:100930000CFB02F244EA0344A2424ED92C190CF1FA
:10094000FF3304D2A24202D9ACF102032C44A41A10
:10095000BEE7C7F1200CBD4000FA07F320FA0CF8FF
:100960004FEA154E24FA0CFCBC404CEA0302ABB231
:10097000B8FBFEFC110C0EFB1C800CFB03F941EADA
:100980000040814523D928180CF1FF3104D281455C
:1009900002D9ACF102012844A0EB090092B2B0FBED
:1009A000FEFC0EFB1C000CFB03F842EA00439845DA
:1009B0000FD9EB180CF1FF3204D2984502D9ACF1F3
:1009C00002022B44A3EB080342EA014192E761468D
:1009D000E2E76246F6E76046A3E76346B7E783428D
:1009E00005D90EB1C6E900700021084677E7B3FAD1
:1009F00083F181B9834201D3BA420AD8BC1A60EBB1
:100A0000030301209C46002E67D0C6E9004C00215C
:100A100065E70846F7E7C1F1200C8B4002FA01F5C3
:100A200022FA0CF420FA0CFB27FA0CF28F401C433C
:100A300000FA01F34FEA144913431FFA84FE1A0C1B
:100A4000BBFBF9F809FB18BB08FB0EFA42EA0B42A4
:100A500092453ED9A21808F1FF3004D2924502D93E
:100A6000A8F102002244A2EB0A029BB2B2FBF9F801
:100A700009FB182208FB0EFE43EA024296452AD9DA
:100A8000A21808F1FF3304D2964502D9A8F1020357
:100A9000224443EA0040A2EB0E02A0FB05939A42D7
:100AA000CE46984602D306D14F4504D20138B9EB61
:100AB000050E63EB040886B1B7EB0E0362EB080783
:100AC00007FA0CFCCB40CF404CEA0303C6E90037E1
:100AD0009DE74046C7E74346DBE73146FFE60000B7
:100AE0000149024801F0ACBFB8A80601C3A806013D
:100AF0002DE970418FB0EFF30584B4B908F097F891
:100B000098B14FF0FF310423CDE90844CDE90A1331
:100B1000CDE90C440F4810494FF400620F4B08AD6B
:100B2000C02603DF0FB0BDE8708100220023CDE9AD
:100B300006234FF0FF330422CDE9033200234FF4A4
:100B40000062CDE9013300930349044B014803F0EF
:100B500067FDE7E700000021C00D0021E10A060162
:100B60000B6801330B60014B1B681847C02700213D
:100B7000014B1860704700BFC027002170B50446C4
:100B8000044E4518AC4200D170BD336814F8010B17
:100B90009847F7E7C027002170B504460D468AB094
:100BA000EFF30586A6B908F042F888B1282231464D
:100BB000684608F0E6F82B4622466946094800F0E8
:100BC000BDF9019B13B1684607F01DFD0AB070BD69
:100BD00000232246009369462B46034800F0AEF9F5
:100BE000F4E700BF39860601610B0601F7B5124F25
:100BF0000A9ABB680546C3F8802000220E4608F01A
:100C000053F8044668B10D4B0D48CDE9006345210A
:100C10002B460C4A07F0D9FFBB68D3F8800007F0D9
:100C2000F2FF28463146FFF7A9FF2046BB68C3F80C
:100C3000804003B0F0BD00BF600300216AD106010F
:100C4000E3A806012EA90601F8B50F4600293ED0FB
:100C500006680122304607F065FD0146044630462D
:100C600007F028FDC3070DD4A423194A19491A48CF
:100C700007F0F3FC3946194807F0EFFCA4211448AB
:100C800007F047FF2146304607F02AFD2518294680
:100C90000022304607F00EFD2D1AAC420DD0AC23D9
:100CA0000B4A0F490C4807F0D8FC39460D4807F0AD
:100CB000D4FCAC21064807F02CFF21463046002228
:100CC00007F014FD2146BDE8F84007F052BEF8BD1C
:100CD0003FA9060160A9060171A906018EA90601B6
:100CE000C6A90601ECA906012DE9F04706681446DD
:100CF000B3684A42B3F5004F2CBF0825042502EA29
:100D0000010731EA02021ED0BD4228BF3D46B94666
:100D1000CF1B07F1FF3A1AEA070F0ED034494FF400
:100D20009C73344A344807F098FC344807F095FC2B
:100D30004FF49C712F4807F0ECFE74B94FF0000996
:100D40004846BDE8F087A94204D82146BDE8F047EF
:100D500007F051BE4FF00009DBE7B068B0EBD40FED
:100D6000ECD93919491B07F0E7FC0146304607F07A
:100D70003EFD80460028E1D0B36809EBC005B3F51D
:100D8000004F2CBF082304231D44354455447F42A3
:100D90002F40A7EB09094946304607F0C3FC4C44F5
:100DA000073424F00704A41B804507464FEAE404F7
:100DB00008D202464146304607F053FD41463046D0
:100DC00007F094FD3946304607F08AFC38448442E7
:100DD00008D239463046224607F043FD21463046C8
:100DE00007F084FD01223946304607F07FFCA7E773
:100DF00028AA06013FA9060171A9060143AA060116
:100E0000B2F5802FF8B507460D46164612D2042AD1
:100E10000ED844494FF4F173434A444807F01DFC8F
:100E2000434807F01AFC4FF4F1713F4807F071FE98
:100E3000042200E00822B61AEC1D354424F0070411
:100E400025F007052D1B172D4FEAD5060ED8394979
:100E500040F2EB13344A354807F0FFFB344807F003
:100E6000FCFB40F2EB11304807F053FE00233C60DE
:100E70003146E3603046A66007F067FC012185003B
:100E80000746304607F058FC1B35ED082B18B342D7
:100E90000ED9294940F2FB13234A244807F0DDFB11
:100EA000234807F0DAFB40F2FB111F4807F031FE40
:100EB0000023194604F110029F422EDA2A462046EA
:100EC000002107F02BFC002320461A46194607F0A4
:100ED000FCFB771B19462046012207F007FC3A4627
:100EE000294607F01BFC2B4600222946204607F026
:100EF000ECFB3146204607F011FC3B4631462046CC
:100F0000002207F0E2FB31462046012207F0EEFB0B
:100F10002946BDE8F84007F0E9BC42F8041B01335C
:100F2000CAE700BF60AA06013FA9060171A9060130
:100F300081AA06019AAA0601C3AA06012DE9F04F6B
:100F40008B4692461C46002591B002909AF800000C
:100F500008B928465FE325280AF1010707D059465A
:100F6000029B98470028C0F25683013512E21822EE
:100F700000210AA807F005FF9AF80130252B78D048
:100F800000221046964694461646394617F8013B0D
:100F90002B2B00F09D8000F29480202B00F09B8092
:100FA000232B00F09B802EB19DF8306046F00406A4
:100FB0008DF83060BCF1000F05D09DF8306046F030
:100FC00008068DF83060BEF1000F05D09DF8306046
:100FD00046F010068DF8306028B19DF8300040F0E2
:100FE00020008DF830002AB19DF8302042F04002F8
:100FF0008DF830209DF8302002F04400442803D1C1
:101000006FF386128DF830209DF830202A2B42F0A5
:1010100080028DF830207BD19DF831204B1C42F0AE
:1010200001028DF831201A782E2A0CBF01210021EF
:101030009DF8312061F341028DF8312074D15A7846
:101040002A2A6AD000210A260133184610F8012BFB
:10105000A2F13007092F40F28E809DF830200E91CA
:10106000C2F3400040EAD17161F341028DF83020B3
:101070005AE00AF102078DF833309DF83130D90774
:1010800040F1498154F8049BB9F1000F07DA9DF84B
:101090003020C9F1000942F004028DF830205A07CF
:1010A00040F1428154F8048BB8F1000F80F2418185
:1010B0009DF831306FF341038DF831304FF0FF3838
:1010C00037E12D2B0CD0302B7FF46DAF01225CE784
:1010D0004FF0010C59E74FF0010E56E7012054E79D
:1010E000012652E733460CFB0202303A1E4616F840
:1010F000010BA0F13007092FF4D9994293D09DF844
:1011000030100D92D20F62F341018DF830108AE752
:101110000B4600224FF00A0CE8E79DF8312002331D
:1011200042F004028DF831201F4617F8012B6C2A7B
:1011300041D025D8682A2BD06A2A46D04C2A4CD0D8
:101140001F4617F8012B9DF83130782A8DF833208F
:1011500000F2D980572A4DD8412A03D0453A022AB5
:1011600000F2D18004229DF8323062F302038DF840
:10117000323001239EE006FB01210346303964E74B
:10118000742A26D07A2ADBD106229DF831300DE070
:101190005A78682A9DF8312006D1012161F3C602F0
:1011A0008DF831209F1CCCE71346022262F3C60360
:1011B0008DF83130C5E75A786C2A9DF8312001D17D
:1011C0000421EBE713460322F0E705229DF83130B6
:1011D000ECE707229DF83130E8E7BDF8303023F422
:1011E000F04323F0020343F4804343F00203ADF8DD
:1011F0003030A6E7A2F15801202900F2848001A036
:1012000050F821F0C9120601071306010713060161
:10121000071306010713060107130601071306014A
:1012200007130601071306016511060107130601DE
:10123000C912060189120601651106016511060130
:10124000651106010713060189120601071306013D
:10125000071306010713060107130601D112060141
:10126000C9120601ED120601071306010713060154
:10127000ED12060107130601C91206010713060144
:1012800007130601C912060101209DF8321003F070
:10129000780360F30201402B8DF8321002BF9DF8F5
:1012A000301041F001018DF83010632A31D1003B3C
:1012B00018BF01239DF83020C2F340010B4363F3B4
:1012C00041028DF83020D8E602209DF83210DEE78A
:1012D00003219DF8322003F07803A3F1400061F36D
:1012E000020243428DF832204341E3E703219DF897
:1012F000322013F0780F61F3020214BF01230023A0
:101300008DF83220D6E79DF8303043F001038DF898
:1013100030300023CEE79DF93020002AACBF4FF0DB
:10132000FF39DDF83490BAE69B077FF5C7AEDDF8EC
:1013300038800023CDE90D339DF832309DF831100F
:1013400003F00703012BC1F3C30138D1CB1E042BDB
:1013500022D8DFE803F003090921210054F8043BF7
:10136000DA17CDE90A3206E0073424F00704F4E87E
:101370000223CDE90A239DF8303013F0030656D03E
:101380003B4652465946029807F0ADFB0028C0F292
:1013900042810544BA46D9E554F8043B01294FEA95
:1013A000E372CDE90A3205D19DF828300A93002373
:1013B0000B93E0E70229DED1BDF92830D0E7022BFC
:1013C00023D1CB1E042B13D8DFE803F0030A0A1243
:1013D000120000232268201D0A920B930446CAE7DC
:1013E000E01D20F00700F0E80223CDE90A23F5E72D
:1013F00054F8043B01290A934FF000030B93D3D018
:101400000229B8D1BDF82830D0E7042B09D1E31D5B
:1014100023F0070303F10804D3E90023CDE90A23ED
:10142000A9E7032B04BF54F8043B0A93A3E79DF8F4
:1014300033007828AED8622822D825283FF48FAD13
:101440005828A7D1DDE90A010DF1260300930CAA63
:1014500004AB07F002FB8246B8F1000F0DF1260045
:101460000CDB9DF83020A0EB0A036FF38612984541
:101470008DF8302002D9A8EB03030D9380463DE0A0
:101480006338152886D801A252F820F00D15060100
:1014900071150601951306019513060195130601B2
:1014A00095130601711506019513060195130601A2
:1014B0009513060195130601CB1506019915060132
:1014C0009D1506019513060195130601E514060105
:1014D000951306019915060195130601951306014A
:1014E00099150601B8F1000FDDF828A00ADB414686
:1014F000504607F026FC00260AEB0008BAF1000F60
:101500000CD147E7504607F015FCF4E700260A9B8C
:101510000DF1100A8DF810300DF11108A8EB0A0337
:1015200006B101339DF83220D00668D50233520649
:101530000D9948BF0E9A0B4448BF9B18B9F1000F94
:1015400076DD9DF83020A9EB0309C2F380030393F5
:1015500053076DD4500661D546B159463046029BBB
:101560009847002857DB039B01351E46302356E081
:101570001E070FD413F0100618BF2026DDE90A233A
:10158000002BBFF65FAF524263EB43032D26CDE93C
:101590000A2357E72B26F1E7002653E70A9840B3C2
:1015A0000DF126030093002104AB0CAA07F055FAB5
:1015B000BDF83230824603F0EF0343F4F04343F0CA
:1015C00010030026ADF8323046E70A9B07293FF6A4
:1015D000E1AEDFE801F00C04060C08080C0C1D70ED
:1015E000D8E61D80D6E6EA17C3E90052D2E61D60B0
:1015F000D0E6DFF8C8A006460AF105088EE7110715
:1016000048BF013393E7184603935946029B984716
:101610000028039B04DA11B0BDE8F08F20234D446D
:101620004A46002AA5EB090109F1FF39EBDC0D461A
:1016300036B159463046029B98470028EBDB01350E
:101640009DF83230D90601D41A0706D55946302004
:10165000029B98470028DEDB01359DF83230DB061F
:1016600007D559469DF83300029B98470028D2DBE6
:1016700001350D9E2E44731B002B16DC434652464B
:101680005946029807F02FFA0028C4DB0544A94404
:10169000A9EB0503002B7FF77DAE59462020029B66
:1016A00098470028B7DB0135F2E759463020029B06
:1016B00098470028AFDB0135DDE700BFEEAA060141
:1016C00037B501220421044607F0EEFA002814BFC2
:1016D0000125002509D0064B452101930423054A25
:1016E00000930548234607F070FA284603B030BD42
:1016F000F4AA0601FAAA0601E3A80601F8B50C4F00
:101700001546BB68089A0446C3F880200E46FFF7CA
:10171000D7FF48B932462B46204607F00EFA002282
:10172000BB68C3F88020F8BD6FF00C00F7E700BF7E
:101730006003002138B50A4D069AAB680446C3F829
:101740008020FFF7BDFF38B9204607F019FA0022C4
:10175000AB68C3F8802038BD6FF00C00F7E700BF1E
:1017600060030021044608B54FF02002EFF3118317
:1017700082F31288BFF36F8F07F0DCFE204607F07C
:10178000E2FE034806F069FF00F06AF8FCE700BFDC
:101790000FAB06012DE9F74F16461446CDE90001BF
:1017A000DFF89080DFF89090019B9D192D1B14B9F4
:1017B00003B0BDE8F08F009B4046013B032B96BF72
:1017C0001E4A3F21D15C06F048FF4FF0000B1C4F32
:1017D0005C4526D9384615F80B1006F03EFF0BF194
:1017E000010BBBF1080FF3D1164806F036FF0027B6
:1017F000DFF854A0DFF854B0BC4216D9E95D584672
:10180000A1F120025F2A28BF2E2106F026FF013712
:10181000082FF1D10E4806F020FF072CC8D9083C4C
:10182000C2E7484606F019FFD9E7504606F015FF13
:10183000EDE700BF58AB060163AB06016CAB0601D8
:101840005DAB060167AB060165AB060169AB06013E
:10185000BDC60601014910220A60704710ED00E084
:1018600072B6404080F31188BFF36F8FBFF34F8F84
:1018700030BF62B6BFF36F8F704700BF37B5054604
:101880000C46C9B18B6810480093D1E9002345216B
:1018900007F09BF9636945210093D4E903230B48C2
:1018A00007F093F94521E269094807F08EF94521CF
:1018B000A269084807F089F92146284603B0BDE827
:1018C000304002F099BC00BF70AB0601A4AB06012A
:1018D000D8AB0601ECAB060143B2002B08DB0122BA
:1018E00000F01F0002FA00F0024A5B0942F82300F0
:1018F000704700BF00E100E070B54C1C072C0546A6
:101900000E460FD95723104A1049114806F0A5FE7C
:101910003146104807232A4606F09FFE57210A4801
:1019200007F0F7F86BB2002BACBF03F160430A4B32
:101930004FEA4414E4B2ABBF03F5614305F00F0571
:1019400083F800435C5570BD1FAC060155AC060121
:1019500071A9060170AC060114ED00E0034808B55A
:1019600006F07BFE0020FFF7FDFE00BFB0AC0601D5
:10197000014B024A1A607047C42700215D19060115
:1019800008B5034B1B689847BDE8084000F0DEB976
:10199000C427002130BFFFF7FDBF00BF0B4A08B5C9
:1019A0000B4B22F07F029A60BFF34F8FBFF36F8F14
:1019B000D3F8882022F47002C3F8882002F0C4FC17
:1019C00005F006FB00F050FC02F0C8FC0004060124
:1019D00000ED00E00A4A0B4993680968C3F88800E3
:1019E000C3F88C1008494B6843F080534B600023C8
:1019F00083F31188BFF36F8F9368D3F88C0070471F
:101A00006003002134A2060100ED00E01B498A6852
:101A100082F891E04FF030001044EFF3098C80E839
:101A2000F01F202080F31288BFF36F8F144F4FF008
:101A300000668A698A603E6092F991E0D2F8880077
:101A40000023C2F8883080F3118804B5104600F0F6
:101A5000A9FCBDE80440D2F89000EFF3148323F012
:101A6000010343EA000383F31488BFF36F8F02F18D
:101A7000300090E8F01F8CF3098870476003002164
:101A800004ED00E01EF0040F0CBFEFF30880EFF34D
:101A90000980816911F8021CEFF31482032908D030
:101AA00012F0010F01D10229FFD001B507F09AF819
:101AB00001BDD0F818800D4981614FF4B27C6645B4
:101AC00002D3066040F2631609488068D0F890108F
:101AD00021F00101C0F89010BFF34F8F22F00102F6
:101AE00082F31488BFF36F8F70470000911C0601CA
:101AF000600300210C4C9846A36883B50546D86F57
:101B000017460E4606F050FAA4683146D4E91A3258
:101B10009B1AC4F894000193636E3A4600932846DA
:101B2000434600F073F800BF6003002130B5017B2D
:101B300042F8203C039B104D42F81C3C049B11F0E2
:101B4000040F42F8183C059B0C4918BF294642F87F
:101B5000143C4FF0807321F0010142F8043C42F83C
:101B6000081C0023A2F120044FF43C420465C0E9A4
:101B70002423C0F8883030BDF51A060175860601A9
:101B80000C4B70B59D6806460C465DB1D5F8943097
:101B900063B107F04CF838B9163603D1D5F8940084
:101BA000A04200D8002070BDE86FF9E71636F9D1E1
:101BB000686EF5E76003002108B5094B0D46986093
:101BC000144600F0EFFB204685F30988002163B638
:101BD00081F31188BFF36F8F0022002306F04AFDC6
:101BE0006003002101B5EFF30580A0F110004FEA7A
:101BF000C0000449014409C99847BDE801400249B1
:101C000008470000C49B06014D1D060186461E487C
:101C10008068D0F894004FF4806C6044EC4680F308
:101C200009880EB52DE901101748806800F0BAFB4D
:101C3000BDE80110DCF80000DCF804C02DE901105B
:101C40006246494007F09DF8BDE801106044BDE8D8
:101C50000E4080F30988704603B40B488068D0F8C2
:101C6000901051F00101EFF3148C5CF0010CC0F8FE
:101C70009010BFF34F8F8CF31488BFF36F8F03BCAA
:101C8000DFF808C060470000600300217586060188
:101C9000DFF88CC0DCF808C0DCF894C00CF5806C70
:101CA000BCF1080CCCF800D0CCF804E08CF3098827
:101CB00040F2631C664503D1EC462DE9305002E04A
:101CC000EC462DE93010DFF85CC04FEA8606B444DC
:101CD000DCF800C0E047DDF810E0DDF80CC08CF364
:101CE000098803B40E488068D0F8901051F00101C3
:101CF000C0F89010BFF34F8FEFF3148C5CF0010C21
:101D00008CF31488BFF36F8F03BC4FF000014FF0CA
:101D100000024FF00003C4465CF0010C6047000075
:101D20006003002128A3060137B54FF0FF3301936C
:101D30000023C55C1DB18B4201D00133F9E7184681
:101D4000002101910199116003B030BD044B9968E5
:101D50009869884203D003494FF080520A60704767
:101D60006003002104ED00E010B5204C452120481F
:101D700006F02BFFA36A990103D545211D4806F003
:101D800024FFA36ADA0103D545211B4806F01DFF95
:101D9000164CA36ADB0203D54521184806F015FF4F
:101DA000A36A180303D54521154806F00EFF0F4C12
:101DB000A36A590303D54521124806F006FFA36A1A
:101DC0009A0303D54521104806F0FFFE074CA36A8D
:101DD000DB0303D545210D4806F0F7FEA36A00207A
:101DE0006FEA03436FEA1343A36210BD00ED00E006
:101DF000CCAC0601E9AC060101AD060120AD06013F
:101E00004FAD060172AD06019CAD0601BBAD0601EA
:101E10002DE9F041404C05460E4640484521174605
:101E200006F0D3FEA36AD80603D545213C4806F048
:101E3000CCFEA36A190703D545213A4806F0C5FE32
:101E4000354CA36A9A072FD46FF01508324CA36A59
:101E5000DE0703D54521344806F0B7FEA36A9C0689
:101E600003D54521314806F0B0FE2B4EB36AD806A3
:101E70002FD4B36A99072CD40024274A936A43F0DD
:101E8000FF0393622A4BAA6923F00103934240D8CF
:101E9000284B23F0010393423BD9274BAB6101232D
:101EA00020463B70BDE8F0814521244806F08DFEB8
:101EB000D4F83480A36A1B06C6D542464521204883
:101EC00006F083FE002EC1D0A36A23F08003A36234
:101ED000BCE773681A05CFD529464046FFF750FE88
:101EE000044618B180F309880224C6E7B36ADB060A
:101EF000C2D540F24913134A1349144806F0ADFB0A
:101F0000134806F0AAFB40F249110E4806F001FE04
:101F1000B3E70023C4E700BF00ED00E0EBAD06012E
:101F200006AE06013EAE06018EAE0601B2AE060159
:101F3000331D0601351D0601451D060156AE06017D
:101F400073AE0601E6AE060120AF060171A90601D7
:101F50006AAF0601F8B52C4C05460F462B484521C3
:101F6000164606F032FEA36AD90403D54521284857
:101F700006F02BFEA36A1A0503D54521254806F075
:101F800024FE214CA36A9B0510D52348452106F069
:101F90001CFEA26BA36A180408D545211F4806F051
:101FA00014FE1FB1A36A23F40043A362164CA36A74
:101FB000590503D545211A4806F007FEA36ADA053C
:101FC00019D54521174806F000FE0F4A936A43F4DD
:101FD0007F439362144BAA6923F00103934210D804
:101FE000124B23F0010393420BD9114BAB61012338
:101FF00000203370F8BDA36A9B04E6D545210D4847
:10200000E1E70023F4E700BF00ED00E08DAF06013B
:10201000A8AF06013EAE0601BEAF0601DCAF060169
:10202000F6AF060116B00601331D0601351D060187
:10203000451D0601B2AE06012DE9F0436F4B054682
:10204000D3F804808946144600268BB0C8F30807ED
:1020500086F31188BFF36F8F02F07F43B3F17F4F98
:1020600011D1D0070FD4510603D4220708D401267A
:1020700008E04521624806F0A8FD14F0040400D0F1
:102080004D4600267DB94FF47C735E4A5E495F4839
:1020900006F0E3FA5E4806F0E0FA4FF47C71594826
:1020A00006F037FD00250024FB1E8DF80740092BA4
:1020B00000F29180DFE803F0058488648F8F8F8FB2
:1020C0008F8C4E4F4521534806F07FFD8DF8074019
:1020D000FC6A14F0020405D045214F4806F075FD56
:1020E000002406E0FB6A002B1DDA45214B4806F070
:1020F0006CFD9DF807309BB92022294602A806F006
:1021000035FE099B002E73D0C3F3080222B96FEA93
:1021100053236FEA43230993204602A9FFF7AEFB3E
:102120000BB0BDE8F083FB6A5B003CD545213C4821
:1021300006F04BFDAB6933F8022C4DF602739A4260
:1021400006D145212A68374806F03FFD2C68D0E7C4
:1021500097F828303BB101210DF107022846FFF71F
:1021600057FE0446C5E797F8293033B101210DF138
:1021700007022846FFF7EEFEF3E77B8D9BB213B113
:10218000FFF7F2FDEDE7284940F2C2231D4A1F4840
:1021900006F063FA254806F060FA40F2C2211948B9
:1021A00006F0B7FCA5E7204940F2C623154A1748B8
:1021B00006F053FA1E4806F050FA40F2C621EEE748
:1021C00000210DF10702C9E700210DF10702D0E758
:1021D0004521184882E7184918F4F87F174A18482B
:1021E00008BF0A46A7F11003452106F0EEFC77E789
:1021F00023F4FF7323F001038DE700BF00ED00E03F
:1022000061B00601E6AE060189B0060171A90601BA
:102210009CB00601DAB00601F6B006011CB1060159
:102220002FB1060153B10601EFB7060174B10601E3
:1022300098B10601C8B1060133B0060148B00601E5
:10224000F1B10601024A536943F01003536170472C
:1022500000ED00E0EFF30880EFF3098101B572466D
:10226000FFF7EAFE01BD00BF002320210348C2188A
:102270000133802B82F80013F9D1704700E100E0B0
:10228000002080F31488BFF36F8F002080F30A884A
:1022900080F30B8800200E490860BFF34F8F0D4874
:1022A00080F3088800F02CF8202080F311880A4879
:1022B0004FF40061401880F30988EFF31480022185
:1022C000084380F31488BFF36F8FFFF767FB0000AC
:1022D00094ED00E0C01F0021C00500210023184636
:1022E0000649D1F89020C2F30722934200D17047EB
:1022F000C1F89830C1F8A0000133F6E700ED00E026
:1023000010B572B6002484F31388FFF7E7FF234665
:102310004FF0FF300B4A03F120010133102B42F83C
:102320002100F8D100234FF0FF3003F160010133A9
:10233000102B42F82100F8D162B6BFF34F8FBFF3E4
:102340006F8F10BD00E100E0064B9B68834207D110
:10235000EFF3058323B1044A536843F0805353607D
:1023600004F092BC6003002100ED00E01FB5094CB1
:10237000094A23460121094800F0CEF800230393BF
:10238000074B0121E41A01A80193029400F0A4F97B
:1023900004B010BD00002021000000216CA0060147
:1023A000000000212DE9F84F846F064674B32546DE
:1023B00094F8C87004F1C0090024DFF8A480DFF8A5
:1023C000A4B0DFF8A4A06B68EBB1102C0CD9514677
:1023D000E0235A46254806F040F9254806F03DF925
:1023E000E021584606F095FB0C236343296808EB6F
:1023F000030248F803106B6801345360AB68013F77
:102400009360E4B202D00C35A945DCD1D6F8943003
:10241000FBB1D6E91935F76F1D44102CA5EB070564
:102420000CD91149F6230F4A104806F016F9104846
:1024300006F013F9F6210B4806F06BFB0C236343FF
:1024400007490134CA18CF500A4B55601868E4B2E6
:1024500090602146BDE8F84F014800F0B3B900BFD5
:10246000E801002109B2060145B2060171A9060181
:1024700067B2060144A0060138B5134CD4F8903079
:10248000C3F30723013B984207D9024645210F4871
:1024900006F09BFB6FF0150038BD0B680D7A23F03A
:1024A0001F0205F01F031A43CB686D0923F01F03B9
:1024B00043EA450343F00103C4F89800C4F89C20A4
:1024C000C4F8A030E8E700BF00ED00E099B20601D3
:1024D0000522044BC3F89420BFF34F8FBFF36F8FD7
:1024E000704700BF00ED00E0BFF35F8F0022024B9A
:1024F000C3F89420704700BF00ED00E0044B054A8C
:10250000D3F890301078C3F30723181A704700BF30
:1025100000ED00E0780400212DE9F04F89460646E1
:102520004FF0000ADFF89081644D98F8004087B0C2
:10253000CA4506DB88F8004016342BD007B0BDE84A
:10254000F08FD6F804B0BBF1000F54D0BBF11F0FD1
:1025500018D91BF01F0F15D13368DA0612D11846AF
:10256000019306F069FB019B07460BEB0300013862
:1025700006F062FB874220D06FF015073A464521EE
:102580004F4802E0524645214E4806F01EFBEA2322
:1025900088F8003040F211134B4A4C494C4806F081
:1025A0005CF849464B4806F058F840F2111146488D
:1025B00007B0BDE8F04F06F0ACBA17F1160FDDD04A
:1025C000BC42DBDDC5F89870D5F89C00C5F8987062
:1025D000D5F8A03020F01F0043F01F0BD6E90031E2
:1025E0001944984201F1FF321DD1934507D131467C
:1025F000F8B206F05BFB0AF1010A0C3698E7C5F861
:102600009870D5F89C3021F01F0103F01F030B4395
:102610003146C5F89C30E0B206F048FB10F1160FC9
:10262000B5D0441CE7E7013B9345E0B223F01F031C
:102630000AD1C5F89870D5F8A020314602F01F02E3
:102640001343C5F8A030E7E70192C5F89870D5F8B4
:10265000A01001F01F010B43C5F8A030314606F071
:1026600025FB10F1160F92D0C5F89870D5F89C1084
:102670009DF81030019A61F304038DF81030D5F8FD
:10268000A0309DF810105B0863F347118DF810100F
:10269000D6E900310B4402930BF1FF3B23F01F03FB
:1026A0005B449A1A013022F01F0202A9C0B20592BF
:1026B000FFF7E2FEB2E700BF7804002100ED00E082
:1026C00073B306014BB30601C4B20601EFB70601AE
:1026D00071A906019BB306012DE9F74F324E8946D9
:1026E00005464FF00008B346304FC84502DB03B043
:1026F000BDE8F08FD5F804A0BAF1000F4FD02968DB
:102700000846019106F098FA019904460AEB010087
:10271000013806F091FA84424FF01402244B18D08D
:102720006FF0150302FB08F84BF8083040F2211354
:10273000204A2149214805F090FF4946204805F0EC
:102740008CFF40F221111B4803B0BDE8F04F06F0AA
:10275000E0B914F1160F3460E8D01978A142E5DD34
:1027600002FB08B0C7F89840C7F89840D7F89C40DB
:1027700000F10801007B64F304000871D7F8A000A1
:102780000C79400860F347140C71D7F89C1021F0C5
:102790001F017160D7F8A01021F01F01316108F10D
:1027A000010814360C35A0E7B402002100ED00E06A
:1027B00078040021C4B20601EFB7060171A9060131
:1027C000C7B3060170B5254B0E461B780446194663
:1027D0000025234AD2F89000C0F3072081420BDB8A
:1027E00020490968C2F89810C2F8A0500025B542E7
:1027F00008DB16330FD070BDC2F89810C2F8A05095
:102800000131E7E762682AB31F2A16D82A46452114
:10281000154806F0DAF94FF49873144A144915482C
:1028200005F01BFF3146144805F017FFBDE8704066
:102830004FF498710D4806F06CB9D106E6D12268C4
:10284000D206E3D12146D8B206F030FA10F1160FC5
:10285000E1D0431C01350C34C9E700BF78040021E6
:1028600000ED00E0B40200214BB30601C4B2060142
:10287000EFB7060171A90601F6B3060170B5234C46
:102880002349D4F890300D68C3F307239D4216D92D
:102890004FF4A4731F4A2049204805F0DEFED4F807
:1028A000902029461E48C2F3072205F0D6FE19489B
:1028B0004FF4A47106F02DF94FF0FF3070BD0020E9
:1028C000FFF712FE174B4A68C4F8C030854205D1A5
:1028D000154B00201D70FFF7FBFDEFE71368167A1C
:1028E00023F01F0106F01F031943D368760923F074
:1028F0001F0343EA460343F00103C4F89800103273
:10290000C4F89C100130C4F8A030DFE700ED00E00F
:1029100078A00601C4B20601EFB7060171A906014D
:1029200023B40601AAFF440078040021014B18607B
:10293000704700BFC82700210239012902D8034B84
:102940001B6818474FF0FF30704700BFC8270021B1
:1029500010B5064C049AA368C3F88020FFF7ECFF7B
:102960000022A368C3F8802010BD00BF60030021CF
:102970002DE9F843023B012B06460C46154615D8B7
:10298000B2B181B11746DFF82C8006EB0409D8F804
:10299000003016F8010B9847013003D0B145F6D14D
:1029A000013FF2D1EC1B2046BDE8F8830024FAE792
:1029B0001446F8E7C82700212DE9F3471546DFF84C
:1029C0006C800C9A9946D8F808300746C3F88020E6
:1029D000A5FB01A20C4672B9514606F065F9064600
:1029E000B0B1134B4521CDE900A3124A3B46124832
:1029F00006F0EBF806E000912B4645210D4A0F4802
:102A000006F0E3F8D8F80830D3F8800006F0FBF8B9
:102A10004B462A4621463846FFF7AAFFD8F8083029
:102A2000C3F8806002B0BDE8F08700BF60030021FA
:102A30006AD1060190B40601E3A8060157B4060165
:102A40000FB407B504AB53F8042B022104480193DB
:102A5000FEF774FA03B05DF804EB04B0704700BFF2
:102A6000C98D060108B50848084B186006F06DFDD1
:102A700038B10748FFF75AFF0548FEF779F80020FC
:102A800008BD6FF01200FBE7349B0601C80200216D
:102A9000952A06010A2838B50446074D04D128684E
:102AA00083680D215B68984728688368E1B25B689A
:102AB0009847204638BD00BFC802002170B51646B1
:102AC0000C46056961B922492423224A224805F0AF
:102AD000C4FD224805F0C1FD24211E4806F019F866
:102AE000636863B91E4925231A4A1B4805F0B5FDE2
:102AF0001C4805F0B2FD2521164806F00AF86B685F
:102B00005BB100229C4212D12368A96852B9A1424C
:102B10006B6000D1AB60002323606EB9002070BDF4
:102B20000B46EFE7A142136008BFAA60F3E71968FC
:102B30001A460029F4D13EB16B68A86823606C6026
:102B40000028EBD1AC60EAE76FF01500E7E700BFC3
:102B5000E1B40601B4B4060171A90601EAB40601A4
:102B6000F9B406010BB50601436802695B682DE9FB
:102B7000F0479F6B546805469F6314B32668DFF8DF
:102B80004880DFF84890DFF848A0A3681F4214D0BF
:102B9000636863B9494645234246504605F05DFDEA
:102BA0000C4805F05AFD4521404605F0B2FFD4E936
:102BB0000132214628463A40984716B134463668D5
:102BC000E3E7BDE8F08700BFB4B4060122B5060113
:102BD00071A906010BB506012DE9F04F0546DFF896
:102BE000A89185B0D9F808301446109ACFB2C3F82E
:102BF0008020FDF725FD294606F027FA002800F081
:102C0000B3804521614A624805F0DFFFD9F80830FA
:102C1000D3F8800005F0F7FF6B6814F4FC2FD5F8AB
:102C200010A003930ED05B4940F2E6235A4A5B485A
:102C300005F013FD5A4805F010FD40F2E621564814
:102C400005F067FF04F03003302B0ED1554940F2F8
:102C5000E923514A514805F000FD534805F0FDFCB9
:102C600040F2E9214C4805F054FF40F20223234092
:102C7000022B0ED14D4940F2ED23474A474805F05B
:102C8000ECFC4B4805F0E9FC40F2ED21424805F030
:102C900040FF04F00603042B0BD146493F4840F2A5
:102CA000F1233D4A05F0D9FC40F2F1213A4805F004
:102CB00030FF14F4406622D0A3050ED43E494FF4F1
:102CC0003D73354A354805F0C8FC3C4805F0C5FC65
:102CD0004FF43D71304805F01CFFB6F5406F0ED142
:102CE00037494FF43E732C4A2C4805F0B6FC354862
:102CF00005F0B3FC4FF43E71274805F00AFFE004ED
:102D000004D51EB1E10748BF84F440640126039B4B
:102D1000BE401B6824F4805B1E420ED12A4940F25B
:102D200005331D4A1D4805F098FC284805F095FC20
:102D300040F20531184805F0ECFEDAF80030E20701
:102D40004CBF1E4323EA06065A46D8F800303946DF
:102D50002846CAF8006098470022D9F80830C3F81E
:102D6000802005B0BDE8F08FD5F80880D8F8003095
:102D7000002B7FF451AF4521154B044A1548CDF87F
:102D8000008005F022FF41E7600300217DBC0601C1
:102D90004AB50601FCB50601D2B5060171A90601C6
:102DA00059B606017DB60601B6B60601F3B60601B0
:102DB00027B7060179B70601ACB70601F1B70601DE
:102DC0002CB806016DB8060199B80601D7B80601FE
:102DD00076B5060184B50601F7B504461E4E0A9A7B
:102DE000B3680D46C3F88020FDF72AFC214606F0A3
:102DF0002CF9D8B14521194A194805F0E6FEB36807
:102E0000D3F8800005F0FFFE01220421284605F0DA
:102E10004BFF0746B0B1134B4521019304230F4AE2
:102E2000009311482B4605F0D0FEE8E7A3685A68E6
:102E3000002AE9D1009345210C4B084A0C4805F0C3
:102E4000C4FEDCE7A368294620465B689847B36860
:102E5000C3F8807003B0F0BD6003002164BC0601BC
:102E60004AB50601F4AA0601E3A80601E9B806017D
:102E700084B506012DE9F7430446184E9046B36821
:102E80000C9A0F46C3F88020FDF7DAFB214606F0C6
:102E9000DCF8054688B14521114A124805F095FE37
:102EA000B368D3F8800005F0AEFE009345210E4BC9
:102EB0000B4A0E4805F089FEF2E7A368D3F80890A4
:102EC000B9F1000FF1D0424639462046C847B368F1
:102ED000C3F8805003B0BDE8F08300BF6003002159
:102EE00044BC06014AB50601F6B8060184B50601E0
:102EF000F7B50446154E0A9AB3680F46C3F880200A
:102F0000FDF79EFB214606F0A0F8054688B1452155
:102F10000F4A104805F059FEB368D3F8800005F059
:102F200072FE009345210C4B094A0C4805F04DFEFA
:102F3000F2E7A368DA68002AF3D0394620469047C2
:102F4000B368C3F8805003B0F0BD00BF6003002138
:102F500026BC06014AB506010AB9060184B5060178
:102F6000F7B50446154E0A9AB3680F46C3F8802099
:102F7000FDF766FB214606F068F8054688B1452155
:102F80000F4A104805F021FEB368D3F8800005F021
:102F90003AFE009345210C4B094A0C4805F015FEFA
:102FA000F2E7A3681A69002AF3D039462046904711
:102FB000B368C3F8805003B0F0BD00BF60030021C8
:102FC00006BC06014AB506011CB9060184B5060116
:102FD000F7B50446154E0A9AB3680F46C3F8802029
:102FE000FDF72EFB214606F030F8054688B1452155
:102FF0000F4A104805F0E9FDB368D3F8800005F0EA
:1030000002FE009345210C4B094A0C4805F0DDFDFA
:10301000F2E7A3685A69002AF3D039462046904760
:10302000B368C3F8805003B0F0BD00BF6003002157
:10303000E9BB06014AB5060130B9060184B50601AF
:103040002DE9F74F0546DFF86C911446D9F80830A2
:103050000E9ACEB2C3F88020FDF7F2FA294605F0A9
:10306000F4FF002800F096804521534A534805F0AC
:10307000ACFDD9F80830D3F8800005F0C4FD002B72
:1030800032D14F4940F295234E4A4F4805F0E5FAB8
:103090004E4805F0E2FA40F2952122E02303D5F8EC
:1030A00004A0D5F810B00BD54949474840F28F230A
:1030B000444A05F0D2FA40F28F21424805F029FD3A
:1030C00004F4C043B3F5C04FD9D1424940F2912333
:1030D0003C4A3D4805F0C1FA3F4805F0BEFA40F2CF
:1030E0009121384805F015FD04F4E823B3F5C82F05
:1030F0000ED13A494FF42673324A334805F0ADFAFF
:10310000374805F0AAFA4FF426712E4805F001FD64
:1031100004F4C823B3F5804F0ED1324940F29F2307
:10312000284A294805F099FA2F4805F096FA40F206
:103130009F21244805F0EDFC0127DAF80030B74064
:103140001F420ED1294940F2A5231E4A1E4805F010
:1031500084FA274805F081FA40F2A521194805F0C4
:10316000D8FC220405D5DBF800301F4201D084F4DE
:10317000C02404F4C02304F4B03231462846D8F801
:103180001870B8470022D9F80830C3F8802003B07F
:10319000BDE8F08FD5F80880D8F81830002B7FF400
:1031A0007DAF4521134B044A1348CDF8008005F04C
:1031B0000CFD5EE760030021C5BB06014AB50601B0
:1031C000E0B90601D2B5060171A906010ABA0601E5
:1031D00059B9060173B90601B4B9060135BA060139
:1031E000B6BA06010ABB060154BB060199B806012E
:1031F000D7B8060141B9060184B5060173B5044686
:10320000144E089AB368C3F88020FDF719FA2146D6
:1032100005F01BFF054688B145210F4A0F4805F010
:10322000D4FCB368D3F8800005F0EDFC0093452191
:103230000B4B094A0B4805F0C8FCF2E7A3681A6A71
:10324000002AF3D020469047B368C3F8805002B0FC
:1032500070BD00BF60030021A9BB06014AB506018D
:1032600099BB060184B5060108B5436803491A688D
:10327000006906F030F8002008BD00BF8CA10601EF
:10328000F7B50446154E0A9AB3680F46C3F8802076
:10329000FDF7D6F9214606F03BF8054688B14521F1
:1032A0000F4A104805F091FCB368D3F8800005F090
:1032B000AAFC009345210C4B094A0C4805F085FCFB
:1032C000F2E7A3681A68002AF3D0394620469047EF
:1032D000B368C3F8805003B0F0BD00BF60030021A5
:1032E000BCBD06014AB506017AB5060184B50601E2
:1032F00073B50446214E089AB3680D46C3F8802082
:10330000FDF79EF9214606F003F858B345211C4A03
:103310001C4805F05AFCB368D3F8800005F073FC34
:103320002946204698470022B368C3F8802002B09F
:1033300070BDA3685B68002BF2D16FF05700F2E715
:1033400001220421284605F0AFFC0028F1D00E4BE5
:103350004521019304230A4A00930C482B4605F0AB
:1033600034FCD8E7A3685A68002AE9D100934521C4
:10337000074B034A074805F028FCCCE7600300210F
:10338000A6BD06014AB50601F4AA0601E3A8060196
:10339000D8BC060184B506012DE9F04F85B0814601
:1033A0003E4E02AFBC6B8A46B1685FFA82F8C1F844
:1033B00080401FFA83FBFDF743F9494605F0A8FF5B
:1033C0000246002862D04521354A364805F0FDFB0B
:1033D000B368D3F8800005F016FC0135EAB29045D9
:1033E00003F10C031FD8D9F8083042469D682146E6
:1033F0005B464846A847B3680C37C3F880A0BD4673
:10340000BDE8F08FCB1D23F00703ADEB030D0DF1ED
:103410000B04A30824F003040A46204651467B60AF
:1034200005F0A4FC2346D3E900011A7A3B6002F0C0
:10343000010205F039FC3B6882460028CDD00C2003
:1034400045432C44227A184812F0010F174A08BF4E
:1034500002467B68616855F82330CDE90012144AB2
:103460000FE00C2101FB08F15046796005F01CFCCF
:10347000796805460028C5D00B4B094ACDE90013F1
:10348000534645210B4805F0A0FBA1E708F1FF33A7
:103490001E2BE6D94521024A074897E76003002121
:1034A00092BD06014AB506016AD10601F4AA0601D9
:1034B0007BBD0601E3A80601E3BC060170B5044626
:1034C0000E4E069AB368C3F88020FDF7B9F821467E
:1034D00005F01EFF054648B109484521094A05F097
:1034E00074FBB368D3F8800005F08DFBA368204619
:1034F0001B689847B368C3F8805070BD6003002113
:103500004AB506015ABD060138B504460B4D069A68
:10351000AB68C3F880202046FDF792F8214605F0FD
:10352000F7FE0028F7D006484521064A05F04DFB76
:10353000AB68D3F8800005F066FB00BF6003002194
:103540004AB5060137BD060138B50446114D069A45
:10355000AB68C3F88020FDF773F8214605F0D8FE6C
:1035600080B10D4845210D4A05F02FFBAB68D3F81B
:10357000800005F048FB204698470022AB68C3F85E
:10358000802038BDA3685B69002BF4D16FF0570031
:10359000F3E700BF600300214AB5060120BD060124
:1035A00073B50446144E089AB368C3F88020FDF73B
:1035B00047F8214605F0AEFF054688B145210F4A80
:1035C0000F4805F002FBB368D3F8800005F01BFB41
:1035D000009345210B4B094A0B4805F0F6FAF2E738
:1035E000A3689A68002AF3D020469047B368C3F8CE
:1035F000805002B070BD00BF6003002119BF0601FA
:103600004AB50601F4BD060184B5060173B504464A
:10361000214E089AB3680D46C3F88020FDF710F8D4
:10362000214605F077FF58B345211C4A1C4805F098
:10363000CCFAB368D3F8800005F0E5FA29462046B5
:1036400098470022B368C3F8802002B070BDA36819
:103650001B68002BF2D16FF05700F2E701222846D9
:10366000114605F021FB0028F1D00E4B45210193B6
:1036700001230A4A00930C482B4605F0A6FAD8E726
:10368000A3681A68002AE9D100934521074B034A31
:10369000074805F09AFACCE76003002105BF060150
:1036A0004AB50601F4AA0601E3A80601FEBD06011B
:1036B00084B5060173B505461C4C089AA3680E46EE
:1036C000C3F88020FCF7BCFF294605F023FFD0B1EA
:1036D0004521174A174805F078FAA368D3F8800007
:1036E00005F091FA01220221304605F0DDFAB0B171
:1036F000114B4521019302230D4A00930F48334695
:1037000005F063FAE9E7AB681A68002AEAD100938A
:1037100045210B4B064A0B4805F057FADDE7A36835
:10372000C3F880006FF0850002B070BD6003002117
:10373000EDBE06014AB50601F4AA0601E3A806019A
:10374000FEBD060184B50601F7B50546154E0A9A79
:10375000B368CFB2C3F88020FCF772FF294605F0AA
:10376000D9FE044688B145210F4A104805F02DFACC
:10377000B368D3F8800005F046FA009345210C4B5E
:10378000094A0C4805F021FAF2E7AB685A68002AAA
:10379000F3D02846394690472046B368C3F88040A6
:1037A00003B0F0BD60030021D8BE06014AB5060192
:1037B00006BE060184B5060137B50446124D089AC7
:1037C000AB68C3F88020FCF73BFF214605F0A2FE62
:1037D00088B145210D4A0E4805F0F7F9AB68D3F8DA
:1037E000800005F010FA009245210A4B074A0A486A
:1037F00005F0EBF9F2E7A26851680029F3D0AA6856
:10380000C2F8800003B030BD60030021BFBE0601D6
:103810004AB5060106BE060184B5060173B5044625
:10382000214E089AB3680D46C3F88020FCF708FFC4
:10383000214605F06FFE58B345211C4A1C4805F08F
:10384000C4F9B368D3F8800005F0DDF929462046B5
:1038500098470022B368C3F8802002B070BDA36807
:103860001B69002BF2D16FF05700F2E7012208210B
:10387000284605F019FA0028F1D00E4B4521019396
:1038800008230A4A00930C482B4605F09EF9D8E716
:10389000A3681A69002AE9D100934521074B034A1E
:1038A000074805F092F9CCE760030021E6BF060166
:1038B0004AB50601F4AA0601E3A806010FBE0601F7
:1038C00084B5060173B50446214E089AB3680D46C7
:1038D000C3F88020FCF7B4FE214605F01BFE02462B
:1038E00050B345211B4A1C4805F06FF9B368D3F863
:1038F000800005F088F92946204698470022B368E1
:10390000C3F8802002B070BDA368DB68002BF2D141
:103910006FF05700F2E70821284605F0C5F90028A6
:10392000F2D00E4B4521019308230A4A00930C481C
:103930002B4605F04AF9D9E7A36819690029EAD1AD
:1039400000934521074B034A074805F03EF9CDE7B0
:1039500060030021D0BF06014AB506016AD1060105
:10396000E3A806010FBE060184B5060173B505463E
:10397000144E089AB368C3F88020FCF761FE29460C
:1039800005F0C8FD044688B145210F4A0F4805F0EF
:103990001CF9B368D3F8800005F035F90093452190
:1039A0000B4B094A0B4805F010F9F2E7AB68DA69EE
:1039B000002AF3D0284690472046B368C3F88040D9
:1039C00002B070BD60030021B6BF06014AB5060112
:1039D0001ABE060184B5060173B50546144E089A51
:1039E000B368C3F88020FCF72BFE294605F092FD52
:1039F000044688B145210F4A0F4805F0E6F8B36840
:103A0000D3F8800005F0FFF8009345210B4B094ADD
:103A10000B4805F0DAF8F2E7AB681A6A002AF3D02F
:103A2000284690472046B368C3F8804002B070BD76
:103A3000600300219BBF06014AB5060128BE0601AE
:103A400084B5060173B50546144E089AB368C3F8E9
:103A50008020FCF7F5FD294605F05CFD044688B1A1
:103A600045210F4A0F4805F0B0F8B368D3F880003D
:103A700005F0C9F8009345210B4B094A0B4805F0A6
:103A8000A4F8F2E7AB689A6A002AF3D02846904778
:103A90002046B368C3F8804002B070BD60030021C7
:103AA00081BF06014AB5060137BE060184B506018D
:103AB00073B50546144E089AB368C3F88020FCF726
:103AC000BFFD294605F026FD044688B145210F4A71
:103AD0000F4805F07AF8B368D3F8800005F093F842
:103AE000009345210B4B094A0B4805F06EF8F2E7AD
:103AF000AB68DA6A002AF3D0284690472046B368BC
:103B0000C3F8804002B070BD6003002166BF0601AB
:103B10004AB5060145BE060184B5060173B50546E2
:103B2000144E089AB368C3F88020FCF789FD294633
:103B300005F0F0FC044688B145210F4A0F4805F016
:103B400044F8B368D3F8800005F05DF80093452190
:103B50000B4B094A0B4805F038F8F2E7AB689A6B53
:103B6000002AF3D0284690472046B368C3F8804027
:103B700002B070BD600300214BBF06014AB50601CB
:103B800054BE060184B5060173B50546144E089A65
:103B9000B368C3F88020FCF753FD294605F0BAFC52
:103BA000044688B145210F4A0F4805F00EF8B36866
:103BB000D3F8800005F027F8009345210B4B094A04
:103BC0000B4805F002F8F2E7AB68DA6B002AF3D095
:103BD000284690472046B368C3F8804002B070BDC5
:103BE000600300212FBF06014AB5060163BE06012E
:103BF00084B5060173B50446144E089AB368C3F839
:103C00008020FCF71DFD214605F084FC054688B1A7
:103C100045210F4A0F4804F0D8FFB368D3F880005D
:103C200004F0F1FF009345210B4B094A0B4804F0C7
:103C3000CCFFF2E7A3681A6C002AF3D02046904725
:103C4000B368C3F8805002B070BD00BF60030021AC
:103C5000A4BE06014AB5060173BE060184B506017D
:103C600073B50446144E089AB368C3F88020FCF775
:103C7000E7FC214605F04EFC054688B145210F4A78
:103C80000F4804F0A2FFB368D3F8800004F0BBFF34
:103C9000009345210B4B094A0B4804F096FFF2E7CD
:103CA000A3685A6C002AF3D020469047B368C3F843
:103CB000805002B070BD00BF600300218DBE0601C0
:103CC0004AB5060182BE060184B506014FF0E02325
:103CD0009A69196910B511F4803F98690849094B30
:103CE00001D1824206D21A680C6822441A604FF051
:103CF000E02212691B680A681344181A10BD00BF3D
:103D0000540300215C03002120220020084B83F88B
:103D10002320084A084B1A60084B18604FF0E02334
:103D20005A6198611A6942F007021A61704700BF30
:103D300000ED00E08FD00300540300215C0300215C
:103D400008B5FFF7C3FF0B4B0B4A1868116808440E
:103D5000106000221A60094A09491368C01AB0FBB2
:103D6000F1F001FB0033136003F0CEFBBDE8084027
:103D7000FDF7ECBF5C030021500300214C03002140
:103D800090D00300F8B5454C59B1421C09D14FF011
:103D9000E022136923F0010313614FF07F43236096
:103DA000F8BD431C266836D0012836DD422836DCB3
:103DB000471E4FF02003EFF3118583F31288BFF302
:103DC0006F8F374800F0E8FD68B98E23354A3649D1
:103DD000364804F042FC3249354804F03EFC8E215E
:103DE000304804F096FE2E4800F0F2FDFFF76EFF1B
:103DF0004FF0E02300222F49D3F818C00B68184475
:103E00002D4B08601A602D4B1A68831A09D543F6AA
:103E10000953236019E04220CAE70027C9E7422777
:103E2000C7E7DFF89CE0121A0EFB073303F5743383
:103E30008F33B3FBFEF30EFB032343F60952934289
:103E400029D9204A9342E4D922604FF0E022246825
:103E50009369013C546100249C4538BFB444ACEBE9
:103E6000030C6044946108600D4800F0A3FD68B93C
:103E7000B9230C4A14490D4804F0EFFB08491348D4
:103E800004F0EBFBB921074804F043FE85F31188E9
:103E9000BFF36F8F84E71346BBE700BF54030021D5
:103EA00058030021FDBF060123C0060171A90601C8
:103EB00038C00601500300215C0300214C0300219F
:103EC00090D0030020C5FB0050C0060167C006016A
:103ED00038B54FF02003EFF3118583F31288BFF359
:103EE0006F8F1B4800F058FD68B98E23194A1A4994
:103EF0001A4804F0B2FB1649194804F0AEFB8E21B3
:103F0000144804F006FE124800F062FDFFF7DEFEE2
:103F1000144B1C68144B1B68E41A04440C4800F052
:103F200049FD68B9B9230B4A10490C4804F095FBC8
:103F300007490F4804F091FBB921064804F0E9FD58
:103F400085F31188BFF36F8F0A48B4FBF0F038BDDA
:103F500058030021FDBF060123C0060171A9060117
:103F600038C00601500300214C03002150C0060157
:103F700067C0060190D0030038B54FF02003EFF37F
:103F8000118583F31288BFF36F8F194800F004FD89
:103F900068B98E23174A1849184804F05EFB144983
:103FA000174804F05AFB8E21124804F0B2FD104865
:103FB00000F00EFDFFF78AFE124B1C6804440C480B
:103FC00000F0F8FC68B9B9230A4A0F490B4804F01D
:103FD00044FB07490D4804F040FBB921054804F0B3
:103FE00098FD85F31188BFF36F8F204638BD00BF61
:103FF00058030021FDBF060123C0060171A9060177
:1040000038C006015003002150C0060167C00601F8
:104010002DE9F04304460D4617469946A3B0EFF349
:10402000058313BB04F003FEF8B14FF0FF311648CF
:104030000A469C2603DF20BB684604F0F6FD4A468C
:1040400039462A9B2846A0470446684604F0EEFD00
:10405000EFF305838BB904F0EAFD70B10A489D26A1
:1040600003DF204623B0BDE8F0834FF0FF324FF06E
:10407000FF33054800F074FDDDE7034800F096FECD
:10408000EFE71F24EDE700BFE428002138B5054C19
:10409000054DAC4200D338BD204605F01EFC183457
:1040A000F7E700BF2C9A0601C49B06010E4B70B5C2
:1040B00053F82040013053F82060A64200D870BD6C
:1040C000D4E900352846984765B1EB6830B100283F
:1040D000B8BF4042FF28A8BFFF2018705A7842F0AE
:1040E00001025A700834E8E720A2060170B50546BF
:1040F00010B90024204670BD0378002BF9D00E4C77
:104100000E4EB44208D10C4CB442F2D0204605F019
:104110001CFA50B91834F7E7204605F016FA10B12A
:104120002368AB42E6D01834EBE72846216804F058
:1041300011FE0028EED1DDE72C9A0601C49B060192
:1041400010B50B4C8CB0109AA3680146C3F88020C0
:104150006846302204F052F840B96846FFF7C6FFBF
:104160000022A368C3F880200CB010BD0020F7E740
:1041700060030021F8B5124E089AB3680546C3F8EB
:104180008020FCF75DFA01220021074603F0D8FFEA
:10419000044670B100233A46294603F05FFF094800
:1041A0004521094A04F011FDB368D3F8800004F0FA
:1041B0002AFD284605F0C9F9B368C3F88040F8BD68
:1041C000600300214AB506017CC006010022034BB2
:1041D0009B68186EC3F88020704700BF6003002101
:1041E00010B504464521034804F0EFFC204605F0D5
:1041F000B6F900BF93C00601F7B504460E464FF06E
:104200002003EFF3118783F31288BFF36F8F02F05F
:104210000DFD0022042C98BF1F4B054694BF53F898
:1042200024301E4B0092452122461D4804F0CDFC4F
:104230003EB1F369C3F308031BB14521194804F0EB
:10424000C4FC35B1284605F0AAF9034608B1027846
:1042500002B9154B2A464521144804F0B6FC3146F4
:104260002046FFF7BDFF042C0CD111498F23114AC2
:10427000114804F0F2F9114804F0EFF98F210D48CC
:1042800004F047FC87F31188BFF36F8F284603B013
:10429000BDE8F040FEF758B838A20601A7C00601F5
:1042A000BDC00601EAC00601B5C0060110C1060185
:1042B0004FC106012DC1060171A906016CC106019D
:1042C000982310B50F4C012203FB0044002386B055
:1042D000CDE904230F22CDE90232182201930A4BC3
:1042E0000A4902FB00334FF4A072009302FB001155
:1042F000074B204600F0ECF8637B23F00403637364
:1043000006B010BD98000021600300218004002148
:10431000CD4A0601012208B5094B02201A70FFF7A9
:10432000C5FE03F097FF0320FFF7C0FE00F090FAF0
:10433000FCF7DEFB034A137B23F00103137308BD74
:1043400079040021300100210248034A0021121A99
:1043500004F017BD000000217C04002180B5DFF8C7
:10436000B880ACB088F308880024E0232B4D2C4E95
:1043700085F82230EC772C766C76AC766B6ADFF8B9
:10438000A49043F4E0236B62FDF75CFFFDF762FA53
:104390004FF0FF33AB62EB62FEF770FAFDF7E6FF1A
:1043A00040F20113ADF824301F4BCDE91F44249394
:1043B00006ABB3602794FFF769FE2046FFF776FE51
:1043C0000120FFF773FE02F0A9F9184B184D059371
:1043D000012318494FF42062CDE9034328464B4698
:1043E000CDE901440094B56100F072F807466A7B9C
:1043F000284622F004026A7301F032FD2046FFF7DE
:104400005FFF0D4B4A4639462846F3603475C6F8BF
:104410000480FDF7D1FB00BFC00D002100ED00E0DE
:104420006003002115430601A4030021EBC106012E
:1044300030010021C01500219800002152EA03013B
:1044400010B402D110BC01F053BD024910BC1830A9
:1044500002F056BE8D6006010022034B6FF057003C
:104460009B68C3F880207047600300210022034B43
:104470006FF057009B68C3F88020704760030021ED
:1044800070B505460F4E069AB368C3F88020FCF756
:10449000D7F800230922294605F06AF8044648B1F6
:1044A00009484521094A04F090FBB368D3F880001D
:1044B00004F0A9FB284601F01BFDB3682046C3F8B1
:1044C000804070BD600300214AB50601D4C50601D5
:1044D0002DE9FF47DDE90FA8BAF10F0F04460E469C
:1044E00015461F4661D1464B9F4262D118F0040F1A
:1044F00014D0304605F055F880B940F20223414A05
:104500004149424804F0A9F821464148324604F0A6
:10451000A4F840F202213B4804F0FBFA4FF00009F6
:10452000204605F0DAF9304605F0D7F9E667C4F819
:1045300080902046214605F0C5F904F15803C4E9EE
:10454000163304233046C4E90699C4F8089084F869
:104550000C80637384F80EA084F80F9005F021F8A6
:1045600000283AD01F3525F01F0573191A1FC4E91A
:1045700018260822A566A3F108050E9B3146029372
:104580000D9BE26601930C9B2A46009320463B4616
:10459000FDF7CCFA00231F4E6365B3680BBB2846BA
:1045A000C4F8843004B0BDE8F0870AF110031E2B74
:1045B0009CD940F2FF13134A1749144804F04DF8F0
:1045C00051466FF00F030E22144804F046F840F2F3
:1045D000FF110C4804F09DFA88E7073525F0070520
:1045E000C3E7204603F0A4FB18F0080F03D02146D0
:1045F000B06803F00BFDB368D3F88430CFE700BF99
:10460000CD4A0601F3C10601C7C2060171A9060120
:104610000AC306016003002116C2060196C2060104
:104620002DE9F04387B00446DDE914980D4616469F
:104630001F46EFF3058373B1174940F26E23174A03
:10464000174804F00AF8174804F007F840F26E2102
:10465000124804F05EFA00230593129B324604933D
:10466000119B29460393109B204602930F9B0193B5
:104670000E9B00933B46FFF72BFFB8F1FF3F08BFAF
:10468000B9F1FF3F04D04A4643462046FFF7D6FE25
:10469000204607B0BDE8F08335C30601F3C106012B
:1046A00071A9060147C306012DE9F04F054687B001
:1046B0000E46DDE916AB17469946FBF7C1FF4FF0F2
:1046C000FF330922294604F053FF354C002857D008
:1046D0004521344A344804F078FAA368D3F88000BE
:1046E00004F091FA149B5B0735D445212D4A2F48DD
:1046F000F1E70593149B3A460493139B31460393C9
:10470000129B28460293119B0193109B00934B46EA
:10471000FFF7DEFEBBF1FF3F08BFBAF1FF3F04D059
:1047200052465B462846FFF789FE284607B0BDE89B
:10473000F08FA268139992F90E208A42D9DD4521A3
:10474000184A1B48C7E7139A10321E2AF1D945218F
:10475000144A1848BFE7149B13F00103F3D0452116
:10476000104A1548B7E7D8F808301B68BB42B9D2E1
:10477000009345213B460B4A104804F026FAACE76B
:104780003046FBF75DFF4FF0FF330B22314680468A
:1047900004F0EEFE0028E6D04521024A08489AE7D8
:1047A00060030021BDC506014AB50601DFC306014D
:1047B0007EC4060145C406010EC406019BC3060162
:1047C0006CC306012DE9F0471D4E88B0119C91463F
:1047D0009A46129AB3680746C3F88020884600229A
:1047E0001421204604F060FA054670B1154B1648B6
:1047F0000193142345210093144A234604F0E5F95C
:10480000B368D3F8800004F0FEF9D4E90423CDE9BD
:104810000623E3684A460493A3684146039363680A
:104820003846029323680193109B00935346FFF789
:104830003BFFB368C3F8805008B0BDE8F08700BF05
:10484000600300216AD10601E3A80601A6C506019E
:104850002DE9F043474C484D484F87B0AC422646BF
:104860000ED9474940F2D5233A46464803F0F5FEB3
:10487000454803F0F2FE40F2D521384604F049F9EC
:10488000AE4204F1300435D3404C414FDFF8EC80A8
:10489000BC420ED93F4940F2CA234246394803F090
:1048A000DCFE394803F0D9FE40F2CA21404604F04C
:1048B00030F9BC4244D301F081F82E4C2F4E304FDA
:1048C000DFF8C080AC420ED939464FF43D73324612
:1048D000404603F0C2FE2C4803F0BFFE4FF43D718A
:1048E000304604F016F9AC422CD307B0BDE8F043D3
:1048F00001F048BE54F8043C059354F8103C04936E
:1049000054F8143C039354F8183C029354F81C3C9C
:10491000019354F8203C009354E90A2354E90C0114
:10492000FFF7D6FD54F8303C5E6597E7216804F048
:10493000C9FF6368985904360028F7D10834A7E7FF
:104940000026F6E7606A431C12D020EAE070C11727
:1049500009304FF00A024FF0000341F10001FBF76C
:1049600053FFD4F8009002460B464846FFF766FD19
:104970003034A7E7E4280021E4280021F3C1060130
:10498000D0C4060171A90601FDC40601C49F060139
:10499000C49F06011CC50601006838B1044B00F035
:1049A00003001B7DC01A18BF01207047012070470B
:1049B00060030021054903468A68087D196802439F
:1049C0000020914204BF186001207047600300215D
:1049D000024A117D93680B43036070476003002116
:1049E00038B505460E4C069AA368C3F88020FBF73D
:1049F00027FE00230922294604F0BAFD48B10948E0
:104A00004521094A04F0E1F8A368D3F8800004F0D6
:104A1000FAF8A368C3F880006FF0850038BD00BFC6
:104A2000600300214AB506018FC5060170B5054631
:104A30000F4E069AB368C3F88020FBF701FE0023EF
:104A40000922294604F094FD044648B1094845214D
:104A5000094A04F0BAF8B368D3F8800004F0D3F838
:104A600005F1180002F062FCB368C3F8804070BD25
:104A7000600300214AB5060167C5060170B5054609
:104A80000F4E069AB368C3F88020FBF7D9FD0023C8
:104A90000922294604F06CFD044648B10948452125
:104AA000094A04F092F8B368D3F8800004F0ABF838
:104AB00005F1180002F086FCB368C3F8804070BDB1
:104AC000600300214AB5060141C5060108B50D4B3A
:104AD0009B6893F90E30002B09DA0B490B4827230A
:104AE0000B4A03F0BAFD2721094804F012F84FF0F1
:104AF0002002EFF3118382F31288BFF36F8FFCF76C
:104B0000AFFEF4E7600300210BC6060171A90601A0
:104B1000EAC5060170B505460E4E069AB368C3F89D
:104B20008020FBF78DFD0122294604F041FD04465B
:104B300048B109484521094A04F047F8B368D3F859
:104B4000800004F060F8284604F049FDB368C3F81B
:104B5000804070BD600300214AB506011AC70601F6
:104B60002DE9F341044617461E46EFF3058363B172
:104B70006D4965236D4A6E4803F06FFD6D4803F083
:104B80006CFD6521694803F0C4FF4FF02003EFF38B
:104B9000118883F31288BFF36F8F6748FFF7FCFE1D
:104BA00068B98E23654A6649614803F056FD62493B
:104BB000644803F052FD8E21604803F0AAFF5E486E
:104BC000FFF706FFE368604AFBB1A068916888427E
:104BD0003DD057EA06033CD15748FFF7EBFE68B9D2
:104BE000B923564A5949524803F037FD52495848AB
:104BF00003F033FDB921514803F08BFF88F311888E
:104C0000BFF36F8F6FF00F001EE0916891F90E10E7
:104C10000133E360936848482161A360FFF7CAFE4F
:104C200068B9B923454A4949414803F016FD42494C
:104C3000474803F012FDB921404803F06AFF88F3AA
:104C40001188BFF36F8F002002B0BDE8F0812169A9
:104C5000DEE791F90E1090F90E306FF07E02994266
:104C6000A8BF19469142B8BF11468B4243DD04F0FC
:104C7000AEFC054622464146CDE900762E4801F0BD
:104C800019FB0028E0D04FF02003EFF3118683F3E7
:104C90001288BFF36F8F2848FFF77EFE68B98E2316
:104CA000264A2749224803F0D8FC2349254803F027
:104CB000D4FC8E21214803F02CFF1F48FFF788FE0B
:104CC000236821699C420AD04BB193F90E30994276
:104CD000A8BF19466FF07E039942B8BF1946A06875
:104CE00004F075FC00B945B13146134800F022FECE
:104CF0006FF00A00A8E70025BCE70F48FFF75AFE4F
:104D000068B9B9230D4A1149094803F0A6FC0A49BC
:104D10000F4803F0A2FCB921084803F0FAFE86F31D
:104D20001188BFF36F8FE3E735C3060133C6060171
:104D300071A9060155C6060184030021FDBF0601C5
:104D400023C0060138C006016003002150C00601DF
:104D500067C006012DE9F0410546114E1746B368BC
:104D6000089A8846C3F88020FBF76AFC002229468F
:104D700004F01EFC044648B10A4845210A4A03F0E3
:104D800024FFB368D3F8800003F03DFF3B46424662
:104D90002846FFF7E5FEB368C3F88040BDE8F08120
:104DA000600300214AB5060106C7060138B504466E
:104DB000EFF3058363B15049C723504A504803F0CD
:104DC0004CFC504803F049FCC7214C4803F0A1FEBD
:104DD000A368002B00F08A804B4DAA68934240F0F4
:104DE0008880E3684BB949494548DF23434A03F0CB
:104DF00034FCDF21414803F08CFEEFF3058363B1FF
:104E00003D49FD23424A3E4803F027FC414803F058
:104E100024FCFD213E4803F07CFEAB68DB7B012BCC
:104E20000CD13D49FE233A4A354803F016FC394877
:104E300003F013FCFE21364803F06BFEAA68D37B17
:104E4000013BD373E368012B05D9013BE36001F01B
:104E500099FB002038BD4FF02003EFF3118583F359
:104E60001288BFF36F8F2D48FFF796FD68B98E2328
:104E70002B4A2C49224803F0F0FB28492A4803F02A
:104E8000ECFB8E21264803F044FE2448FFF7A0FDEA
:104E90002169A06804F09BFB204601F0EFFBA060B5
:104EA00060B190F90E2022610022C0F88C2000F041
:104EB000D7FF2946194800F03DFDC8E7E0601748D4
:104EC000FFF778FD68B9B923154A18490C4803F073
:104ED000C4FB1249164803F0C0FBB921104803F087
:104EE00018FE85F31188BFF36F8FB0E76FF01500E0
:104EF000B0E74FF0FF30ADE735C3060133C606011A
:104F000071A9060155C60601600300217AC6060193
:104F100091C60601BCC60601BFC606018403002176
:104F2000FDBF060123C0060138C0060150C00601BE
:104F300067C0060170B505460E4E069AB368C3F801
:104F40008020FBF77DFB0022294604F031FB04465C
:104F500048B109484521094A03F037FEB368D3F840
:104F6000800003F050FE2846FFF720FFB368C3F827
:104F7000804070BD600300214AB50601F0C60601FD
:104F80002DE9F04704460E46904699469DF820A02C
:104F900000F108054FF02003EFF3118783F3128827
:104FA000BFF36F8F2846FFF7F7FC68B98E233A4AA4
:104FB0003A493B4803F051FB29463A4803F04DFB80
:104FC0008E21354803F0A5FD2846FFF701FDBAF113
:104FD000000F00D0666804F10C0001F04FFB60B1D7
:104FE0000024C0F81480C0F88C4000F039FF284637
:104FF000394600F09FFC00201EE0B9F1000F2ED0D2
:10500000082102F0E3FBC8B92846FFF7D3FC68B9D2
:10501000B923214A2449224803F01FFB294623488B
:1050200003F01BFBB9211C4803F073FD87F31188C3
:10503000BFF36F8F6FF00B00BDE8F0870123C0F85E
:1050400004800360036803F0030266B92368134316
:10505000036063682060002BC9D16060C7E74046E9
:10506000C8F80090EEE7336833F003030BD1026019
:10507000626812B9C4E90000B9E7136803F00303DA
:1050800003431360E9E713430360336803F003034A
:1050900018433060ABE700BFFDBF060123C0060127
:1050A00071A9060138C0060150C0060167C006019B
:1050B00070B505460F4E069AB368C3F88020FBF71B
:1050C000BFFA4FF0FF32294604F093FA044648B184
:1050D00009484521094A03F078FDB368D3F88000F8
:1050E00003F091FD284604F09FFAB3682046C3F808
:1050F000804070BD600300214AB50601DFC706018C
:1051000070B5054600F108044FF02003EFF3118657
:1051100083F31288BFF36F8F2046FFF73DFC68B919
:105120008E23104A1049114803F097FA214610487F
:1051300003F093FA8E210B4803F0EBFC2046FFF7B7
:1051400047FC05F10C0001F099FA28B10022C0F8E3
:105150008C20426100F084FE31462046BDE870405C
:1051600000F0E8BBFDBF060123C0060171A90601DE
:1051700038C0060170B505460F4E069AB368C3F8ED
:105180008020FBF75DFA0022294604F032FA04463B
:1051900048B10A4845210A4A03F017FDB368D3F81D
:1051A000800003F030FD2846FFF7AAFFB3682046D1
:1051B000C3F8804070BD00BF600300214AB50601FE
:1051C000C4C70601F8B505460F4E089AB3680F46E6
:1051D000C3F88020FBF734FA0022294604F009FACC
:1051E000044648B109484521094A03F0EEFCB3687A
:1051F000D3F8800003F007FD3946284604F01EFA74
:10520000B368C3F88040F8BD600300214AB50601C9
:10521000A8C70601F8B505460F4E089AB3680F46B1
:10522000C3F88020FBF70CFA0022294604F0E1F9CC
:10523000044648B109484521094A03F0C6FCB36851
:10524000D3F8800003F0DFFC3946284604F000FA6A
:10525000B368C3F88040F8BD600300214AB5060179
:105260008BC706012DE9F743064690461F4600F11D
:1052700008054FF02003EFF3118983F31288BFF381
:105280006F8F2846FFF788FB68B98E23254A264989
:10529000264803F0E2F92946254803F0DEF98E217D
:1052A000204803F036FC2846FFF792FB34683CB3F5
:1052B0002368726823F00303944220464FF00101F3
:1052C000336008BF736004F0A3F904462846FFF773
:1052D00071FB68B9B923134A1649144803F0BDF9A4
:1052E0002946154803F0B9F9B9210E4803F011FC1D
:1052F00089F31188BFF36F8F204603B0BDE8F083B8
:1053000058EA0703E2D049462846CDE9008706F16E
:105310000C0200F0CFFF0028EED1084B9B685C69BF
:10532000EAE700BFFDBF060123C0060171A906011F
:1053300038C0060150C0060167C0060160030021A5
:105340002DE9F0410546114E1746B368089A884684
:10535000C3F88020FBF774F90022294604F049F9CC
:10536000044648B10A4845210A4A03F02EFCB368B6
:10537000D3F8800003F047FC3B4642462846FFF73F
:1053800071FFB368C3F88040BDE8F081600300217D
:105390004AB5060178C7060138B504460E4D069A8F
:1053A000AB68C3F88020FBF74BF90022214604F0DC
:1053B00020F948B109484521094A03F006FCAB68C9
:1053C000D3F8800003F01FFC2368AA68C2F88000AD
:1053D000B3FA83F0400938BD600300214AB50601E5
:1053E00060C7060170B505460E4E069AB368C3F84D
:1053F0008020FBF725F90022294604F0FAF804463C
:1054000048B109484521094A03F0DFFBB368D3F8E6
:10541000800003F0F8FB284604F024F9B368C3F8D1
:10542000804070BD600300214AB5060147C70601F0
:1054300070B505460E4E069AB368C3F88020FBF798
:10544000FFF80022294604F0D4F8044648B1094880
:105450004521094A03F0B9FBB368D3F8800003F093
:10546000D2FB284604F002F9B368C3F8804070BD4F
:10547000600300214AB506012EC7060170B5044637
:105480000D461646FBF7DCF80122214604F0F2F83F
:1054900050B109484521094A03F097FB084B9B6826
:1054A000D3F8800003F0AFFB324629462046BDE822
:1054B000704004F0EEB800BF4AB50601AFC806015F
:1054C0006003002138B5064C069DA368C3F88050E0
:1054D000FFF7D4FF0022A368C3F8802038BD00BFC7
:1054E0006003002138B504464FF02003EFF3118527
:1054F00083F31288BFF36F8F1548FFF74DFA68B931
:105500008E23144A1449154803F0A7F8104914488B
:1055100003F0A3F88E210F4803F0FBFA0C48FFF7C5
:1055200057FA204601F0AAF850B10022C0F88C20AA
:1055300000F096FC2946BDE83840054800F0FAB96D
:10554000D4E902329A4218BF0133A360F2E700BFE8
:1055500088030021FDBF060123C0060171A90601D1
:1055600038C0060170B505460F4E069AB368C3F8F9
:105570008020FBF765F80022294604F07BF80446FA
:1055800048B10A4845210A4A03F01FFBB368D3F823
:10559000800003F038FB2846FFF7A4FFB3682046DD
:1055A000C3F8804070BD00BF600300214AB506010A
:1055B0009DC80601F7B5044616461D46EFF3058360
:1055C0007BB152EA05030CD035497923354A364878
:1055D00003F043F8354803F040F87921314803F0EF
:1055E00098FA4FF02003EFF3118783F31288BFF38B
:1055F0006F8F2F48FFF7D0F968B98E232D4A2E49B7
:10560000294803F02AF82A492C4803F026F88E216D
:10561000284803F07EFA2648FFF7DAF9A368D3B1E9
:10562000013B2348A360FFF7C5F968B9B923214AB4
:1056300023491D4803F011F81D49224803F00DF8D5
:10564000B9211C4803F065FA87F31188BFF36F8F07
:10565000002003B0F0BD56EA050318D11448FFF747
:10566000A9F968B9B923134A15490F4802F0F5FFA3
:105670000F49144802F0F1FFB9210E4803F049FA2E
:1056800087F31188BFF36F8F6FF00F00E1E72246B9
:105690003946CDE90065064800F00CFED9E700BFA9
:1056A00013C80601F3C7060171A90601BCC60601AD
:1056B00088030021FDBF060123C0060138C0060192
:1056C00050C0060167C0060170B504464FF02003C4
:1056D000EFF3118583F31288BFF36F8F1348FFF741
:1056E0005BF968B98E23124A1249134802F0B5FFDC
:1056F0000E49124802F0B1FF8E210D4803F009FA5D
:105700000A48FFF765F96FF00A06204600F0B6FF79
:1057100020B1C0F88C6000F0A3FBF6E7A06029463A
:10572000BDE87040014800F005B900BF88030021C2
:10573000FDBF060123C0060171A9060138C006019C
:105740002DE9F0410546114E1746B368089A884680
:10575000C3F88020FAF774FF0022294603F08AFF7D
:10576000044648B10A4845210A4A03F02EFAB368B4
:10577000D3F8800003F047FA3B4642462846FFF73D
:1057800019FFB368C3F88040BDE8F08160030021D1
:105790004AB506018BC8060170B505460F4E069A3C
:1057A000B368C3F88020FAF74BFF0022294603F0C4
:1057B00061FF044648B10A4845210A4A03F005FA48
:1057C000B368D3F8800003F01EFA2846FFF77CFF89
:1057D000B3682046C3F8804070BD00BF600300215D
:1057E0004AB5060178C8060138B504460D4D069A3B
:1057F000AB68C3F88020FAF723FF0022214603F0AC
:1058000039FF034648B108484521084A03F0DDF94D
:10581000AB68D3F8800003F0F6F9AA68A068C2F874
:10582000803038BD600300214AB5060161C8060119
:1058300010B5084C23685BB1FEF74AFB03462068AD
:10584000054A03440021BDE81040136101F00CBE7D
:1058500010BD00BF980300216003002170B504460D
:105860000D464FF02003EFF3118683F31288BFF348
:105870006F8F2648FFF790F868B98E23244A254990
:10588000254802F0EAFE2149244802F0E6FE8E2176
:105890001F4803F03EF91D48FFF79AF80023204AFD
:1058A00014F1090013614FF0FF3243F1000182420D
:1058B0008B4121D30A23B0FBF3F0002C194B20DCE1
:1058C0001860194B1D60FFF7B3FF1048FFF772F81F
:1058D00068B9B9230E4A15490F4802F0BEFE0B49BC
:1058E000134802F0BAFEB921094803F012F986F311
:1058F0001188BFF36F8F70BD0A220023FAF784FF6F
:10590000DBE70228B8BF0220DAE700BF90030021DE
:10591000FDBF060123C0060171A9060138C00601BA
:1059200060030021980300219403002150C0060168
:1059300067C0060138B504460D46E9B9EFF30583A3
:10594000D3B9194B9A699B689A4215D0FFF732F880
:1059500068B9D023154A1649164802F07EFE214642
:10596000154802F07AFED021104803F0D2F8BDE8C5
:1059700038400020FCF72EB82046FFF71BF868B926
:10598000B9230A4A0A490B4802F067FE21460A4831
:1059900002F063FEB921054803F0BBF885F31188D6
:1059A000BFF36F8F38BD00BF60030021FDBF06014C
:1059B00050C0060171A9060167C0060138B54FF055
:1059C0002003EFF3118583F31288BFF36F8F29480B
:1059D000FEF7E2FF68B98E23274A2849284802F0DB
:1059E0003CFE2449274802F038FE8E21224803F06D
:1059F00090F82048FEF7ECFFEFF3058363B12249EE
:105A0000FD23224A1E4802F028FE214802F025FE0E
:105A1000FD211E4803F07DF81E4CA368DB7B012BA3
:105A20000CD11D49FE23194A154802F016FE1848EC
:105A300002F013FEFE21154803F06BF8A268D37B39
:105A4000013BD3730B48FEF7B5FF68B9B9230A4A87
:105A500012490B4802F001FE0649114802F0FDFD13
:105A6000B921054803F055F885F31188BFF36F8F0E
:105A700038BD00BF90030021FDBF060123C0060111
:105A800071A9060138C0060135C3060191C6060199
:105A9000BCC6060160030021BFC6060150C0060156
:105AA00067C006010C4B10B599420C460BD10B494F
:105AB0000B4840F2E7330B4A02F0CFFD40F2E731EA
:105AC000084803F026F8D4E9003213605A60002336
:105AD000C4E9003310BD00BF98000021E3C80601EF
:105AE00071A90601C1C80601836810B504465BB9F7
:105AF0000B490C4840F283230B4A02F0AEFD40F202
:105B00008321094803F005F82146A068FFF7CAFF82
:105B1000637B23F0020363730023A36010BD00BF07
:105B200004C9060171A90601C1C8060138B50446B9
:105B30004FF02003EFF3118583F31288BFF36F8FCB
:105B40001948FEF729FF68B98E23184A18491948E1
:105B500002F083FD1449184802F07FFD8E2113489E
:105B600002F0D7FF1048FEF733FF2046FFF7BCFFD7
:105B70000D48FEF71FFF68B9B9230C4A0F490D48BD
:105B800002F06BFD08490E4802F067FDB921074895
:105B900002F0BFFF85F31188BFF36F8F04F1180087
:105BA000BDE8384001F074BB90030021FDBF060141
:105BB00023C0060171A9060138C0060150C00601C4
:105BC00067C0060138B50246144803F0ABFD144D1A
:105BD000044600B9EC68CAB9AB6863B911498923B6
:105BE000114A124802F039FD114802F036FD8921B0
:105BF0000D4802F08EFFAB685A7BD20606D1A2692F
:105C000022B9DA897F2A01D9AB6138BDAB68A342DA
:105C100001D0FFF70DFEAC61F7E700BF7C03002168
:105C2000600300211BC90601C1C8060171A9060154
:105C3000BCC6060170B590F90D200446002A437BCE
:105C400006DA03F07F03014643731E48FFF72AFF7D
:105C5000637B63F07F0363731B4B9C4209D11B4939
:105C60001B48BA231B4A02F0F8FCBA21194802F07B
:105C700050FF194A02F11C05D2E90730AB421BD094
:105C8000D3B194F90E6093F90E108E420FD0891B98
:105C900000290CDD5968C4E900310C605C60906833
:105CA000031B58425841BDE87040FFF78BBF834249
:105CB00002D01B68002BE6D1C4E9005004601462D6
:105CC000EDE700BF7C03002198000021E3C8060136
:105CD00071A90601C1C806016003002138B5044658
:105CE0004FF02003EFF3118583F31288BFF36F8F1A
:105CF0002948FEF751FE68B98E23284A28492948C9
:105D000002F0ABFC2449284802F0A7FC8E2123486E
:105D100002F0FFFE2048FEF75BFE244B244A986801
:105D20001168884218D1FFF783FD1B48FEF742FE39
:105D300068B9B923194A1F491A4802F08EFC16495E
:105D40001D4802F08AFCB921144802F0E2FE85F3F6
:105D50001188BFF36F8F38BD00211160174A126898
:105D6000BAB1C2897F2A14D8427BD20611D1144A13
:105D700090F90E10126891420BDB124A904208D043
:105D80001A69A24202DCFFF755FFCCE7121B1A6129
:105D9000CBE70022FBE700BF90030021FDBF060117
:105DA00023C0060171A9060138C006016003002165
:105DB0008C03002150C0060167C006019803002132
:105DC000940300219800002170B590F90D2004463D
:105DD000002A437B39DBDA0637D18269002A34D1C5
:105DE00063F07F034373194B984209D1184919484E
:105DF000BA23194A02F031FCBA21174802F089FE91
:105E0000164A02F11C05D2E90730AB4218D0BBB1EB
:105E100094F90E6093F90E108E420CD0891B002964
:105E200009DD5A68C4E9003214605C600020BDE8F6
:105E30007040FFF7C7BE984202D01B68002BE9D123
:105E4000C4E9005004601462F0E770BD98000021BE
:105E5000E3C8060171A90601C1C80601600300215B
:105E600038B504464FF02003EFF3118583F3128811
:105E7000BFF36F8F1748FEF78FFD68B98E23164A60
:105E80001649174802F0E9FB1249164802F0E5FBF3
:105E90008E21114802F03DFE0E48FEF799FD204686
:105EA000FFF792FF0B48FEF785FD68B9B9230A4A50
:105EB0000D490B4802F0D1FB06490C4802F0CDFB1E
:105EC000B921054802F025FE85F31188BFF36F8FD5
:105ED00038BD00BF90030021FDBF060123C00601AD
:105EE00071A9060138C0060150C0060167C006014D
:105EF00038B504464FF02003EFF3118583F3128881
:105F0000BFF36F8F1D48FEF747FD68B98E231C4A0B
:105F10001C491D4802F0A1FB18491C4802F09DFBDA
:105F20008E21174802F0F5FD1448FEF751FD637B02
:105F30005A0716D41148FEF73DFD68B9B923104A37
:105F40001349114802F089FB0C49124802F085FB05
:105F5000B9210B4802F0DDFD85F31188BFF36F8F87
:105F600038BD23F0040320466373FFF72DFF294655
:105F7000BDE838400148FFF7DDBC00BF90030021B9
:105F8000FDBF060123C0060171A9060138C0060144
:105F900050C0060167C0060138B504464FF0200323
:105FA000EFF3118583F31288BFF36F8F1D48FEF75F
:105FB000F3FC68B98E231C4A1C491D4802F04DFBB6
:105FC00018491C4802F049FB8E21174802F0A1FD38
:105FD0001448FEF7FDFC637BDA0616D41148FEF781
:105FE000E9FC68B9B923104A1349114802F035FB9E
:105FF0000C49124802F031FBB9210B4802F089FD2F
:1060000085F31188BFF36F8F38BD23F0100320464E
:106010006373FFF7D9FE2946BDE838400148FFF712
:1060200089BC00BF90030021FDBF060123C006010B
:1060300071A9060138C0060150C0060167C00601FB
:1060400070B505460E4E069AB368C3F88020FAF77D
:10605000F7FA294603F040FB044648B109484521B8
:10606000094A02F0B2FDB368D3F8800002F0CBFD1C
:106070002846FFF791FFB3682046C3F8804070BD03
:10608000600300214AB5060193CB060170B50446B2
:106090004FF02003EFF3118683F31288BFF36F8F65
:1060A0002048FEF779FC68B98E231F4A1F49204813
:1060B00002F0D3FA1B491F4802F0CFFA8E211A488A
:1060C00002F027FD1748FEF783FC14F80B3C13F091
:1060D000280F10D154F8103CA4F1180513B128462C
:1060E000FFF702FD14F80B3C284623F0140304F8D4
:1060F0000B3CFFF769FE0B48FEF75CFC68B9B9235F
:10610000094A0D490A4802F0A8FA06490B4802F06C
:10611000A4FAB921044802F0FCFC86F31188BFF30D
:106120006F8F70BD90030021FDBF060123C00601E3
:1061300071A9060138C0060150C0060167C00601FA
:1061400010B590F90D200446002A437B06DA03F0CF
:106150007F03014643730648FFF7A4FC054B98688C
:10616000031B58425841BDE81040FFF72BBD00BF4C
:106170007C0300216003002138B504460D46FFF77B
:10618000DFFF637B43F002036373FDB1164BA56031
:106190009C4209D115491648BA23164A02F05DFA05
:1061A000BA21144802F0B5FC2B689D4215D0A3B16A
:1061B00094F90E1093F90E20914208D0521A002A39
:1061C00005DD5A68C4E9003214605C6038BD6A6855
:1061D000934202D01B68002BECD16B68C4E90053DA
:1061E0001C606C60F2E700BF98000021E3C8060164
:1061F00071A90601C1C806012DE9F041044688468F
:1062000016461D464FF02003EFF3118783F31288E3
:10621000BFF36F8F1F48FEF7BFFB68B98E231E4A7E
:106220001E491F4802F019FA1A491E4802F015FAD1
:106230008E21194802F06DFC1648FEF7C9FB204676
:106240004146FFF799FF1348FEF7B4FB68B9B9233D
:10625000114A1549124802F000FA0E49134802F09B
:10626000FCF9B9210C4802F054FC87F31188BFF304
:106270006F8FB5F1FF3F08BFB6F1FF3F08D0324640
:106280002B4604F118000A49BDE8F04100F038BF80
:10629000BDE8F08190030021FDBF060123C0060187
:1062A00071A9060138C0060150C0060167C0060189
:1062B0008D60060138B50446104B0D469868104BAA
:1062C00011461860DDE90423FFF796FF2046FEF72C
:1062D00071FB68B9D0230B4A0B490C4802F0BDF999
:1062E00021460B4802F0B9F9D021064802F011FC12
:1062F0002846BDE83840FBF76DBB00BF60030021B6
:106300008C030021FDBF060150C0060171A90601E2
:1063100067C00601F8B504460D464FF02003EFF3C1
:10632000118683F31288BFF36F8F3A48FEF734FB70
:1063300068B98E23384A3949394802F08EF935490F
:10634000384802F08AF98E21334802F0E2FB3148E6
:10635000FEF73EFB637B6DB2DA0657D1A269002AD5
:1063600054D103F07F03637321462F48FFF79AFB54
:10637000637BA57363F07F0363732C4B9C4209D14D
:106380002B492748BA232B4A02F067F9BA2129483A
:1063900002F0BFFB284A02F11C05D2E90730AB42EC
:1063A0002FD073B394F90E7093F90E108F4223D04F
:1063B000C91B002920DD5A68C4E9003214605C6002
:1063C0000120FFF7FFFB01241248FEF7F3FA68B93A
:1063D000B923114A1949124802F03FF90D491848EA
:1063E00002F03BF9B9210C4802F093FB86F31188C7
:1063F000BFF36F8F2046F8BD834202D01B68002B8D
:10640000D2D1C4E9005004601462D9E7A573002416
:10641000DAE700BF90030021FDBF060123C006019B
:1064200071A9060138C006017C03002198000021F3
:10643000E3C80601C1C806016003002150C006017F
:1064400067C0060108B5FFF765FF38B1044B9B68CC
:10645000DB7B1BB9BDE8084003F05AB908BD00BF9B
:106460006003002170B50446183000F011FF4FF0B2
:106470002003EFF3118683F31288BFF36F8F254853
:10648000FEF78AFA68B98E23234A2449244802F089
:10649000E4F82049234802F0E0F88E211E4802F07B
:1064A00038FB1C48FEF794FA94F90D20637B002A10
:1064B00006DA03F07F0321461B486373FFF7F2FA05
:1064C0001A4D637BA86843F010036373031B5842A3
:1064D0005841FFF777FB0F48FEF76CFA68B9B9230C
:1064E0000D4A13490E4802F0B8F80A49114802F063
:1064F000B4F8B921084802F00CFB86F31188BFF309
:106500006F8FAB68A34203D1BDE8704003F000B9C0
:1065100070BD00BF90030021FDBF060123C006012E
:1065200071A9060138C006017C0300216003002127
:1065300050C0060167C0060170B505460E4E069AAA
:10654000B368C3F88020FAF77BF8294603F0C4F853
:10655000044648B109484521094A02F036FBB368B0
:10656000D3F8800002F04FFB2846FFF77BFFB368AB
:106570002046C3F8804070BD600300214AB5060183
:10658000AACB060138B54FF02003EFF3118583F352
:106590001288BFF36F8F2D48FEF7FEF968B98E237E
:1065A0002B4A2C492C4802F058F828492B4802F075
:1065B00054F88E21264802F0ACFA294C2348FEF705
:1065C00007FAA368DB7B73B9264940F28533264A74
:1065D000214802F042F8254802F03FF840F28531A8
:1065E000214802F096FAEFF3058373B1204940F297
:1065F00086331D4A184802F030F81C4802F02DF886
:1066000040F28631184802F084FAA2680020D37B59
:106610000133D373FFF7D6FA0C48FEF7CBF968B90C
:10662000B9230B4A13490C4802F017F807491248DE
:1066300002F013F8B921064802F06BFA85F31188CD
:10664000BFF36F8FBDE8384003F062B890030021BC
:10665000FDBF060123C0060171A9060138C006016D
:106660006003002142C90601C1C80601BCC606017B
:1066700035C3060150C0060167C0060138B504469F
:106680004FF02003EFF3118583F31288BFF36F8F70
:106690001B48FEF781F968B98E231A4A1A491B482C
:1066A00001F0DBFF16491A4801F0D7FF8E2115488B
:1066B00002F02FFA1248FEF78BF9204603F032F869
:1066C000044628B1FFF710FA04F1180000F0E0FDCD
:1066D0000B48FEF76FF968B9B9230A4A0D490B4810
:1066E00001F0BBFF06490C4801F0B7FFB92105488E
:1066F00002F00FFA85F31188BFF36F8F204638BD83
:1067000090030021FDBF060123C0060171A9060107
:1067100038C0060150C0060167C006010021044BC5
:10672000084603F11C02C3E90722FFF797B800BF30
:106730006003002138B504460D4D069AAB68C3F8D6
:106740008020F9F77DFF214602F0C6FF034648B1DD
:1067500008484521084A02F038FAAB68D3F88000AF
:1067600002F051FAAA6894F90E00C2F8803038BDE0
:10677000600300214AB5060176CB060138B501F168
:1067800010031E2B05460C4612D940F2A543144AAD
:106790001449154801F061FF214614486FF00F03BA
:1067A0000E2201F05AFF40F2A5410D4802F0B1F966
:1067B000EFF3058373B10E4940F2A643084A0A4835
:1067C00001F04BFF0B4801F048FF40F2A64104489E
:1067D00002F09FF921462846BDE83840FFF732BE57
:1067E000C1C8060173C9060171A9060196C2060156
:1067F00035C30601BCC60601F7B507461C4E0A9A0A
:10680000B3680C46C3F88020F9F71AFF394602F046
:1068100063FF0546B0B14521164A174802F0D5F985
:10682000B368D3F8800002F0EEF997F90E3062B247
:106830009A4213DA0093452123460E4A0F4802F08C
:10684000C4F9EDE70E2C02DC14F1100FEDDA23464B
:106850004521084A0A4802F0B8F9E1E738462146DE
:10686000FFF78CFF2846B368C3F8805003B0F0BD33
:106870006003002159CB06014AB5060132CA060160
:10688000F9C90601F8B5EFF3058373B13F4940F24A
:10689000DC433F4A3F4801F0E0FE3F4801F0DDFEA7
:1068A00040F2DC413A4802F034F94FF02003EFF3B4
:1068B000118683F31288BFF36F8F3848FEF76CF8A8
:1068C00068B98E23364A3749324801F0C6FE33494B
:1068D000354801F0C2FE8E21314802F01AF9334DDD
:1068E0002E48FEF775F8A96805F11C004B7B03F0F4
:1068F0007F034B73FFF7D6F8AC68637B63F07F03CD
:1069000063732B4B9C4209D12A492248BA23204A5F
:1069100001F0A3FEBA211E4802F0FBF8D5E90731C9
:10692000254883422DD063B394F90E7093F90E205D
:10693000974221D0D21B002A1EDD5A68C4E90032DA
:1069400014605C600120FFF73DF91448FEF732F84F
:1069500068B9D023124A19490E4801F07EFE0F494A
:10696000174801F07AFED0210D4802F0D2F83046E7
:10697000BDE8F840FBF72EB88B4202D01B68002B15
:10698000D4D1C4E900010C602C62DBE735C30601F9
:10699000C1C8060171A90601BCC606019003002109
:1069A000FDBF060123C0060138C0060160030021B7
:1069B00098000021E3C806017C03002150C00601B5
:1069C00067C006012DE9F04105460E46EFF3058349
:1069D00073B143494FF49F63424A434801F03DFE7F
:1069E000424801F03AFE4FF49F613E4802F091F8B0
:1069F00055EA060303D1FFF745FF00206DE06FF075
:106A000001044FF0FF33641B63EB0603012C73F1A9
:106A1000000302DA02F0CBFE44194FF02003EFF33B
:106A2000118883F31288BFF36F8F3148FDF7B4FFED
:106A300068B98E232F4A30492B4801F00EFE2C49AD
:106A40002E4801F00AFE8E212A4802F062F82C4FEF
:106A50002748FDF7BDFFB8682A4B1860FFF770FBA9
:106A6000B8682A4633461830274900F049FBBA680F
:106A70001F48537B43F010035373FDF79BFF68B926
:106A8000D0231C4A2149184801F0E7FD1849204845
:106A900001F0E3FDD021174802F03BF84046FAF739
:106AA00099FFBB685B7BDB060ED51A4940F2195390
:106AB0000C4A0D4801F0D1FD0C4801F0CEFD40F22A
:106AC0001951084802F025F802F071FE201A63EB14
:106AD0000303012873F100038FDBBDE8F08100BFE1
:106AE00035C30601C1C8060171A90601BCC606016D
:106AF00090030021FDBF060123C0060138C0060136
:106B0000600300218C0300218D60060150C0060146
:106B100067C0060181CA060110B5064C049AA36835
:106B2000C3F88020FFF7AEFE0020A368C3F8800002
:106B300010BD00BF6003002138B505460C46EFF3D9
:106B4000058373B111494FF4A563114A114801F04F
:106B500084FD114801F081FD4FF4A5610C4801F05E
:106B6000D8FFB4F1FF3F08BFB5F1FF3F06D10B4B93
:106B70009868FFF777FC4FF0FF3038BD2846214674
:106B8000FFF720FF0A235843F7E700BF35C306018C
:106B9000C1C8060171A90601BCC606016003002137
:106BA00010B5064C049AA368C3F88020FFF7C4FF11
:106BB0000022A368C3F8802010BD00BF600300213D
:106BC00010B5064C049AA368C3F8802002F0C0FDFB
:106BD0000022A368C3F8802010BD00BF600300211D
:106BE00070B505460E4E069AB368C3F88020F9F7D3
:106BF00027FD294602F070FD044648B109484521A9
:106C0000094A01F0E2FFB368D3F8800001F0FBFF0E
:106C1000284602F0B1FDB3682046C3F8804070BD3D
:106C2000600300214AB5060149CB0601014B986873
:106C3000704700BF60030021024B98680023C0F832
:106C40008030704760030021EFF305833BB9054BAB
:106C50009B68D8897F288CBF0020012070470020C6
:106C6000704700BF60030021064A08B50499936885
:106C7000C3F88010FFF7E8FF93680022C3F8802074
:106C800008BD00BF600300212DE9F04104464FF02C
:106C90002003EFF3118683F31288BFF36F8F4E4802
:106CA000FDF77AFE68B98E234C4A4D494D4801F0F4
:106CB000D4FC49494C4801F0D0FC8E21474801F0F2
:106CC00028FF4548FDF784FE637B1A0717D5424825
:106CD000FDF770FE68B9B923404A4449414801F0C4
:106CE000BCFC3D49424801F0B8FCB9213B4801F0E9
:106CF00010FF86F31188BFF36F8FBDE8F08123F09A
:106D0000200242F00801D2094ED16173A36813B189
:106D10002046FEF7E9FE04F1180000F0B9FA4FF042
:106D2000000804F15807A56DBD4201D0002D45D1E2
:106D30000120FEF747FF204601F058F8204601F0F9
:106D40007FF9E06F02F0D2FD204602F0CFFD294B23
:106D50009B68A342BBD1EFF30583002BB7D11E483C
:106D6000FDF728FE68B9D0231C4A20491D4801F0D0
:106D700074FC19491E4801F070FCD021174801F03D
:106D8000C8FE3046FAF726FE40F24B631A4A1B490A
:106D9000144801F062FC1A4801F05FFC40F24B61BC
:106DA000154801F0B6FE92E703F05F0343F00803D5
:106DB000214614486373FEF775FEA7E72846FEF7E1
:106DC00093FE05F1180000F063FA2846C5F88C80A0
:106DD000FEF7FAFFA7E700BF90030021FDBF060101
:106DE00023C0060171A9060138C0060150C0060182
:106DF00067C0060160030021C1C80601EFB70601A4
:106E0000C1CA06017C0300212DE9F0410446164663
:106E10001D464FF02003EFF3118883F31288BFF370
:106E20006F8F3F48FDF7B8FD68B98E233D4A3E4954
:106E30003E4801F012FC3A493D4801F00EFC8E211B
:106E4000384801F066FE3648FDF7C2FD637B1B073C
:106E500045D455EA06035CD0364FBB68A3425BD0ED
:106E6000A26858339A4257D0EFF3058373B1324981
:106E700040F26A63314A2D4801F0EFFB304801F0DF
:106E8000ECFB40F26A612D4801F043FEB86804F162
:106E90005801FFF771F9B5F1FF3F08BFB6F1FF3FA9
:106EA00006D0B86832462B462649183000F028F93B
:106EB0001B48FDF77FFD68B9D0231A4A22491B48B9
:106EC00001F0CBFB1649214801F0C7FBD021154842
:106ED00001F01FFE4046BDE8F041FAF77BBD0024FB
:106EE0000F48FDF767FD68B9B9230E4A16490F48E8
:106EF00001F0B3FB0A49154801F0AFFBB92109487D
:106F000001F007FE88F31188BFF36F8F2046BDE8BC
:106F1000F0816FF00F04E3E76FF02C04E0E700BFAF
:106F200090030021FDBF060123C0060171A90601DF
:106F300038C006016003002135C30601C1C806013F
:106F4000E3CA06018D60060150C0060167C0060154
:106F5000F8B50B4F1546BB68089A0446C3F8802065
:106F60000E4602F0A5FB48B932462B462046FFF7F5
:106F70004BFF0022BB68C3F88020F8BD0020F8E773
:106F80006003002138B50F4D069AAB680446C3F87C
:106F9000802002F08DFB80B9237BDB070AD52346D6
:106FA00009484521094A01F010FEAB68D3F880007A
:106FB00001F029FE2046FBF7C7F90020AB68C3F8B3
:106FC000800038BD60030021F8CA060133CB0601FA
:106FD00009480A4A08B50A49121A01F0C7FE094AC7
:106FE00009490A4801F0C2FEBDE808400848094ABC
:106FF0000949121A01F0BABEC0270021242B002132
:10700000F0DD060100000000F0D5060100000021BF
:107010000000002100000021F0D50601034B1B6891
:107020000BB9FCF755BF0020704700BF9C0300213F
:10703000114B10B51C689C4208BF0024FFF7EEFFFF
:1070400003466CB1D4E90402C01A62EBE373012871
:1070500073F100020DDBB0F1004F73F1000301DBAF
:107060006FF00040054B1B6913B19842A8BF18464A
:1070700010BD0020F6E700BF982800216003002122
:1070800030B5036868B10A4A5268904209D043B1EA
:10709000D3E90421D0E90445121941EB0501C3E904
:1070A0000421426813605A600023C0E9003330BDF8
:1070B0009828002170B50468E4B1104A136893421F
:1070C00015D000242546516833B9FFF7A7FF0146C4
:1070D000201A65EBE17170BDD3E90426A41845EBD5
:1070E00006058342F1D08B42EFD01B68ECE7002409
:1070F0002546EAE720462146EDE700BF9828002113
:10710000B3F1FF3F08BFB2F1FF3F2DE9F041044664
:107110000E46984615461F4600F09E80036863B1F0
:107120004E495D234E4A4F4801F097FA4E4801F010
:1071300094FA5D214A4801F0ECFCA6604FF0200370
:10714000EFF3118683F31288BFF36F8F4748FDF783
:1071500023FC68B98E23464A4649424801F07DFA2D
:107160004249454801F079FA8E21414801F0D1FCAD
:107170003E48FDF72DFC6FF001024FF0FF30531B2E
:1071800060EB0703002B1BDB3C4BD3E90013521AC7
:1071900060EB0303551B63EB0707012D77F1000339
:1071A000BCBF01250027C4E90457354AD2E9003C99
:1071B000934218D1C4E9002CCCF80040546026E07A
:1071C000FFF72CFF013548F100082D1848EBE0705F
:1071D000C4E90450E9E7091A65EB07059C45C4E9D1
:1071E0000415E7D01B68002BE4D0D3E90407D4E9E9
:1071F0000415814275EB070EEDDA411A67EB0505C0
:10720000C3E904155968C4E900310C605C60136877
:1072100093420BD09C4209D1FFF70AFF18B1194BDA
:107220001B69834202D00021FCF7ACFD0F48FDF73B
:10723000C1FB68B9B9230E4A13490A4801F00DFA97
:107240000A49124801F009FAB921094801F061FC24
:1072500086F31188BFF36F8FBDE8F081E6CB06019E
:10726000C2CB060171A90601BCC60601A00300211C
:10727000FDBF060123C0060138C00601C801002178
:10728000982800216003002150C0060167C0060154
:1072900038B504464FF02003EFF3118583F31288CD
:1072A000BFF36F8F1A48FDF777FB68B98E23194A31
:1072B00019491A4801F0D1F91549194801F0CDF9D9
:1072C0008E21144801F025FC1148FDF781FB23684D
:1072D000DBB12046FFF7D4FE00240D48FDF76AFB22
:1072E00068B9B9230B4A0F490C4801F0B6F90849AF
:1072F0000D4801F0B2F9B921064801F00AFC85F306
:107300001188BFF36F8F204638BD6FF01504E4E796
:10731000A0030021FDBF060123C0060171A90601DB
:1073200038C0060150C0060167C0060170B50446AA
:107330004FF02003EFF3118683F31288BFF36F8FB2
:107340001948FDF729FB68B98E23184A18491948CE
:1073500001F083F91449184801F07FF98E21134890
:1073600001F0D7FB1048FDF733FB2046FFF7A2FEE4
:1073700005460D480C46FDF71DFB68B9B9230B4ABD
:107380000E490C4801F069F907490D4801F065F90B
:10739000B921064801F0BDFB86F31188BFF36F8F5A
:1073A0002846214670BD00BFA0030021FDBF060195
:1073B00023C0060171A9060138C0060150C00601AC
:1073C00067C0060170B504464FF02003EFF3118645
:1073D00083F31288BFF36F8F1B48FDF7DDFA68B99E
:1073E0008E231A4A1A491B4801F037F916491A48E0
:1073F00001F033F98E21154801F08BFB1248FDF79F
:10740000E7FA2046FFF756FE144BD3E9004504196E
:107410000D4845EB0105FDF7CDFA68B9B9230B4AD4
:107420000F490C4801F019F907490E4801F015F908
:10743000B921064801F06DFB86F31188BFF36F8F09
:107440002046294670BD00BFA0030021FDBF0601F4
:1074500023C0060171A9060138C00601C801002138
:1074600050C0060167C0060170B504460D464FF0D6
:107470002003EFF3118683F31288BFF36F8F1B484D
:10748000FDF78AFA68B98E23194A1A491A4801F099
:10749000E4F81649194801F0E0F88E21144801F08B
:1074A00038FB1248FDF794FAFFF7C2FD012805DD0D
:1074B000A04203DB29462046FCF764FC0B48FDF79D
:1074C00079FA68B9B9230A4A0D490B4801F0C5F8A1
:1074D00006490C4801F0C1F8B921054801F019FB33
:1074E00086F31188BFF36F8F70BD00BFA00300212A
:1074F000FDBF060123C0060171A9060138C00601BF
:1075000050C0060167C006012DE9F8430446FEF7A6
:10751000E5FB4FF02003EFF3118583F31288BFF3EF
:107520006F8F4C48FDF738FA68B98E234A4A4B49A9
:107530004B4801F092F847494A4801F08EF88E21F5
:10754000454801F0E6FA484F4248DFF82081484EAE
:10755000FDF73EFA3C60D8F800403A6844454FEAEF
:10756000E270D6E9001E0BD054B1D4E9043C9A4233
:1075700070EB0C0928DA9B1A6CEB000CC4E9043C94
:10758000002452184EEB0000C6E900203C60FFF7D3
:107590004FFD2146FCF7F6FB2E48FDF70BFA68B9C4
:1075A000B9232D4A33492E4801F057F8294932486A
:1075B00001F053F8B921284801F0ABFA85F311889E
:1075C000BFF36F8FBDE8F88359184EEBE370D31A01
:1075D0003B6000220023C6E90010C4E904232046D2
:1075E000FFF74EFD1B48FDF7E5F968B9B9231A4AC4
:1075F00020491B4801F031F816491F4801F02DF8C9
:10760000B921154801F085FA85F31188BFF36F8F12
:107610002046A36898474FF02003EFF3118583F3CA
:107620001288BFF36F8F0B48FDF7B6F968B98E2348
:10763000094A0A490A4801F010F80649094801F0C8
:107640000CF88E21044801F064FA0248FDF7C0F9F5
:1076500081E700BFA0030021FDBF060123C0060192
:1076600071A9060138C006019C0300219828002159
:10767000C801002150C0060167C0060170B54FF077
:107680002003EFF3118683F31288BFF36F8F1B483B
:10769000FDF782F968B98E23194A1A491A4800F091
:1076A000DCFF1649194800F0D8FF8E21144801F07C
:1076B00030FA1248FDF78CF9FCF70AFC144BD3E9B9
:1076C000004504190D4845F10005FDF773F968B947
:1076D000B9230B4A0F490C4800F0BFFF07490E4879
:1076E00000F0BBFFB921064801F013FA86F31188B8
:1076F000BFF36F8F2046294670BD00BFA003002155
:10770000FDBF060123C0060171A9060138C00601AC
:10771000C801002150C0060167C00601F7B5134D2E
:107720000A9AAB680446C3F88020FFF7A7FF01223E
:1077300007460E462046082101F0B6FA70B10C4B00
:107740000C4801930823452100930B4A234601F07E
:107750003CFAAB68D3F8800001F055FAAA68C4E996
:107760000076C2F8800003B0F0BD00BF60030021C6
:10777000F4AA0601E3A8060106CC060138B50446C2
:1077800078B1FCF7F9FB054606480023A4FB00018D
:10779000054AF9F739F80446FCF7EEFB431B9C4217
:1077A000FAD838BD40787D0140420F0010B5064C34
:1077B000049AA368C3F88020FFF7E0FF0020A368C5
:1077C000C3F8800010BD00BF6003002173B50646FA
:1077D0000D4601F0DEFE80B9154B9B68D3F884405E
:1077E00014B32A1D09D200200021CDE90001204652
:1077F00046F0040100F064FD08B9002414E00460C0
:10780000041D8EB1731E1C420ED02523094A0A495D
:107810000A4800F022FF21460948324600F01DFFC9
:107820002521044801F075F9204602B070BD00BF63
:10783000600300211CCC060140CC060171A90601A1
:1078400072CC06012DE9F8430E46F8F7F9FE002840
:1078500037D083790F2B34D1876897B307F10805A8
:107860004FF02003EFF3118883F31288BFF36F8F7B
:107870002846FDF791F868B98E23134A1349144836
:1078800000F0EBFE2946134800F0E7FE8E210E487B
:1078900001F03FF900242846FDF79AF8A146384642
:1078A000FEF7ECFE30B1C0F88C900134FEF7D8FA48
:1078B000002EF4D128464146FEF73CF82046BDE8AC
:1078C000F8836FF01500FAE7FDBF060123C006013B
:1078D00071A9060138C006017FB5124E0A9AB36835
:1078E0000391C3F88020CDB201220421044601F0A7
:1078F000DBF988B10C4B0D4801930423452100931B
:107900000B4A234601F061F96FF00C000022B368C6
:10791000C3F8802004B070BD29462046FFF792FFCF
:10792000F4E700BF60030021F4AA0601E3A8060102
:10793000AECC06012DE9F34180460C4617461E46A3
:10794000F8F77EFE002836D083790F2B33D1856877
:107950008DB3D8E8AF3F9C4230D105F108044FF019
:107960002003EFF3118883F31288BFF36F8F204653
:10797000FDF712F868B98E23124A1349134800F034
:107980006CFE2146124800F068FE8E210D4801F081
:10799000C0F82046FDF71CF82A4641462046CDE9AE
:1079A0000076FEF787FC10F10B0F08BF6FF0730035
:1079B00002B0BDE8F0816FF01500F9E76FF00A0042
:1079C000F6E700BFFDBF060123C0060171A906014D
:1079D00038C006012DE9F341DFF8548017461E46F2
:1079E0000A9AD8F808300D46C3F8802004210122F5
:1079F000044601F059F998B10E4B0F480193042346
:107A0000452100930D4A234601F0DFF86FF00C008A
:107A10000022D8F80830C3F8802002B0BDE8F08119
:107A20003A46334629462046FFF784FFF0E700BF79
:107A300060030021F4AA0601E3A806019ACC06011E
:107A4000F0B50D4685B031B94521204801F0BDF8AB
:107A5000002005B0F0BD0C890B68E20708D414F0D3
:107A6000040405D11A464521194801F0AEF8EFE7A4
:107A70006C682CB92A464521164801F0A6F8E7E7BC
:107A8000E7189F4206D9002290F8C8C0624508DB7B
:107A90000120DEE72A4645210F48009401F095F8C1
:107AA000D6E746687EB10168B9420CD206EB010EFA
:107AB0009E4508D9CDE901162A464521074800947C
:107AC00001F083F8C4E701320C30DFE7C2CC0601D5
:107AD000E5CC06011BCD06014BCD06018FCD06017D
:107AE00038B50C46054658B9134914484FF4847309
:107AF000134A00F0B2FD4FF48471114801F009F807
:107B00005CB910490D4840F209130D4A00F0A5FD7B
:107B100040F209110A4800F0FCFFD5F8C42004F136
:107B2000700305F1C001C4E91C1200201360C5F800
:107B3000C430A56738BD00BF02CE060171A9060199
:107B4000DBCD060118CE060110B5044658B90A4926
:107B50000A4840F21B130A4A00F07FFD40F21B1155
:107B6000074800F0D6FFD4E91C32002013605A60A9
:107B7000C4E91C0010BD00BF18CE060171A90601A2
:107B8000DBCD06012DE9F0470F461646044628B125
:107B900039B132B945213C4801F017F86FF01504AE
:107BA0005DE03A4B1B78BB4205D23A464521384846
:107BB00001F00BF8F2E74FF02003EFF3118883F3A5
:107BC0001288BFF36F8F3348FCF7E6FE68B98E2347
:107BD000314A3249324800F040FD2E49314800F028
:107BE0003CFD8E212C4800F094FF00252948FCF72D
:107BF000EFFEC0222946204684F8C85001F0C1F8A3
:107C000004F1C003C4E93033002F3BD04FF00C091E
:107C1000B2462046DAF800100436FFF711FF08BB21
:107C20002A464521DAF800301F4800F0CEFF6FF0F9
:107C300015041848FCF7BEFE68B9B923164A1B495B
:107C4000174800F00AFD1349194800F006FDB92154
:107C5000114800F05EFF88F31188BFF36F8F204654
:107C6000BDE8F08709FB054356F8042C013507CA27
:107C700083E8070094F8C830BD4203F1010384F89B
:107C8000C830C5D30024D4E72ECE06017A040021E3
:107C900060CE060170040021FDBF060123C006016D
:107CA00071A9060138C006019FCE060150C0060129
:107CB00067C0060108B500F0F2FF154BC0B21028EE
:107CC00018700ED913494FF4B173134A134800F0DA
:107CD000C4FC134800F0C1FC4FF4B1710E4800F031
:107CE00018FF00220F481146FFF74CFF70B10E49F4
:107CF00040F26513084A094800F0AFFC0B4800F059
:107D0000ACFC40F26511044800F003FF002008BD00
:107D10007A040021C4CE0601DBCD060171A906015B
:107D2000BCC60601A4030021D9CE0601E2CE06019D
:107D300038B504464FF02003EFF3118583F3128822
:107D4000BFF36F8F1F48FCF727FE68B98E231E4ACA
:107D50001E491F4800F081FC1A491E4800F07DFCB6
:107D60008E21194800F0D5FE1648FCF731FE1A4B5B
:107D700021469B68986FFFF7B3FE58B11749144826
:107D800040F22F13164A00F068FC40F22F111448FD
:107D900000F0BFFE0B48FCF70DFE68B9B9230A4A94
:107DA00010490B4800F059FC06490F4800F055FCFB
:107DB000B921054800F0ADFE85F31188BFF36F8F40
:107DC00038BD00BF70040021FDBF060123C00601BD
:107DD00071A9060138C0060160030021D9CE060151
:107DE000DBCD060150C0060167C0060138B5044668
:107DF0004FF02003EFF3118583F31288BFF36F8FE9
:107E00001D48FCF7C9FD68B98E231C4A1C491D4852
:107E100000F023FC18491C4800F01FFC8E21174875
:107E200000F077FE1448FCF7D3FD2046FFF78CFEE8
:107E300058B11649134840F23D13154A00F00DFCA5
:107E400040F23D11124800F064FE0B48FCF7B2FD11
:107E500068B9B923094A0F490A4800F0FEFB0649F0
:107E60000D4800F0FAFBB921044800F052FE85F3FA
:107E70001188BFF36F8F38BD70040021FDBF06016C
:107E800023C0060171A9060138C00601D9CE06013A
:107E9000DBCD060150C0060167C0060170B504467F
:107EA0000D464FF02003EFF3118683F31288BFF3E2
:107EB0006F8F1C48FCF770FD68B98E231A4A1B4966
:107EC0001B4800F0CAFB17491A4800F0C6FB8E2178
:107ED000154800F01EFE1348FCF77AFD01216A09DF
:107EE000201D50F8223005F01F0501FA05F523EAA0
:107EF000050540F822500B48FCF75CFD68B9B92332
:107F0000094A0D490A4800F0A8FB06490B4800F051
:107F1000A4FBB921044800F0FCFD86F31188BFF3EF
:107F20006F8F70BD74040021FDBF060123C00601E0
:107F300071A9060138C0060150C0060167C00601DC
:107F400038B5064C064DAC4201D3002038BD6268FE
:107F5000002154F8080B00F014FFF4E7C49F060159
:107F6000C49F060108B50348452100F02EFE049881
:107F700000F049FE06CF0601024608B50348452138
:107F800000F023FE049800F03EFE00BF25CF06015E
:107F900036289ABF024B53F820000248704700BFB2
:107FA0004CA2060149CF060110B5F8F749FB04467B
:107FB00060B910496923104A104800F04EFB104880
:107FC00000F04BFB69210C4800F0A3FDA3790B2BBB
:107FD0000CD00C496A23084A084800F03EFB0A48C6
:107FE00000F03BFB6A21044800F093FDA368586849
:107FF00010BD00BF71CF06014BCF060171A906016C
:1080000084CF06019DCF0601C5CF060130B585B0EE
:108010000D46044601F01DFC0190284601F019FCB4
:10802000019BCDE90204013305D0013003D00348A0
:1080300001A9F8F71FFB05B030BD00BF1B98060172
:1080400008B501F006FC431C014604D0BDE8084019
:108050000148F8F70FBB08BD6598060137B505461E
:1080600015F1090F144618462ED015F1080F06DA3F
:1080700015F1700F47D0163541D003B030BD013532
:10808000FBD1264DA86801F0E4FB0146A079FFF77B
:108090007FFF2368AA68CDE900030B4620484521ED
:1080A00000F093FDEFF305830BB900F0C0FD45210F
:1080B0001C4A1D4800F089FD02220120211D03B049
:1080C000BDE83040F9F766BBFFF762FF0A4603469A
:1080D0004521164800F079FD34B94521144803B014
:1080E000BDE8304000F071BDA079FFF751FF452198
:1080F0000246104803B0BDE8304000F066BD0A46B5
:108100000D484521F6E7FFF743FF0A4603464521A0
:108110000A4803B0BDE8304000F057BD60030021BD
:108120003AD0060170D0060182D00601D8CF0601F0
:10813000F2CF06011CD006018AD00601ADD006019F
:1081400038B51546044668B311B183798B4229D1FD
:10815000E3799A070AD5EDB1013526D1E37913F019
:10816000010F0CBF00206FF06F001AE0104B9868F1
:1081700001F06FFB431C14D04209231D53F8222049
:10818000012300F01F0003FA00F01042E3D14FF08A
:10819000FF3006E0E37913F0010F14BF00206FF009
:1081A000150038BD6FF00800FBE70020F9E700BFBD
:1081B00060030021F7B50D461646074600223146FA
:1081C000284600F071FD044660B1094B4521CDE918
:1081D0000063084A2B46084800F0F7FC0E242046AE
:1081E00003B0F0BD32462946384600F0BFFDF6E741
:1081F0006AD1060197D30601E3A80601F7B50E463A
:10820000144605462146304601AAF9F78DFD019F27
:108210000346CFB9A04206D1324645210B4800F0B3
:10822000D4FC162009E0441C09D2224631462846D7
:10823000FFF7C0FF2B1903F8017C03B0F0BD452107
:10824000034800F0C2FCECE70E20F6E7EDD0060193
:108250000BD10601024A0349034800F0FEB900BFF2
:10826000BEC60601A1D30601BED3060170B50E4CF1
:108270000E4D0F4EAC420CD90E49182332460E4813
:1082800000F0EBF90D4800F0E8F91821304600F055
:1082900040FCAC4201D3002070BD2046D4E901125D
:1082A00001F02DFB1834E5E7E4280021E428002143
:1082B000E5D3060107D4060171A90601FDC4060134
:1082C0002DE9F04F85B0DDE90E9706468A4648460F
:1082D0003946904601F06FFA06F11404CDE9020127
:1082E0004FF02003EFF3118583F31288BFF36F8FF4
:1082F0002046FCF751FB68B98E233C4A3C493D4877
:1083000000F0ABF921463C4800F0A7F98E21374830
:1083100000F0FFFB2046FCF75BFBEFF305837BB12E
:1083200059EA07030CD035494923354A314800F052
:1083300094F9344800F091F94921314800F0E9FB03
:10834000DFF8A890DFF8ACB0424651463046F8F767
:10835000CBFC0746FFF792F9CFB12046FCF72AFB8A
:1083600068B9B923214A2849224800F076F9214604
:10837000264800F072F9B9211C4800F0CAFB85F3C9
:108380001188BFF36F8F384605B0BDE8F08F029BB0
:10839000181A039B63EB0101012871F10003DCDB78
:1083A000CDE9000106F10C0229462046FDF782FFC7
:1083B0004FF02003EFF3118583F31288BFF36F8F23
:1083C0002046FCF7E9FA68B98E234A465846084920
:1083D00000F043F92146084800F03FF98E21484655
:1083E00000F097FB2046FCF7F3FAADE7FDBF06016E
:1083F00023C0060171A9060138C006011DD406017B
:10840000E5D30601BCC6060150C0060167C00601DF
:10841000F8B505460E4600F114044FF02003EFF3C3
:10842000118783F31288BFF36F8F2046FCF7B4FAED
:1084300068B98E231A4A1B491B4800F00EF92146E1
:108440001A4800F00AF98E21154800F062FB204618
:10845000FCF7BEFA28463146F8F7F6FB05F10C00AA
:1084600001F066F928B139462046BDE8F840FDF72D
:1084700061BA2046FCF79EFA68B9B923084A0C494C
:10848000094800F0EAF821460A4800F0E6F8B92168
:10849000034800F03EFB87F31188BFF36F8FF8BDF0
:1084A000FDBF060123C0060171A9060138C00601FF
:1084B00050C0060167C006012DE9F0411A4F089A25
:1084C000BB680646C3F8802008460D46F8F7B8F8A2
:1084D000012209218046FFF733FE0446A8B1424637
:1084E00029460923FFF7BAFD4521104A104800F03C
:1084F0006CFBBB68D3F8800000F085FB3346452158
:108500000A4A0C4800F061FBF3E7304601F0FFF93E
:108510000028F3D0294601F0A7F9BB682046C3F82C
:108520008040BDE8F08100BF60030021B1D40601A6
:108530004AB5060163D4060138B50E4C069AA36805
:108540000546C3F8802001F0E2F950B92B460A48ED
:1085500045210A4A00F039FBA368D3F8800000F0F7
:1085600052FBA16801F094F90020A368C3F88000D1
:1085700038BD00BF6003002163D4060199D4060111
:108580000020024B9B68C3F8800070476003002105
:10859000002307B50A46009301460348FBF738FD60
:1085A00003B05DF804FB00BFD9F4051170B4DDE938
:1085B000035401F50046B6F5803F0DD2FF2B0BD8D2
:1085C000FF2C09D844EA0324134644EA0142014639
:1085D00070BC0348FBF71CBD6FF0800070BC704797
:1085E000E1F40511002307B501461A46009303483C
:1085F000FBF70EFD03B05DF804FB00BFD1F40511DD
:108600007047002070472DE978410446466800F124
:108610000805EFF3058353B900F009FB38B1314683
:108620002846BE2603DF00236360BDE8788131461B
:108630002846F8F7A3FAF6E710B504460B68084693
:1086400001330B604B685A1C202A0B444A601C7291
:1086500001D1FFF7D8FF204610BD0FB407B504A91C
:1086600051F8040B0191F8F797FA03B05DF804EBA9
:1086700004B07047044608B5084611461A46A0479C
:10868000EFF305837BB900F0D2FA60B14FF4AD7619
:1086900003DF0446EFF3058343B900F0C8FA28B1BD
:1086A0002046BF2603DFFEF7C1FAF2E72046F9F7BE
:1086B0004BFEF8E7836800EBC101B3F5004F2CBF18
:1086C00051F8220031F81200704700EBC1018068B8
:1086D000B0F5004F2CBF41F8223021F8123070471E
:1086E000012208B5FFF7E6FFD04008BD836800EB24
:1086F000C101B3F5004F08D34B681AB143F0010331
:108700004B60704723F00103FAE74B881AB143F03E
:1087100001034B80704723F00103FAE75300012265
:10872000FFF7D3BF8368B3F5004F2CBF08230423A2
:10873000C91A081AC0087047B0F5004F2CBF0820AE
:10874000042007310844C008704708B50B460121D2
:10875000FFF7F2FF01331B1AB3FA83F0C0F11F00D9
:1087600008BD2DE9F041174603220E460446FFF7E7
:10877000A1FF8642054607F104080BD1012303FA45
:1087800007F7E36823EA0703E360002344F828308F
:10879000BDE8F081314602222046FFF78BFF0646F6
:1087A0002B4601460322204644F82850FFF78DFF50
:1087B000334629462046BDE8F0410222FFF785BF37
:1087C00070B50D4686680446FFF78AFFB6F5004F80
:1087D000014601D3012809D03046FFF7B6FF2946EC
:1087E00002462046BDE87040FFF7BBBF70BD2DE9D3
:1087F000F047054680688846FFF7A7FF05EB800A2B
:10880000DAF810900646B9F1000F1BD00327DAF80A
:10881000104028462146FFF763FF404507D3324604
:1088200021462846FFF79DFF2046BDE8F08703223A
:1088300021462846FFF73EFF013FCAF8100001D04D
:108840008145E4D14FF0FF34E9680136B4400C4073
:10885000EAD094FAA4F2B2FA82F2131D55F823403A
:10886000DEE72DE9F04114460E460546FFF738FFD6
:10887000A4EB0608371B0744424631462846FFF75B
:108880004DFF3A4621462846FFF748FF434600225F
:1088900021462846FFF719FF21462846FFF720FF0B
:1088A0003B46211800222846BDE8F041FFF70DBFE6
:1088B0002DE9F041164604460F46FFF711FF3146F9
:1088C00005462046FFF70CFF05442A463946204658
:1088D000FFF724FF31462046FFF702FF2B463118F1
:1088E00000222046BDE8F041FFF7EFBE2DE9F04140
:1088F0000D4686680446FFF7F3FEB6F5004F0146C5
:1089000001D3012833D03046FFF71FFF04EB80026C
:1089100016699EB9012303FA00F0E3682946034370
:10892000E360204615612B460222FFF7CEFE0322AC
:1089300029462046BDE8F041FFF7C7BE0222314676
:108940002046FFF7B7FE0746034629462046FFF7B5
:10895000BCFE0322334629462046FFF7B6FE3946C1
:108960002B462046FFF7B1FE02223146E1E7BDE883
:10897000F081F8B50C460546FFF7B2FE2618012235
:1089800031462846FFF796FEC3070CD431462846E9
:10899000FFF716FF21462846FFF7A2FE21462218C0
:1089A0002846FFF785FF002221462846FFF782FE72
:1089B000271A012239462846FFF77CFE10EA0206F4
:1089C00013D139462846FFF7FBFE2146324628469A
:1089D000FFF770FE2246211A2846FFF769FF21465D
:1089E00032462846FFF766FE241A21462846BDE88F
:1089F000F840FFF77BBF70B5066809B9002070BD6D
:108A0000B068B0EBD10FF9D9FFF796FE01460546E5
:108A10003046FFF7ECFE04460028EFD00146304612
:108A2000FFF75EFEA84209D92544214630462A4672
:108A3000FFF717FF29463046FFF758FF214630461B
:108A40000122FFF753FEB368B3F5004F2CBF082394
:108A5000042303EBC4042044D1E72DE9F84F9A46E0
:108A6000D37880466F2B0F461546A3F1410B29D0D2
:108A700024D8582B14BF0A261026DDF82890324639
:108A8000002340463946F7F7BFFE092AD4B21ED864
:108A90003034B045E4B277F1000309F8014D01D359
:108AA000D14511D82B789B0605D5082E15D1AB786A
:108AB00043F00803AB704846BDE8F88F03F0F703B6
:108AC000702BD7E70826D8E780460F46D7E7BBF1DB
:108AD000190F94BF37345734DBE7102EEBD1AB7846
:108AE00043F01003E6E72DE9F041074688461546B6
:108AF0001E461446B442A4EB050002D33EB92378C7
:108B00002BB1414614F8010BB8470028F2DABDE852
:108B1000F08108B5EFF3058343B900F088F828B178
:108B2000404080F311884FF0030002DF404080F3A3
:108B300011884FF0040002DF08BD2DE9F041154611
:108B40001C46F7F77DFDC0B183790E2B15D18668E1
:108B50009EB1EFF305834BB900F069F830B13046B0
:108B6000294622469C2603DFBDE8F0812A4623469B
:108B70003046BDE8F041FBF7F3BF6FF01500F3E7B7
:108B80002DE95041F7F75CFDB0B183790E2B13D17D
:108B900084688CB1E3687BB1EFF305833BB900F0E7
:108BA00046F820B120469D2603DFBDE850812046CF
:108BB000BDE85041FCF7FAB86FF01500F5E77047D3
:108BC00008B5F8F7D5FE002008BD0FB407B504A915
:108BD00051F8040B0191F7F7DFFF03B05DF804EBE8
:108BE00004B0704738B50446056800F020F820B19D
:108BF0002368023B022B28BF032521462846BDE8F7
:108C00003840F8F73BBE044600B589B00021202269
:108C1000684600F0B6F8E368694603200693F8F763
:108C20002DFE00210120F8F729BE70477047EFF3B1
:108C3000148000F00100704740E800F313F4803F17
:108C4000D8B208BF6FF01500704721B140E840F07E
:108C5000C0F38040704740E800F0F9E721B140E8F8
:108C600040F0C0F3C040704740E800F0F9E7002A48
:108C700018BF042208B542F00802F7F761FD00387A
:108C800018BF012008BD002A18BF042208B542F011
:108C90000102F7F755FD003818BF012008BD08B5DF
:108CA000F9F72CFC013808BD00F019B830B54B6855
:108CB0000C6885B00A894D890094013B24F01F049B
:108CC000234402F01F0242EA451223F01F036946C3
:108CD0008DF808200393F9F7CFFB05B030BDF8B548
:108CE000164604460D46012296B1FFF7CCFF68B93F
:108CF0002046FFF7A1FF0746013D6019FFF79CFFE3
:108D000017F1160F07D14FF0FF3000E00020F8BD3B
:108D1000FFF7ADFFEBE78742F5D10121204636B1E1
:108D2000FFF79CFFB0FA80F040094042EFE7FFF701
:108D30008CFFF7E7034600201A5C02B97047013048
:108D4000FAE7034600201A5C0AB1884200D1704756
:108D50000130F8E7431E013913F8012F11F8010F14
:108D6000824201D1002AF7D1101A704710B5431E74
:108D70000A44914200D110BD11F8014B03F8014F94
:108D8000F7E70346C9B20244934200D1704703F8A3
:108D9000011BF9E74FF0FF3070472DE97841044699
:108DA0000D46EFF3058313B9FFF741FF28B92946B4
:108DB0002046BDE87841F9F7BFBD204629464FF46B
:108DC000A17603DFBDE87881FFF7E7BF43680020A5
:108DD0005B681B680B60704743685B68586842407B
:108DE0000A4042405A6000207047436800205A6899
:108DF00053680B4353607047436800205A685368B8
:108E000023EA010353607047436800205A6853689F
:108E10004B4053607047012312F4407F10B503FAB2
:108E200001F1446816D012F0320F13D193050ED51C
:108E3000130507D5FFF7D9FF636819610020636840
:108E4000D96110BD5305F7D5FFF7D6FFF4E7636886
:108E50005961F3E76FF08500F3E7B3F5C02F10B564
:108E6000406819D0B2F5804F16D044680120B2F5A1
:108E7000005F00FA01F102D16162002010BDB2F57D
:108E8000A03F0CBFA162E162B3F5802F0CBF21634C
:108E90006163A1632162F0E76FF08500EEE708B53A
:108EA00043689B689847002008BD08B5452000220C
:108EB0000321F8F721FDBDE808404520F8F70CBD77
:108EC00008B5462000220321F8F716FDBDE808404A
:108ED0004620F8F701BD08B5472000220321F8F726
:108EE0000BFDBDE808404720F8F7F6BC08B5482060
:108EF00000220321F8F700FDBDE808404820F8F7FC
:108F0000EBBC036930B55C68012303FA01F1A36887
:108F1000194223D022F4706323F001030BBB12F437
:108F2000007012D060684FF02003EFF3118583F3D7
:108F30001288BFF36F8F130508D5036819430160CA
:108F400085F31188BFF36F8F002030BD5305F7D52F
:108F5000A368026823EA01011140F0E76FF01500F1
:108F6000F3E76FF08500F0E703695A685368186803
:108F7000936803400B6000207047036910B5586880
:108F8000D0E9013001404FF02000EFF3118480F36D
:108F90001288BFF36F8F186842400A4042401A603F
:108FA00084F31188BFF36F8F002010BD03695B68E5
:108FB000D3E901230B404FF02001EFF3118081F33F
:108FC0001288BFF36F8F11681943116080F3118805
:108FD000BFF36F8F0020704703695B68D3E90123FB
:108FE0000B404FF02001EFF3118081F31288BFF3A3
:108FF0006F8F116821EA0301116080F31188BFF3BC
:109000006F8F0020704703695B68D3E901230B4031
:109010004FF02001EFF3118081F31288BFF36F8FBF
:1090200011685940116080F31188BFF36F8F0020E1
:109030007047B2F5005F14BF6FF0850000207047E5
:109040000369426800205A60704770B500220D46DF
:1090500020210646FFF774F8044620B1202332464B
:109060002946FEF7FBFF204670BD036840681B6879
:109070001847036840685B681847036840689B6846
:10908000184738B50446FAF777FF0546FAF774FF34
:10909000431BA342FAD338BD10B50446FFF7EDFFDA
:1090A000014660B92046FFF7E0FFA068FFF7E9FF3F
:1090B00020460121FFF7D9FFA068FFF7E2FF00215A
:1090C0002046FFF7D6FFE068FFF7DBFF20460021D0
:1090D000FFF7CBFFA068BDE81040FFF7D2BF10B587
:1090E00004460121FFF7C5FF01212046FFF7BDFF20
:1090F000E068FFF7C6FFA068FFF7C3FF2046BDE8A2
:109100001040FFF7C9BF38B504460121FFF7B1FF92
:1091100001212046FFF7A9FFE068FFF7B2FF2046D4
:10912000FFF7ABFF054600212046FFF79EFFA06832
:10913000FFF7A7FF281E18BF012038BD10B5044651
:10914000FFF797FF01212046FFF78FFFE068FFF749
:1091500098FF20460021FFF788FFA068BDE8104077
:10916000FFF78FBF10B504460021FFF782FFA0680C
:10917000FFF787FF01212046FFF777FFE068FFF741
:1091800080FFE068FFF77DFF20460121FFF771FFB8
:10919000A068BDE81040FFF774BF034611F001005E
:1091A00005D1C1F34201012904D0022907D06FF093
:1091B0008500704776229A606522DA607047212226
:1091C0009A601022F9E72DE9F74F0646884699463E
:1091D00014469AB30121FFF748FF06274FEA4909D1
:1091E00008F10C08BD0702D53046FFF7BBFF17F0AA
:1091F000040727D03046FFF74FFF18F8043C1F4301
:10920000790729D54FF0080A4FF0800B07F00105C8
:1092100045EA0905EDB205EA0B013046FFF78EFF7E
:10922000BAF1010A4FEA5B0BF5D13046FFF76BFF4D
:1092300080B16FF004043046FFF794FF204603B07E
:10924000BDE8F08F18F8043C5807D6D53046FFF734
:1092500046FFD2E727F0040717F0010B58E9035344
:1092600005EB030A34D0AA4506D8013C14F0FF04EC
:1092700008F10C08B6D1DEE75846430030460093AB
:10928000FFF741FF009B1843C205F6D505F8010B17
:10929000AAEB0503594230465941FFF74FFFE2E779
:1092A0004FF0080B802315F8012B02EA030130462A
:1092B000CDE90023FFF742FF019BBBF1010B009AB0
:1092C0004FEA5303F1D13046FFF71DFF0028B0D11C
:1092D0005545E5D3C9E76523C0E900127622C0E908
:1092E00002237047012309B1036070474360704750
:1092F000022309B10360704743607047006800F0C3
:10930000020070470069FFF75EBF0069FFF745BFC5
:1093100070B500220D4621210646FEF711FF0446D6
:1093200020B1212332462946FEF798FE204670BD23
:10933000036910B542681C68116824B1536813B101
:10934000B3FBF4F30B6103238B6093689847002011
:1093500010BD43681B685A68920743BF1B68002012
:109360000B704FF0FF30704743681B685A68D20794
:10937000FCD4196070470346104652B15B681B6805
:109380005A68D20704D40120D8600A781A6070475E
:10939000002070470346104652B15B681B6858684E
:1093A00010F0020004D002220120DA601B680B706A
:1093B000704743681B689A6822F004029A60012291
:1093C000DA60704743681B685868C04300F00100CA
:1093D000704743681A68936843F0080393607047C6
:1093E00043681B689A6822F008029A600222DA60D9
:1093F0007047FFF7E7BF43681B68586800F002003A
:109400007047704743681B68D86800F003007047D6
:10941000012070470369C3E901127047026953686C
:109420000BB1916818477047436810B51A68936884
:1094300043F0040393604FF02003EFF3118483F3B0
:109440001288BFF36F8FFFF7E9FF84F31188BFF332
:109450006F8F10BD08B5002203212220F8F74CFAC7
:109460002220F8F739FA212000220321F8F744FAE4
:10947000BDE808402120F8F72FBA08B500220321E3
:109480002420F8F739FA2420F8F726FA23200022BE
:109490000321F8F731FABDE808402320F8F71CBA99
:1094A00008B5002203212620F8F726FA2620F8F72F
:1094B00013FA252000220321F8F71EFABDE8084020
:1094C0002520F8F709BA08B5002203212820F8F76B
:1094D00013FA2820F8F700FA272000220321F8F7D2
:1094E0000BFABDE808402720F8F7F6B908B50022C6
:1094F00003212A20F8F700FA2A20F8F7EDF92920AD
:1095000000220321F8F7F8F9BDE808402920F8F710
:10951000E3B9704770B500220D4630210646FEF7CC
:109520000FFE044620B1302332462946FEF796FD51
:10953000204670BD4FF0E022136923F00103136150
:1095400070470020704700F0F4B938B1C36818883C
:10955000C0F30800A0F580735842584170474FF09F
:109560002002EFF3118382F31288BFF36F8FFEE7BF
:10957000F8B515460E461A4629460746FEF7E0FDA1
:10958000044620B12B463A463146FEF767FD204699
:10959000F8BDEFF30580003818BF012070470020A8
:1095A000704708B5F7F74CF8003818BF012008BD20
:1095B00070B50D4603210646FEF7C2FD044620B1F4
:1095C000032332462946FEF749FD204670BD90F937
:1095D0000E308B4201D0FCF79DBE0020704710B5C5
:1095E0000024C0E90000C0E9024400F076F92046FA
:1095F00010BD70B50D4605210646FEF7A1FD0446D7
:1096000020B1052332462946FEF728FD204670BDCD
:1096100010B5044630B10268930703D0446809B11D
:1096200000F0F4F8204610BD0022C0E9002282605C
:1096300000F10C02C0E9032200F04FB9012307B585
:109640000A4600930021FBF79BFC03B05DF804FB86
:1096500007B50A46002101230091FBF791FC03B0F6
:109660005DF804FB00210068FFF7D2BF00214068CD
:10967000FFF7CEBF70B50D4607210646FEF760FD29
:10968000044620B1072332462946FEF7E7FC204670
:1096900070BD08B54AB18A4207D3C0E90212C0E9D9
:1096A000000000F01AF9002008BD6FF01500FBE77C
:1096B00038B50446F6F7C4FF002209210546FEF737
:1096C0003FFD10F1160F05D028B109232A46214687
:1096D000FEF7C4FC012038BD70B500220D460921FB
:1096E0000646FEF72DFD044620B1092332462946E1
:1096F000FEF7B4FC204670BD034620B9EFF30582A7
:109700000AB9F8F767B983F31188BFF36F8F704711
:109710004FF02003EFF3118083F31288BFF36F8FB4
:10972000FFF7EABF03460068834208BF0020704786
:1097300038B5054600202C68A54200D004B938BDD4
:109740002046FCF7F3F92046FCF78AFB0120F2E7FC
:1097500008B542F20F73C117C01842F210724FF0F1
:10976000000341F10001F7F74FF8C117FDF72AF99F
:1097700042F21073584308BD10B5437B04469B0763
:1097800014D41830FDF784FD0028637B01DA102B18
:109790000CD123F0100320466373FCF761FBEFF359
:1097A00005831BB9BDE81040FFF7B2BF10BD08B577
:1097B000FDF764FF08BDB1F1FF3F08BFB0F1FF3F07
:1097C00038B505460C461DD051EA000303D1BDE86B
:1097D0003840FDF753BF6FF00103181A4FF0FF3305
:1097E00063EB010100290CDAFDF748FF012D224649
:1097F00074F100042B46BCBF01230022181841EB72
:10980000020138BD4FF0FF300146FAE720B1011FD9
:1098100050F8040CFEF7FCBD70470B6830B55A09D0
:10982000041D54F8225003F01F02012303FA02F230
:109830002A420DD000688A68904209D04A685109CE
:1098400054F8210002F01F029340034344F82130F2
:1098500030BD08B5F6F7F4FE08B1806808BD4FF0DA
:10986000FF30FBE7FEF71ABB10B504460846FFF7CA
:10987000F0FF431C0BD001224109231D53F8214066
:1098800000F01F0002FA00F0204343F8210010BD51
:1098900070B504460846FFF7DCFF431C014610D0B4
:1098A00001224509201D50F8253001F01F06B24065
:1098B00023EA020340F825302046BDE87040FEF759
:1098C000EDBA70BD10B50C46F6F7BAFE20B12146D0
:1098D000BDE81040FFF7C8BF10BD08B5F6F7B0FEF1
:1098E00018B1C37943F00103C37108BD08B5F6F799
:1098F000A7FE18B1C37923F00103C37108BD10B4EA
:1099000000F10C04C0E9034410BCF7F779BA38B58C
:109910000546F6F795FE012200210446FEF710FCED
:1099200028B1224600232946FEF798FB0024204652
:1099300038BD37B501214020FEF72AFE051E02DCA6
:10994000012003B030BD00231A461946CDE900338B
:10995000FEF72CFE04462846FEF744FE002CEFDB03
:049960002046EEE7C8
:08996400D86EFF7F0100000036
:10996C006D82060100000000C18B060100000000A2
:10997C009F8E06012C9A06019F8E0601449A0601C1
:10998C009F8E06015C9A06019F8E0601749A060151
:10999C00B57C060100000000417F060100000000BC
:1099AC00419006018C9A060141900601A49A060189
:1099BC0041900601BC9A060131930601D49A060126
:1099CC0031930601EC9A060131930601049B0601C2
:1099DC00319306011C9B060131930601349B060151
:1099EC00652A060100000000093D06010000000088
:1099FC00693206014C9B060169320601649B060123
:109A0C00693206017C9B060169320601949B0601B2
:109A1C0069320601AC9B060143950601000000006B
:109A2C002EB5060130A10601A0A00601AC2800212C
:109A3C00F00200213CA0060135B506010CA106017F
:109A4C00A0A00601B0280021E402002136A00601E6
:109A5C003CB50601E8A00601A0A00601B42800212F
:109A6C00D802002130A0060143B50601C4A00601AE
:109A7C00A0A00601B8280021CC0200212AA00601D2
:109A8C0038AB060160A0060154A10601A0280021F4
:109A9C00E001002124A0060142AB060148A006010A
:109AAC0054A10601A4280021D00100211EA006010A
:109ABC004EAB060154A0060154A10601A8280021B2
:109ACC00D801002118A00601D1BD0601C8A10601CC
:109ADC00D4A10601D02800217428002112A006016F
:109AEC00D8BD0601BCA10601D4A10601D4280021D1
:109AFC00502800210CA00601DFBD0601B0A1060113
:109B0C00D4A10601D82800212C28002106A006018A
:109B1C00E6BD0601A4A10601D4A10601DC280021A2
:109B2C000828002100A00601EDBD060198A1060140
:109B3C00D4A10601E0280021E4270021FA9F0601A8
:109B4C009BBC060188A10601CC270021BC28002162
:109B5C003C030021F49F0601A7BC060184A1060169
:109B6C00CC270021C02800212C030021EE9F0601E8
:109B7C00B3BC060180A10601CC270021C42800211A
:109B8C001C030021E89F0601BFBC06017CA1060155
:109B9C00CC270021C82800210C030021E29F0601DC
:109BAC00CEBC060178A10601CC270021CC280021CF
:089BBC00FC020021DC9F060100
:109BC40000000000238C060100000000238C060125
:109BD40000000000238C060100000000238C060115
:109BE40000000000238C060100000000238C060105
:109BF40000000000238C060100000000238C0601F5
:109C040000000000238C060100000000238C0601E4
:109C140000000000238C060100000000238C0601D4
:109C240000000000238C060100000000238C0601C4
:109C340000000000238C060100000000238C0601B4
:109C440000000000238C060100000000238C0601A4
:109C540000000000238C060100000000238C060194
:109C640000000000238C060100000000238C060184
:109C740000000000238C060100000000238C060174
:109C840000000000238C060100000000238C060164
:109C940000000000238C060100000000238C060154
:109CA40000000000238C060100000000238C060144
:109CB40000000000238C060100000000238C060134
:109CC40000000000238C0601349B06011D9406014C
:109CD400349B06011D9406011C9B06011D9406017C
:109CE4001C9B06011D940601049B06011D9406019C
:109CF400049B06011D940601EC9A06011D940601BD
:109D0400EC9A06011D940601D49A06011D940601DD
:109D1400D49A06011D94060100000000238C06015C
:109D240000000000238C060100000000238C0601C3
:109D340000000000238C060100000000238C0601B3
:109D440000000000238C060100000000238C0601A3
:109D540000000000238C060100000000238C060193
:109D640000000000238C060100000000238C060183
:109D740000000000238C060100000000238C060173
:109D840000000000238C060100000000238C060163
:109D940000000000238C060100000000238C060153
:109DA40000000000238C060100000000238C060143
:109DB40000000000238C060100000000238C060133
:109DC40000000000238C060100000000238C060123
:109DD40000000000238C060100000000238C060113
:109DE40000000000238C0601749A0601692B060109
:109DF4005C9A0601692B0601449A0601692B060147
:109E04002C9A0601692B060100000000238C060130
:109E140000000000238C060100000000238C0601D2
:109E240000000000238C060100000000238C0601C2
:109E340000000000238C060100000000238C0601B2
:109E440000000000238C060100000000238C0601A2
:109E540000000000238C060100000000238C060192
:109E640000000000238C060100000000238C060182
:109E740000000000238C060100000000238C060172
:109E840000000000238C060100000000238C060162
:109E940000000000238C060100000000238C060152
:109EA40000000000238C060100000000238C060142
:109EB40000000000238C060100000000238C060132
:109EC40000000000238C060100000000238C060122
:109ED40000000000238C060100000000238C060112
:109EE40000000000238C060100000000238C060102
:109EF40000000000238C060100000000238C0601F2
:109F040000000000238C060100000000238C0601E1
:109F140000000000238C060100000000238C0601D1
:109F240000000000238C060100000000238C0601C1
:109F340000000000238C060100000000238C0601B1
:109F440000000000238C060100000000238C0601A1
:109F540000000000238C060100000000238C060191
:109F640000000000238C060100000000238C060181
:109F740000000000238C060100000000238C060171
:109F840000000000238C060100000000238C060161
:109F940000000000238C060100000000238C060151
:109FA40000000000238C060100000000238C060141
:109FB40000000000238C060100000000238C060131
:109FC40097BC06010300000095B2060103000000DF
:089FD400F0C1060103000000CA
:109FDC0000800080FF7F00800080FF7F0080008079
:109FEC00FF7F00800080FF7F00800080FF7F00806B
:109FFC000080FF7F00800080FF7F00800080FF7F5B
:10A00C0000800080FF7F00800080FF7F0080008048
:10A01C00FF7F00800080FF7F00800080FF7F00803A
:10A02C000080FF7F00800080FF7F00800080FF7F2A
:06A03C0000800080FF7FA0
:02A04200FFFF1E
:10A044000300010003000000082030490300000061
:10A05400FF00000000203049FF000000070000005E
:10A064004C203049070000000000002100000000DF
:10A07400060001000200000080A0060100000601A5
:10A08400A5B4060106000000E0FF0B01000000215A
:10A09400ADB4060121000000E0FF1F21178E060168
:10A0A400CD8D0601D98D0601EB8D0601F98D0601D2
:10A0B400098E06015B8E0601BD2A06010000000020
:10A0C400FFFFFFFF00001041AB8E060100000000FF
:10A0D40000001041000100000000104100020000D7
:10A0E40000001041FFFFFFFF00101041C18E060168
:10A0F4000000000000101041000100000010104199
:10A104000002000000101041FFFFFFFF002010417B
:10A11400D78E06010000000000201041000100005D
:10A12400002010410002000000201041FFFFFFFF4B
:10A1340000301041ED8E0601000000000030104197
:10A144000001000000301041000200000030104106
:10A15400038F0601698F06017B8F0601AD8F06010F
:10A16400D98F060107900601339006010000000014
:10A174000000000000002049001020490030204960
:10A184000040204900802049E5920601F192060131
:10A19400FD9206010030304940787D015594060156
:10A1A4000040304940787D017B94060100503049DD
:10A1B40040787D01A19406010060304940787D011A
:10A1C400C79406010070304940787D01ED94060182
:10A1D400539306016993060100000000000000008B
:10A1E4000000000077930601959306012994060167
:10A1F400B3930601C5930601D3930601E1930601C7
:10A20400F3930601F79306010394060113950601DF
:10A214000594060111940601159406016C99060132
:10A22400F4990601249A06012C9A06012C9A060137
:10A23400F5FFFFFFA1C10601AFC10601C3C10601BD
:10A24400D2C10601DEC1060119D1060121D10601E0
:10A254002CD1060133D106013BD1060142D10601BE
:10A264004AD1060158D106015ED1060166D1060124
:10A274006FD1060177D106018ED1060199D106016D
:10A28400A0D10601AAD10601B2D10601BCD10601B2
:10A29400CAD10601D5D10601A7D20601E2D1060131
:10A2A4001BD20601F1D10601FCD106011AD2060126
:10A2B40026D2060134D2060143D206014FD206014A
:10A2C4005FD206016CD2060178D2060184D206015F
:10A2D4008FD206019AD20601A5D20601B2D2060196
:10A2E400BDD20601C9D20601D5D20601E3D20601C8
:10A2F400EED20601FFD206010AD306011BD30601E2
:10A3040044D2060129D3060137D3060143D30601FB
:10A314004ED306015ED3060169D306017AD3060142
:10A3240089D30601657F0601657F0601657F060105
:10A33400657F0601657F0601657F0601657F06016D
:10A34400657F0601657F0601657F0601657F06015D
:10A35400657F0601657F0601657F0601657F06014D
:10A36400657F0601657F0601657F0601657F06013D
:10A37400657F0601657F0601657F0601657F06012D
:10A38400657F0601657F0601657F0601657F06011D
:10A39400657F0601657F0601657F0601657F06010D
:10A3A400657F0601657F0601657F0601657F0601FD
:10A3B400657F0601657F0601657F0601657F0601ED
:10A3C400657F0601657F0601657F0601657F0601DD
:10A3D400657F0601657F0601657F0601657F0601CD
:10A3E4004141060175410601657F0601657F06014D
:10A3F400657F0601657F0601657F0601657F0601AD
:10A40400657F0601657F0601657F0601657F06019C
:10A41400657F0601657F0601657F0601657F06018C
:10A42400657F0601657F0601657F0601657F06017C
:10A43400657F0601657F0601657F0601657F06016C
:10A44400657F0601657F0601657F0601657F06015C
:10A45400657F0601657F0601657F0601657F06014C
:10A46400657F0601657F0601657F0601657F06013C
:10A47400657F0601657F0601657F0601657F06012C
:10A48400657F0601657F0601657F0601657F06011C
:10A49400657F0601657F0601FD310601D92B0601A2
:10A4A40041300601612F0601D92D0601F12E060166
:10A4B400752E0601D12F0601657F0601657F060111
:10A4C400657F0601657F060181320601F1320601CE
:10A4D40049350601BD3406010935060199330601E3
:10A4E400657F0601657F0601657F0601657F0601BC
:10A4F400657F0601657F0601657F0601657F0601AC
:10A50400657F0601657F0601657F0601657F06019B
:10A51400657F0601657F0601657F0601657F06018B
:10A52400AD770601657F0601657F0601657F06013B
:10A53400657F0601657F0601657F0601657F06016B
:10A54400657F0601657F0601E1490601657F060115
:10A55400D5790601D9780601696C0601657F060183
:10A56400657F0601657F0601657F0601657F06013B
:10A57400657F0601657F0601657F0601657F06012B
:10A58400657F0601657F0601657F0601657F06011B
:10A59400154B0601554D0601354F0601B9840601D8
:10A5A4008185060139850601657F0601657F0601FF
:10A5B400657F0601657F0601657F0601657F0601EB
:10A5C400657F0601657F0601657F0601657F0601DB
:10A5D400657F0601657F0601C55106011552060116
:10A5E4007551060141530601B15006019953060104
:10A5F400E553060131540601E95706016555060184
:10A60400C55406019957060141570601A16B06017D
:10A61400657F0601657F0601657F0601ED0B060176
:10A62400856F0601C5470601657F0601657F060142
:10A63400657F0601516F06016D4406015944060108
:10A6440035670601F967060141600601657F060169
:10A6540081440601396506017D4A06012D4A060139
:10A66400657F0601657F0601657F0601657F06013A
:10A67400657F0601657F0601657F0601657F06012A
:10A684001D770601C16B0601E16B0601196B06011A
:10A69400657F0601657F0601657F0601657F06010A
:10A6A400657F0601657F0601657F0601657F0601FA
:10A6B400657F0601657F0601657F0601657F0601EA
:10A6C400657F0601657F0601657F0601657F0601DA
:10A6D400657F0601657F0601657F0601657F0601CA
:10A6E400657F0601657F0601657F0601657F0601BA
:10A6F400657F0601657F0601657F0601657F0601AA
:10A70400657F0601657F0601657F0601657F060199
:10A71400657F0601657F0601657F0601657F060189
:10A72400657F0601657F0601657F0601657F060179
:10A73400657F0601657F0601657F0601657F060169
:10A74400657F0601657F0601657F0601657F060159
:10A75400657F0601657F0601657F0601657F060149
:10A76400657F0601657F0601657F0601657F060139
:10A77400657F0601657F0601657F0601657F060129
:10A78400657F0601657F0601657F0601657F060119
:10A79400657F0601657F0601657F0601657F060109
:10A7A400657F0601657F0601657F0601657F0601F9
:10A7B400657F0601657F0601C53806011D3806015F
:10A7C400657F0601A1350601893B06011D3B060193
:10A7D400F53B0601B13A0601453A0601D9390601AD
:10A7E4006D390601613C0601657F0601657F06013E
:10A7F400657F06010D360601B536060149370601A7
:10A80400B9370601657F0601657F0601657F06018C
:10A81400657F0601657F0601657F0601657F060188
:10A82400657F0601657F0601657F060151290601E2
:10A83400B9290601657F0601657F0601657F06016A
:10A84400657F0601657F0601657F0601657F060158
:10A85400657F0601657F0601657F0601657F060148
:10A86400657F0601657F0601657F0601657F060138
:10A87400657F0601657F0601657F0601657F060128
:10A88400657F0601657F0601657F0601396C060157
:10A89400CD410601657F0601657F0601657F0601DE
:10A8A400657F0601FD16060135170601657F060161
:10A8B400797F06016D7073335F616E3534370048FC
:10A8C400656C6C6F20576F726C642066726F6D20BC
:10A8D400557365725370616365212025730A0025E1
:10A8E400633A2073797363616C6C2025732066610D
:10A8F400696C656420636865636B3A204D656D6FB0
:10A90400727920726567696F6E20257020287369DB
:10A914007A6520257A752920257320616363657320
:10A92400732064656E6965640A007A5F767266797D
:10A934005F6B5F7374725F6F757400574553545F38
:10A94400544F504449522F7A65706879722F6C695C
:10A95400622F6F732F686561702E63006368756E74
:10A964006B5F7573656428682C2063290041535319
:10A97400455254494F4E204641494C205B25735D56
:10A9840020402025733A25640A0009756E657870A5
:10A9940065637465642068656170207374617465AF
:10A9A4002028646F75626C652D667265653F292089
:10A9B400666F72206D656D6F7279206174202570E9
:10A9C4000A006C6566745F6368756E6B28682C207A
:10A9D40072696768745F6368756E6B28682C20639E
:10A9E4002929203D3D20630009636F7272757074DC
:10A9F4006564206865617020626F756E64732028D9
:10AA0400627566666572206F766572666C6F773FF5
:10AA14002920666F72206D656D6F727920617420D4
:10AA240025700A0028616C69676E20262028616CF5
:10AA340069676E202D20312929203D3D20300009F1
:10AA4400616C69676E206D75737420626520612086
:10AA5400706F776572206F6620320A0062797465C0
:10AA640073203E20686561705F666F6F7465725F06
:10AA7400627974657328627974657329000968655D
:10AA840061702073697A6520697320746F6F207315
:10AA94006D616C6C0A00686561705F737A203E209A
:10AAA4006368756E6B737A2873697A656F66287349
:10AAB4007472756374207A5F686561702929006314
:10AAC40068756E6B305F73697A65202B206D696ED3
:10AAD4005F6368756E6B5F73697A65286829203CCB
:10AAE4003D20686561705F737A00286E696C290087
:10AAF400777269746500636865636B5F7379735F0C
:10AB04006D757465785F61646472004661696C6533
:10AB14006420746F207265626F6F743A2073706979
:10AB24006E6E696E6720656E646C6573736C792EE6
:10AB34002E2E0A00465047415F4D4953430046506C
:10AB440047415F425554544F4E00465047415F4C75
:10AB54004544300025633A20002530327820002017
:10AB64002020007C002563004557494425633A2092
:10AB740072302F61313A2020307825303878202007
:10AB840072312F61323A20203078253038782020F5
:10AB940072322F61333A20203078253038780A0019
:10ABA40025633A2072332F61343A202030782530DF
:10ABB4003878207231322F69703A2020307825306D
:10ABC4003878207231342F6C723A20203078253056
:10ABD40038780A0025633A2020787073723A20206E
:10ABE4003078253038780A0025633A204661756C40
:10ABF40074696E6720696E737472756374696F6EBD
:10AC0400206164647265737320287231352F706318
:10AC1400293A203078253038780A00574553545F54
:10AC2400544F504449522F7A65706879722F61727B
:10AC340063682F61726D2F636F72652F6161726338
:10AC44006833322F6972715F6D616E6167652E635F
:10AC5400007072696F203C3D20282831554C203CFF
:10AC64003C2028332929202D2031290009696E76BA
:10AC7400616C6964207072696F72697479202564EB
:10AC840020666F7220256420697271212076616CC0
:10AC9400756573206D757374206265206C657373BC
:10ACA400207468616E20256C750A0A004E4D492097
:10ACB400726563656976656421205265626F6F749D
:10ACC400696E672E2E2E0A0025633A202A2A2A2A24
:10ACD4002A205553414745204641554C54202A2AA1
:10ACE4002A2A2A0A0025633A2020204469766973B7
:10ACF400696F6E206279207A65726F0A0025633A63
:10AD0400202020556E616C69676E6564206D656DE9
:10AD14006F7279206163636573730A0025633A2057
:10AD24002020537461636B206F766572666C6F7755
:10AD34002028636F6E746578742061726561206E7B
:10AD44006F742076616C6964290A0025633A2020B7
:10AD5400204E6F20636F70726F636573736F722020
:10AD6400696E737472756374696F6E730A00256318
:10AD74003A202020496C6C6567616C206C6F6164BB
:10AD8400206F66204558435F52455455524E206902
:10AD94006E746F2050430A0025633A202020496CCA
:10ADA4006C6567616C20757365206F6620746865D7
:10ADB40020455053520A0025633A202020417474E0
:10ADC400656D707420746F20657865637574652093
:10ADD400756E646566696E656420696E73747275F8
:10ADE4006374696F6E0A0025633A202A2A2A2A2A84
:10ADF400204D5055204641554C54202A2A2A2A2AAF
:10AE04000A0025633A202020537461636B696E67DE
:10AE1400206572726F722028636F6E746578742077
:10AE240061726561206D69676874206265206E6F68
:10AE3400742076616C6964290A0025633A20202015
:10AE4400556E737461636B696E67206572726F729D
:10AE54000A0025633A202020446174612041636321
:10AE64006573732056696F6C6174696F6E0A00258F
:10AE7400633A2020204D4D4641522041646472655E
:10AE840073733A20307825780A0025633A2020200D
:10AE9400496E737472756374696F6E204163636580
:10AEA40073732056696F6C6174696F6E0A00256351
:10AEB4003A202020466C6F6174696E672D706F694B
:10AEC4006E74206C617A7920737461746520707279
:10AED40065736572766174696F6E206572726F72E4
:10AEE4000A00574553545F544F504449522F7A65D2
:10AEF400706879722F617263682F61726D2F636F4E
:10AF040072652F616172636833322F636F72746587
:10AF1400785F6D2F6661756C742E63002128282874
:10AF24005343425F54797065202A292028283078B9
:10AF34004530303045303030554C29202B20307886
:10AF440030443030554C2920292D3E43465352205D
:10AF540026202831554C203C3C20283055202B20DD
:10AF640034552929290009537461636B696E67207C
:10AF74006572726F72206E6F7420612073746163E6
:10AF84006B206661696C0A0A0025633A202A2A2A22
:10AF94002A2A20425553204641554C54202A2A2A15
:10AFA4002A2A0A0025633A202020537461636B69BE
:10AFB4006E67206572726F720A0025633A20202042
:10AFC400507265636973652064617461206275738E
:10AFD400206572726F720A0025633A20202042466F
:10AFE400415220416464726573733A203078257845
:10AFF4000A0025633A202020496D707265636973E5
:10B0040065206461746120627573206572726F7269
:10B014000A0025633A202020496E737472756374A4
:10B02400696F6E20627573206572726F720A0052C6
:10B034006573657276656420457863657074696FBD
:10B044006E20280053707572696F757320696E7471
:10B054006572727570742028495251200025633A34
:10B0640020457863657074696F6E206F63637572D1
:10B0740072656420696E205365637572652053742C
:10B084006174650A0065736620213D202828766F67
:10B094006964202A293029000945534620636F75C5
:10B0A4006C64206E6F7420626520726574726965C9
:10B0B400766564207375636365737366756C6C7908
:10B0C4002E205368616C6C206E65766572206F6308
:10B0D4006375722E0A0025633A202A2A2A2A2A2016
:10B0E40048415244204641554C54202A2A2A2A2AAF
:10B0F4000A0025633A202020427573206661756C2E
:10B1040074206F6E20766563746F72207461626C54
:10B114006520726561640A0025633A202020446535
:10B12400627567206576656E740A0025633A20208F
:10B13400204661756C7420657363616C6174696F1A
:10B144006E20287365652062656C6F77290A002577
:10B15400633A20415243485F455843455054207751
:10B1640069746820726561736F6E2025780A0A001D
:10B17400094661756C7420657363616C6174696FF1
:10B184006E20776974686F75742046535220696E17
:10B19400666F0A0009486172644661756C742077B1
:10B1A4006974686F7574204846535220696E666FDF
:10B1B400205368616C6C206E65766572206F6363E2
:10B1C40075720A0025633A202A2A2A2A2A2044650D
:10B1D400627567206D6F6E69746F72206578636540
:10B1E4007074696F6E202A2A2A2A2A0A0025633A73
:10B1F400202A2A2A2A2A20257320256429202A2A5B
:10B204002A2A2A0A00574553545F544F504449523E
:10B214002F7A65706879722F617263682F61726D1D
:10B224002F636F72652F616172636833322F6D70A3
:10B23400752F61726D5F636F72655F6D70752E63DC
:10B2440000726567696F6E5F6E756D203C203136E4
:10B25400202B2031202B202830203F2031203A2061
:10B26400302900094F75742D6F662D626F756E64F9
:10B2740073206572726F7220666F722064796E61DA
:10B284006D696320726567696F6E206D61702E0A47
:10B29400006D70750025633A204661696C65642011
:10B2A400746F20616C6C6F63617465206E657720C8
:10B2B4004D505520726567696F6E2025750A0A0026
:10B2C400574553545F544F504449522F7A65706820
:10B2D40079722F617263682F61726D2F636F72656B
:10B2E4002F616172636833322F6D70752F61726DD7
:10B2F4005F6D70752E63007265675F696E64657853
:10B3040020213D206765745F6E756D5F72656769A6
:10B314006F6E73282900094D656D6F727920646F13
:10B324006D61696E20706172746974696F6E202535
:10B33400702073697A6520257A75206E6F74206693
:10B344006F756E640A0A0025633A2050617274694D
:10B3540074696F6E2025753A2073616E6974792063
:10B36400636865636B206661696C65642E0A0025F9
:10B37400633A20496E76616C696420756E64657207
:10B384006C79696E6720726567696F6E20696E6497
:10B3940065782025750A0009436F6E6669677572C2
:10B3A400696E6720257520737461746963204D503C
:10B3B4005520726567696F6E73206661696C656498
:10B3C4000A0A00094D61726B696E67202575206158
:10B3D4007265617320666F722064796E616D696352
:10B3E40020726567696F6E73206661696C65640AB3
:10B3F4000A0009436F6E6669677572696E67202576
:10B40400752064796E616D6963204D5055207265B5
:10B4140067696F6E73206661696C65640A0A000966
:10B424005265717565737420746F20636F6E6669FD
:10B43400677572653A20257520726567696F6E734A
:10B444002028737570706F727465643A20257529AD
:10B454000A0A0025633A2073797363616C6C2025B2
:10B4640073206661696C656420636865636B3A2068
:10B47400257A7578257A75206172726179206973ED
:10B4840020746F6F206C617267650A007A5F767250
:10B4940066795F7A65706879725F667772697465D8
:10B4A40000464C4153485F30005352414D5F3000D9
:10B4B400574553545F544F504449522F7A6570682E
:10B4C40079722F647269766572732F6770696F2F52
:10B4D4006770696F5F7574696C732E680063616C63
:10B4E4006C6261636B00094E6F2063616C6C626116
:10B4F400636B210A0063616C6C6261636B2D3E684F
:10B50400616E646C657200094E6F2063616C6C62DD
:10B5140061636B2068616E646C6572210A0063620A
:10B524002D3E68616E646C6572004750494F5F330D
:10B53400004750494F5F32004750494F5F31004741
:10B5440050494F5F300025633A2073797363616C0F
:10B554006C202573206661696C656420636865638B
:10B564006B3A206163636573732064656E69656417
:10B574000A0070696E5F636F6E6669677572650055
:10B5840025633A2073797363616C6C20257320669C
:10B5940061696C656420636865636B3A204F70650C
:10B5A400726174696F6E202573206E6F74206465F8
:10B5B40066696E656420666F72206472697665726E
:10B5C40020696E7374616E63652025700A005745A7
:10B5D40053545F544F504449522F7A6570687972BE
:10B5E4002F696E636C7564652F6472697665727316
:10B5F4002F6770696F2E680028666C616773202658
:10B604002028283155203C3C20313329207C202817
:10B614003155203C3C20313429207C2028315520D0
:10B624003C3C20313529207C20283155203C3C20CD
:10B63400313629207C20283155203C3C20313729C3
:10B64400207C20283155203C3C20313829292920D0
:10B654003D3D20300009496E746572727570742026
:10B66400666C61677320617265206E6F74207375F8
:10B6740070706F727465640A0028666C6167732069
:10B684002620282831203C3C203429207C202831C5
:10B69400203C3C203529292920213D2028283120FF
:10B6A4003C3C203429207C202831203C3C20352976
:10B6B40029000950756C6C20557020616E6420500F
:10B6C400756C6C20446F776E2073686F756C6420A2
:10B6D4006E6F7420626520656E61626C65642073B0
:10B6E400696D756C74616E656F75736C790A002889
:10B6F400666C616773202620283155203C3C203934
:10B70400292920213D2030207C7C2028666C61671B
:10B71400732026202831203C3C20312929203D3D1E
:10B72400203000094F7574707574206E65656473FC
:10B7340020746F20626520656E61626C65642066AA
:10B744006F7220274F70656E20447261696E272CDA
:10B7540020274F70656E20536F7572636527206DC7
:10B764006F646520746F20626520737570706F72EA
:10B774007465640A0028666C61677320262028318A
:10B78400203C3C2031292920213D2030207C7C2074
:10B7940028666C6167732026202831203C3C2032C7
:10B7A4002929203D3D20300028666C6167732026DE
:10B7B4002028283155203C3C20313029207C202869
:10B7C4003155203C3C203131292929203D3D203070
:10B7D400207C7C2028666C616773202620283155E4
:10B7E400203C3C2039292920213D203000094F7577
:10B7F40074707574206E6565647320746F2062655F
:10B8040020656E61626C656420746F2062652069D6
:10B814006E697469616C697A6564206C6F77206FF6
:10B824007220686967680A0028666C61677320265D
:10B834002028283155203C3C20313029207C2028E8
:10B844003155203C3C20313129292920213D202813
:10B85400283155203C3C20313029207C202831558A
:10B86400203C3C203131292900094F7574707574CE
:10B874002063616E6E6F7420626520696E697469FD
:10B88400616C697A6564206C6F7720616E642068EE
:10B894006967680A00286366672D3E706F72745F7B
:10B8A40070696E5F6D61736B202620286770696F05
:10B8B4005F706F72745F70696E735F74292831559D
:10B8C4004C203C3C202870696E29292920213D20E8
:10B8D40030550009556E737570706F72746564200D
:10B8E40070696E0A00706F72745F6765745F72616D
:10B8F4007700706F72745F7365745F6D61736B65ED
:10B90400645F72617700706F72745F7365745F62F5
:10B914006974735F72617700706F72745F636C65D2
:10B9240061725F626974735F72617700706F7274C1
:10B934005F746F67676C655F626974730070696ECA
:10B944005F696E746572727570745F636F6E666939
:10B95400677572650028666C61677320262028313C
:10B9640055203C3C2031392929203D3D20300028F8
:10B97400666C61677320262028283155203C3C20C2
:10B98400313329207C20283155203C3C2031342976
:10B99400292920213D2028283155203C3C203133C1
:10B9A40029207C20283155203C3C20313429290091
:10B9B4000943616E6E6F7420626F746820656E61F6
:10B9C400626C6520616E642064697361626C6520D9
:10B9D400696E74657272757074730A0028666C619E
:10B9E400677320262028283155203C3C20313329F8
:10B9F400207C20283155203C3C2031342929292021
:10BA0400213D20305500094D7573742065697468B3
:10BA1400657220656E61626C65206F722064697363
:10BA240061626C6520696E74657272757074730AF4
:10BA3400002828666C616773202620283155203C35
:10BA44003C2031342929203D3D203029207C7C2094
:10BA54002828666C616773202620283155203C3CD9
:10BA6400203136292920213D203029207C7C2028A2
:10BA740028666C61677320262028283155203C3CB9
:10BA840020313729207C20283155203C3C20313876
:10BA940029292920213D2028283155203C3C2031CA
:10BAA4003729207C20283155203C3C203138292955
:10BAB4002900094F6E6C79206F6E65206F662047F0
:10BAC40050494F5F494E545F4C4F575F302C2047CD
:10BAD40050494F5F494E545F484947485F3120639E
:10BAE400616E20626520656E61626C656420666FBC
:10BAF400722061206C6576656C20696E7465727263
:10BB04007570742E0A002828666C616773202620DD
:10BB1400283155203C3C2031342929203D3D20301A
:10BB240029207C7C202828666C61677320262028C5
:10BB3400283155203C3C20313729207C20283155A0
:10BB4400203C3C20313829292920213D203029005E
:10BB5400094174206C65617374206F6E65206F6693
:10BB6400204750494F5F494E545F4C4F575F302C2C
:10BB7400204750494F5F494E545F484947485F3119
:10BB84002068617320746F20626520656E61626C49
:10BB940065642E0A006765745F70656E64696E671C
:10BBA4005F696E74007A5F767266795F6770696F39
:10BBB4005F6765745F70656E64696E675F696E74F4
:10BBC400007A5F767266795F6770696F5F70696E1D
:10BBD4005F696E746572727570745F636F6E6669A7
:10BBE40067757265007A5F767266795F6770696FF0
:10BBF4005F706F72745F746F67676C655F6269749E
:10BC040073007A5F767266795F6770696F5F706FD1
:10BC140072745F636C6561725F626974735F726191
:10BC240077007A5F767266795F6770696F5F706FAD
:10BC340072745F7365745F626974735F72617700B5
:10BC44007A5F767266795F6770696F5F706F72741E
:10BC54005F7365745F6D61736B65645F72617700B8
:10BC64007A5F767266795F6770696F5F706F7274FE
:10BC74005F6765745F726177007A5F767266795F79
:10BC84006770696F5F70696E5F636F6E6669677511
:10BC940072650069326300444452345F4545505232
:10BCA4004F4D004932435F534849454C44310049A4
:10BCB40032435F534849454C4430004932435F4165
:10BCC4005544494F5F434F4E46004932435F544FFA
:10BCD400554348006765745F636F6E666967002546
:10BCE400633A2073797363616C6C202573206661F9
:10BCF400696C656420636865636B3A206E756D5F7B
:10BD04006D736773203E3D2031202626206E756DAD
:10BD14005F6D736773203C2033320A007A5F76725A
:10BD240066795F6932635F7265636F7665725F62BD
:10BD34007573007A5F767266795F6932635F736CDC
:10BD44006176655F6472697665725F756E72656748
:10BD54006973746572007A5F767266795F693263BB
:10BD64005F736C6176655F6472697665725F726534
:10BD740067697374657200636F70795F6D7367735D
:10BD84005F616E645F7472616E73666572007A5F80
:10BD9400767266795F6932635F7472616E73666529
:10BDA40072007A5F767266795F6932635F67657481
:10BDB4005F636F6E666967007A5F767266795F6942
:10BDC40032635F636F6E66696775726500554152D1
:10BDD400545F3400554152545F3300554152545F0F
:10BDE4003200554152545F3100554152545F300086
:10BDF4006572725F636865636B00706F6C6C5F691A
:10BE04006E00706F6C6C5F6F757400636F6E666943
:10BE1400675F676574006972715F74785F656E61EE
:10BE2400626C65006972715F74785F6469736162E2
:10BE34006C65006972715F72785F656E61626C65D2
:10BE4400006972715F72785F64697361626C650026
:10BE54006972715F6572725F656E61626C650069BB
:10BE640072715F6572725F64697361626C650069A7
:10BE740072715F69735F70656E64696E6700697281
:10BE8400715F757064617465007A5F767266795F5C
:10BE9400756172745F6972715F7570646174650055
:10BEA4007A5F767266795F756172745F6972715FC9
:10BEB40069735F70656E64696E67007A5F76726637
:10BEC400795F756172745F706F6C6C5F6F75745FAE
:10BED400753136007A5F767266795F756172745F68
:10BEE400706F6C6C5F6F7574007A5F767266795FE1
:10BEF400756172745F706F6C6C5F696E5F753136FB
:10BF0400007A5F767266795F756172745F706F6CC8
:10BF14006C5F696E007A5F767266795F75617274C0
:10BF24005F6572725F636865636B007A5F767266E1
:10BF3400795F756172745F6972715F6572725F6453
:10BF4400697361626C65007A5F767266795F7561A8
:10BF540072745F6972715F6572725F656E61626C43
:10BF640065007A5F767266795F756172745F697273
:10BF7400715F72785F64697361626C65007A5F7681
:10BF84007266795F756172745F6972715F72785FEE
:10BF9400656E61626C65007A5F767266795F756161
:10BFA40072745F6972715F74785F64697361626CE3
:10BFB40065007A5F767266795F756172745F697223
:10BFC400715F74785F656E61626C65007A5F76722A
:10BFD40066795F756172745F636F6E6669677572A7
:10BFE40065007A5F767266795F756172745F636FFC
:10BFF4006E6669675F67657400574553545F544FB5
:10C00400504449522F7A65706879722F696E636C57
:10C014007564652F7370696E6C6F636B2E68007A3C
:10C024005F7370696E5F6C6F636B5F76616C69647C
:10C03400286C2900095265637572736976652073EB
:10C0440070696E6C6F636B2025700A007A5F737081
:10C05400696E5F756E6C6F636B5F76616C69642883
:10C064006C2900094E6F74206D79207370696E6CB1
:10C074006F636B2025700A007A5F767266795F645D
:10C0840065766963655F69735F72656164790025CC
:10C09400633A2048616C74696E67207379737465C0
:10C0A4006D0A00556E6B6E6F776E206572726F72DB
:10C0B40000756E6B6E6F776E0025633A203E3E3ED0
:10C0C400205A455048595220464154414C2045522B
:10C0D400524F522025643A202573206F6E2043501E
:10C0E400552025640A0025633A204661756C742046
:10C0F400647572696E6720696E74657272757074A6
:10C104002068616E646C696E670A0A0025633A20D0
:10C1140043757272656E74207468726561643A2046
:10C12400257020282573290A00574553545F544F1E
:10C13400504449522F7A65706879722F6B65726E1C
:10C14400656C2F666174616C2E6300726561736F38
:10C154006E20213D204B5F4552525F4B45524E4568
:10C164004C5F50414E49430009417474656D7074CD
:10C17400656420746F207265636F766572206672E1
:10C184006F6D2061206B65726E656C2070616E69E5
:10C194006320636F6E646974696F6E0A004350555F
:10C1A40020657863657074696F6E00556E68616EA2
:10C1B400646C656420696E74657272757074005382
:10C1C4007461636B206F766572666C6F77004B6584
:10C1D400726E656C206F6F7073004B65726E656C68
:10C1E4002070616E6963006D61696E006F73005742
:10C1F4004553545F544F504449522F7A65706879BF
:10C20400722F6B65726E656C2F7468726561642E33
:10C214006300282828287072696F2929203D3D2051
:10C224003135202626207A5F69735F69646C655F07
:10C234007468726561645F656E7472792828656ECE
:10C24400747279292929207C7C20282828313520DA
:10C254002D203129203E3D2028282D313629292919
:10C264002026262028287072696F2929203E3D2027
:10C2740028282D313629292026262028287072695D
:10C284006F2929203C3D20283135202D20312929B2
:10C29400290009696E76616C6964207072696F7235
:10C2A40069747920282564293B20616C6C6F77655B
:10C2B400642072616E67653A20256420746F2025BE
:10C2C400640A00286F7074696F6E73202620282812
:10C2D40031554C203C3C20283229292929203D3D38
:10C2E400203055207C7C207A5F737461636B5F69B6
:10C2F400735F757365725F63617061626C652873E7
:10C304007461636B290009757365722074687265C2
:10C3140061642025702077697468206B65726E658E
:10C324006C2D6F6E6C7920737461636B2025700AB9
:10C334000021617263685F69735F696E5F6973721C
:10C344002829000954687265616473206D6179203D
:10C354006E6F742062652063726561746564206920
:10C364006E20495352730A0025633A20737973632C
:10C37400616C6C202573206661696C656420636858
:10C3840065636B3A2062616420737461636B206F30
:10C39400626A6563740A0025633A20737973636182
:10C3A4006C6C202573206661696C65642063686524
:10C3B400636B3A20737461636B2073697A6520251B
:10C3C4007A7520697320746F6F206269672C206D01
:10C3D400617820697320257A750A0025633A2073F1
:10C3E400797363616C6C202573206661696C656484
:10C3F40020636865636B3A206F7074696F6E732095
:10C4040026204B5F555345520A0025633A20737921
:10C414007363616C6C202573206661696C656420AC
:10C42400636865636B3A2021286F7074696F6E735B
:10C434002026204B5F455353454E5449414C290A0D
:10C444000025633A2073797363616C6C2025732033
:10C454006661696C656420636865636B3A205F6933
:10C46400735F76616C69645F7072696F287072695A
:10C474006F2C204E554C4C290A0025633A207379C1
:10C484007363616C6C202573206661696C6564203C
:10C49400636865636B3A207A5F69735F7072696F72
:10C4A4005F6C6F7765725F6F725F657175616C2821
:10C4B4007072696F2C205F63757272656E742D3EA5
:10C4C400626173652E7072696F290A0074687265FF
:10C4D40061645F64617461203C3D205F5F737461DB
:10C4E4007469635F7468726561645F646174615FD9
:10C4F4006C6973745F656E640009756E6578706548
:10C5040063746564206C69737420656E64206C6F59
:10C51400636174696F6E0A00706F73203C3D205F25
:10C524007A5F6F626A6563745F61737369676E6D66
:10C53400656E745F6C6973745F656E64007A5F76B0
:10C544007266795F6B5F7468726561645F74696D4C
:10C55400656F75745F657870697265735F7469631C
:10C564006B73007A5F767266795F6B5F746872656D
:10C5740061645F74696D656F75745F72656D61691F
:10C584006E696E675F7469636B73007A5F76726657
:10C59400795F6B5F666C6F61745F64697361626C11
:10C5A40065007A5F6D7273685F6B5F746872656152
:10C5B400645F637265617465007A5F767266795F41
:10C5C4006B5F7468726561645F6372656174650052
:10C5D4007A5F767266795F6B5F7468726561645FB7
:10C5E400737461727400574553545F544F504449F7
:10C5F400522F7A65706879722F6B65726E656C2F35
:10C6040069646C652E63005F6B65726E656C2E6386
:10C614007075735B305D2E63757272656E742D3E3A
:10C62400626173652E7072696F203E3D2030005741
:10C634004553545F544F504449522F7A657068797A
:10C64400722F6B65726E656C2F6D757465782E63D1
:10C6540000096D7574657865732063616E6E6F741F
:10C66400206265207573656420696E736964652052
:10C67400495352730A006D757465782D3E6C6F636F
:10C684006B5F636F756E74203E20305500574553C1
:10C69400545F544F504449522F7A65706879722F11
:10C6A4006B65726E656C2F696E636C7564652F6B58
:10C6B40073636865642E6800090A005F6B65726EB7
:10C6C400656C2E637075735B305D2E637572726575
:10C6D4006E742D3E626173652E73636865645F6C6E
:10C6E4006F636B656420213D203155007A5F76725B
:10C6F40066795F6B5F6D757465785F756E6C6F637B
:10C704006B007A5F767266795F6B5F6D75746578BE
:10C714005F6C6F636B007A5F767266795F6B5F6DD7
:10C72400757465785F696E6974007A5F767266798C
:10C734005F6B5F71756575655F7065656B5F74616F
:10C74400696C007A5F767266795F6B5F7175657587
:10C75400655F7065656B5F68656164007A5F7672BA
:10C7640066795F6B5F71756575655F69735F656D2C
:10C77400707479007A5F767266795F6B5F71756544
:10C7840075655F676574007A5F767266795F6B5F63
:10C7940071756575655F616C6C6F635F70726570F0
:10C7A400656E64007A5F767266795F6B5F7175653A
:10C7B40075655F616C6C6F635F617070656E64005A
:10C7C4007A5F767266795F6B5F71756575655F63B5
:10C7D400616E63656C5F77616974007A5F76726617
:10C7E400795F6B5F71756575655F696E6974005714
:10C7F4004553545F544F504449522F7A65706879B9
:10C80400722F6B65726E656C2F73656D2E630028D5
:10C8140028617263685F69735F696E5F6973722808
:10C8240029203D3D203029207C7C20282874696DF6
:10C83400656F7574292E7469636B73203D3D2028E0
:10C8440028286B5F74696D656F75745F7429207B2C
:10C85400307D29292E7469636B732929007A5F76E8
:10C864007266795F6B5F73656D5F636F756E745F1E
:10C87400676574007A5F767266795F6B5F73656D66
:10C884005F7265736574007A5F767266795F6B5F59
:10C8940073656D5F74616B65007A5F767266795F4C
:10C8A4006B5F73656D5F67697665007A5F76726644
:10C8B400795F6B5F73656D5F696E6974005745538B
:10C8C400545F544F504449522F7A65706879722FDF
:10C8D4006B65726E656C2F73636865642E630021EB
:10C8E4007A5F69735F69646C655F746872656164BB
:10C8F4005F6F626A65637428746872656164290095
:10C904007468726561642D3E626173652E70656E34
:10C914006465645F6F6E005F6B65726E656C2E6339
:10C924007075735B305D2E63757272656E74202151
:10C934003D202828766F6964202A293029005F6BFE
:10C9440065726E656C2E637075735B305D2E6375F6
:10C954007272656E742D3E626173652E73636865D1
:10C96400645F6C6F636B656420213D203055002843
:10C974002828287072696F2929203D3D20313520EF
:10C984002626207A5F69735F69646C655F746872D8
:10C994006561645F656E74727928282828766F69EA
:10C9A40064202A293029292929207C7C2028282828
:10C9B4003135202D203129203E3D2028282D3136A7
:10C9C4002929292026262028287072696F292920E0
:10C9D4003E3D2028282D31362929202626202828A6
:10C9E4007072696F2929203C3D20283135202D2083
:10C9F400312929290025633A2073797363616C6CAA
:10CA0400202573206661696C656420636865636BC7
:10CA14003A20696E76616C69642074687265616439
:10CA2400207072696F726974792025640A00256325
:10CA34003A2073797363616C6C2025732066616995
:10CA44006C656420636865636B3A20746872656121
:10CA540064207072696F72697479206D6179206FD6
:10CA64006E6C7920626520646F776E6772616465AD
:10CA74006420282564203C202564290A00217A5F4B
:10CA840069735F7468726561645F73746174655F10
:10CA9400736574285F6B65726E656C2E6370757355
:10CAA4005B305D2E63757272656E742C202828319C
:10CAB400554C203C3C20283429292929000961624D
:10CAC4006F72746564205F63757272656E74206240
:10CAD40061636B2066726F6D20646561640A00098E
:10CAE40063616E6E6F74206A6F696E20696E20498F
:10CAF40053520A0025633A2073797363616C6C2086
:10CB04002573206661696C656420636865636B3AAC
:10CB14002061626F7274696E6720657373656E74E9
:10CB240069616C207468726561642025700A007AFA
:10CB34005F767266795F6B5F7468726561645F616A
:10CB4400626F7274007A5F767266795F6B5F776189
:10CB54006B657570007A5F767266795F6B5F746877
:10CB6400726561645F7072696F726974795F73650D
:10CB740074007A5F767266795F6B5F746872656160
:10CB8400645F7072696F726974795F676574007A43
:10CB94005F767266795F6B5F7468726561645F72F9
:10CBA4006573756D65007A5F767266795F6B5F7425
:10CBB40068726561645F73757370656E6400574570
:10CBC40053545F544F504449522F7A6570687972B8
:10CBD4002F6B65726E656C2F74696D656F75742E3D
:10CBE4006300217379735F646E6F64655F69735F5B
:10CBF4006C696E6B65642826746F2D3E6E6F646578
:10CC040029007A5F6D7273685F6B5F757074696D0C
:10CC1400655F7469636B7300574553545F544F5099
:10CC24004449522F7A65706879722F6B65726E650C
:10CC34006C2F6D656D706F6F6C2E6300616C69672E
:10CC44006E203D3D2030207C7C20282875696E7440
:10CC54007074725F74296D656D20262028616C697B
:10CC6400676E202D20312929203D3D203000096D9B
:10CC74006973616C69676E6564206D656D6F727947
:10CC84002061742025702028616C69676E203D2026
:10CC9400257A75290A007A5F767266795F6B5F661A
:10CCA400757465785F77616974007A5F7672667906
:10CCB4005F6B5F66757465785F77616B650025638C
:10CCC4003A204E554C4C206B5F6D656D5F70617200
:10CCD400746974696F6E2070726F76696465640A32
:10CCE4000025633A20706172746974696F6E2069FB
:10CCF40073207772697461626C6520616E6420656B
:10CD0400786563757461626C65203C7374617274D8
:10CD140020256C783E0A0025633A207A65726F20DC
:10CD240073697A656420706172746974696F6E20C6
:10CD340061742025702077697468206261736520AE
:10CD44003078256C780A0025633A20696E76616C28
:10CD5400696420706172746974696F6E2025702C27
:10CD6400207772617061726F756E6420646574659A
:10CD7400637465642E2062617365203078256C7855
:10CD84002073697A6520257A750A0025633A207034
:10CD94006172746974696F6E2025702062617365B5
:10CDA40020256C78202873697A6520257A752920D6
:10CDB4006F7665726C617073206578697374696EDF
:10CDC40067206261736520256C78202873697A6511
:10CDD40020257A75290A00574553545F544F50440F
:10CDE40049522F7A65706879722F6B65726E656C23
:10CDF4002F6D656D5F646F6D61696E2E6300646F86
:10CE04006D61696E20213D202828766F6964202A8F
:10CE14002930290074687265616420213D20282826
:10CE2400766F6964202A2930290025633A207061CD
:10CE3400727473206172726179206973204E554C4B
:10CE44004C20616E64206E756D5F70617274732026
:10CE54006973206E6F6E7A65726F0A0025633A20DB
:10CE64006E756D5F7061727473206F662025642027
:10CE740065786365656473206D6178696D756D208F
:10CE8400616C6C6F7761626C652070617274697437
:10CE9400696F6E7320282564290A0025633A206986
:10CEA4006E76616C696420706172746974696F6E06
:10CEB40020696E64657820256420282570290A007D
:10CEC4006D61785F706172746974696F6E73203C10
:10CED4003D20313600726574203D3D2030000966E6
:10CEE40061696C656420746F20696E69742064657F
:10CEF4006661756C74206D656D20646F6D61696E1B
:10CF04000A0025633A20556E696D706C656D656E17
:10CF14007465642073797374656D2063616C6C0A45
:10CF24000025633A204261642073797374656D202F
:10CF340063616C6C20696420256C7520696E766F62
:10CF44006B65640A003F00574553545F544F504487
:10CF540049522F7A65706879722F6B65726E656CB1
:10CF64002F7573657273706163652E63006F626AF7
:10CF740020213D202828766F6964202A2930290041
:10CF840009737461636B206F626A656374206E6FEA
:10CF94007420666F756E640A006F626A2D3E747940
:10CFA4007065203D3D204B5F4F424A5F54485245D7
:10CFB40041445F535441434B5F454C454D454E54AA
:10CFC400000962616420737461636B206F626A6537
:10CFD40063740A0025633A202570206973206E6FFC
:10CFE4007420612076616C69642025730A002563CE
:10CFF4003A2061646472657373206973206E6F7480
:10D004002061206B6E6F776E206B65726E656C208D
:10D014006F626A6563740A0025633A20616464720E
:10D024006573732069732061637475616C6C792016
:10D03400612025730A0025633A207468726561646F
:10D04400202570202825642920646F6573206E6F65
:10D05400742068617665207065726D697373696F99
:10D064006E206F6E2025732025700A007065726D26
:10D07400697373696F6E206269746D6170002563F2
:10D084003A2025730A0025633A20257020757365BC
:10D0940064206265666F726520696E697469616C8B
:10D0A400697A6174696F6E0A0025633A20257020DD
:10D0B400257320696E207573650A0025633A206F15
:10D0C4007574206F6620746872656164207265737C
:10D0D4006F7572636520706F6F6C206D656D6F7214
:10D0E400792028257A75290A0025633A20737472F9
:10D0F400696E6720746F6F206C6F6E6720257020D7
:10D1040028257A75290A0025633A206F76657266A8
:10D114006C6F770A0067656E65726963006B5F6D9B
:10D12400656D5F736C6162006B5F6D736771006B3B
:10D134005F6D75746578006B5F70697065006B5F17
:10D144007175657565006B5F706F6C6C5F73696793
:10D154006E616C006B5F73656D006B5F737461630C
:10D164006B006B5F746872656164006B5F74696DFA
:10D174006572007A5F7468726561645F7374616379
:10D184006B5F656C656D656E74004E45545F534FFF
:10D19400434B4554006E65745F6966007379735F31
:10D1A4006D75746578006B5F6675746578006B5F88
:10D1B400636F6E647661720063727970746F206459
:10D1C400726976657200616463206472697665725F
:10D1D40000626272616D2064726976657200636FC9
:10D1E400756E7465722064726976657200646D612F
:10D1F400206472697665720065635F686F73745F3B
:10D20400636D645F7065726970685F6170692064E2
:10D21400726976657200656461632064726976651B
:10D224007200656570726F6D206472697665720054
:10D23400656E74726F7079206472697665720065C8
:10D244007370692064726976657200657370695FD2
:10D254007361662064726976657200666C617368D6
:10D264002064726976657200667067612064726911
:10D27400766572006770696F206472697665720002
:10D28400693263206472697665720069327320645E
:10D2940072697665720069706D2064726976657270
:10D2A400006B7363616E20647269766572006C65ED
:10D2B4006420647269766572006D626F78206472AE
:10D2C40069766572006D64696F206472697665724F
:10D2D4000070696E6D75782064726976657200708D
:10D2E400733220647269766572007074705F636C67
:10D2F4006F636B206472697665720070776D206469
:10D30400726976657200726567756C61746F7220FC
:10D314006472697665720073656E736F72206472ED
:10D324006976657200737973636F6E2064726976CF
:10D334006572007561727420647269766572007733
:10D3440064742064726976657200756172745F6DCD
:10D3540075782064726976657200697473206472EA
:10D364006976657200706369655F6374726C2064CA
:10D37400726976657200697673686D656D20647292
:10D38400697665720065746870687920647269767C
:10D39400657200757365725F636F70790076332E02
:10D3A400302E302D7263312D3332312D67333232CA
:10D3B400623036366134373864002A2A2A20426FB4
:10D3C4006F74696E67205A6570687972204F5320B4
:10D3D4006275696C64202573202573202A2A2A0A21
:10D3E40000574553545F544F504449522F7A657047
:10D3F4006879722F6B65726E656C2F6B68656170EE
:10D404002E630068203C3D205F6B5F686561705F40
:10D414006C6973745F656E640021617263685F692F
:10D42400735F696E5F6973722829207C7C202828C9
:10D4340074696D656F7574292E7469636B73203D0F
:10D444003D202828286B5F74696D656F75745F745F
:10D4540029207B307D29292E7469636B732900256B
:10D46400633A2073797363616C6C20257320666161
:10D47400696C656420636865636B3A206F626A65F2
:10D484006374202570206163636573732064656E23
:10D494006965640A007A5F767266795F6B5F6F62B2
:10D4A4006A6563745F72656C65617365007A5F7643
:10D4B4007266795F6B5F6F626A6563745F616363F1
:10D4C4006573735F6772616E74000000030B171756
:10D4D4001517171717171717170B171717171717E6
:10D4E400170A1717171717171217171717171717DA
:10D4F40017171717091717170F1717170B171717DA
:10D504000F171717171717171717171717171717AF
:10D514000D171717171717170D17171717171717AB
:10D5240017171717171717170B1717171717171793
:10D534000B17171717171717171717171717171783
:10D544000917171717171717091717171717171783
:10D554001717171717171717071717171717171767
:10D564000717171702170100171717171717171799
:10D574000317171717171717001717171717171762
:10D58400171717171717171702171717091717174A
:10D594001717171717171717171717171717171717
:10D5A400011717171717171717171717171717171D
:10D5B400081717171717171700171717171717171D
:10D5C400171717171717171717171717000800003B
:10D5D400C01F0021000A0000C02300210000000039
:0CD5E4000000000000000000000000003B
:10D5F000000000000000000000000000000000002B
:10D60000000000000000000000000000000000001A
:10D61000000000000000000000000000000000000A
:10DDF0000386060195190601958D06010B93060110
:10DE00000000000005930601000000000000000073
:10DE10000000000000C2010000000000000000003F
:10DE2000010000000030304901010000003030499D
:10DE3000010200000030304900C201000000000073
:10DE40000000000001000000004030490101000016
:10DE500000403049010200000040304900C201008A
:10DE600000000000000000000100000000503049E8
:10DE7000010100000050304901020000005030490B
:10DE800000C20100000000000000000001000000CE
:10DE900000603049010100000060304901020000CB
:10DEA0000060304900C201000000000000000000D6
:10DEB000010000000070304901010000007030498D
:10DEC00001020000007030499828002198280021A4
:10DED0000000000000000000000000000000000042
:10DEE0000000000000000000000000000000000032
:10DEF0000000000000000000000000000000000022
:10DF00000000000000000000000000000000000011
:04DF1000000000000D
:10DF1400E4280021E42800210000000000000000A3
:04DF24000E000000EB
:10DF2800AC9B06010000210800000000EC9A0601E5
:10DF38000000300800000000D49A060100003008F4
:10DF480000000000BC9A0601000020080000000044
:10DF5800A49A060100002008000000009800002193
:10DF68000000090002000000000000210000090074
:10DF780000000000949B060100002108000000003A
:10DF88008C9A060100002008000000007C9B060116
:10DF98000000210800000000749A06010000200813
:10DFA80000000000649B060100002108000000003A
:10DFB8005C9A060100002008000000004C9B060146
:10DFC8000000210800000000449A06010000200813
:10DFD80000000000349B060100003008000000002B
:10DFE8002C9A06010000200800000000E428002107
:10DFF80000000301000000001C9B0601000030081F
:10E0080000000000C015002100000B00D8D5060153
:10E01800C00D002100000B00D0D50601049B0601AD
:10E028000000300800000000300100210000090055
:10E0380001000000F8FF00000000000000000000E0
:10E0480000000000000000000000000000000000C8
:10E0580000000000000000000000000000000000B8
:10E0680000000000000000000000000000000000A8
:10E078000000000000000000000000000000000098
:10E088000000000000000000000000000000000088
:10E098000000000000000000000000000000000078
:10E0A8000000000000000000000000000000000068
:10E0B8000000000000000000000000000000000058
:10E0C8000000000000000000000000000000000048
:10E0D8000000000000000000000000000000000038
:10E0E8000000000000000000000000000000000028
:10E0F8000000000000000000000000000000000018
:10E108000000000000000000000000000000000007
:10E1180000000000000000000000000000000000F7
:10E1280000000000000000000000000000000000E7
:10E1380000000000000000000000000000000000D7
:0CE14800000000000000000000000000CB
:04000005010622814D
:00000001FF
